:020000040000FA
:1000000000F80202B5700000FD34000079420000E3
:1000100000000000000000000000000000000000E0
:1000200000000000104E0100584E0100FD34000099
:100030000000000000000000FD340000E176000038
:10004000F5320000FD340000FD340000D5700000E2
:10005000814A0000B56B00008D340000813500003E
:100060005918000095170000FD340000013500000C
:10007000554A00001D8C0000557000008170000082
:10008000FD340000FD340000FD340000357A00002E
:10009000557A0000FD340000FD340000FD340000FE
:1000A000E97E0000F37E0000F7320000696F000077
:1000B000FD3400001D6C0000000000000000000086
:1000C0000348854600F016FF004800479DC9000020
:1000D00000F8020230B50B46014600202022012420
:1000E00009E00D46D5409D4205D31D469540491B6C
:1000F0002546954040191546521E002DF1DC30BDB5
:1001000070B500242546002801DA01244042002968
:1001100001DA01254942FFF7DDFFAC4200D0404241
:10012000002C00D0494270BDF8B5002425460029B6
:1001300004DA0E46012400214042B141002B04DACA
:100140001E46002352420125B34100F0D1FC8C46EB
:1001500017461E46AC4203D0002540428D41AC46B6
:10016000002C02D0002657429E4161463A46334653
:1001700001B0F0BD03460B439B0703D009E008C95B
:10018000121F08C0042AFAD203E00B780370401C47
:10019000491C521EF9D27047D2B201E00270401CD5
:1001A000491EFBD270470022F6E710B513460A46F7
:1001B00004461946FFF7F0FF204610BDCAB2401EA4
:1001C0004178401C8A4202D00029F9D100207047B2
:1001D000421C0178401C0029FBD1801A704730B5C1
:1001E00004460020034600E05B1C934203D2E05C1F
:1001F000CD5C401BF8D030BD30B50546002003462D
:1002000000E05B1C934205D2EC5CC85C201A01D173
:10021000002CF6D130BD00000FB400B58DB00990B0
:100220000B9010A900200091C0430A9000200C9070
:1002300006480690064807906A4609A80F9900F0FC
:10024000C1FC0DB008BC04B018470000E50B00006D
:10025000050C0000FFB5002083B0009050680190AD
:1002600091691446002697680498884705460C99BA
:100270000698084305D009E0A169761C04988847D0
:100280000546216A284688470028F5D1681C03D016
:100290000198C00704D017E00020C04307B0F0BDAC
:1002A0002068011D2160006800900DE00198C007E2
:1002B00004D1009805700098401C0090A169761C3C
:1002C0007F1E049888470546002F1CDD681C1AD045
:1002D000069800280FD0E817C00E401941118A0077
:1002E00006994009511840012A1A096801209040D6
:1002F0000142DBD107E00C980028D7D1216A2846BB
:1003000088470028D2D0E169049888470C980028D3
:1003100007D1002E05DD0198C00702D10098002109
:100320000170A068B84204DD0C98002804D0002FAA
:1003300002D00120C043B1E73046AFE770B50646B2
:1003400011F0CAF8046805460A220021304600F080
:10035000C5FC2C6070BDF8B502464A40D40F42007F
:100360004B0052085B089A4202D2024608461146E8
:100370004A0023D0C30D4A00DDB2120EAD1A202D63
:1003800035DA49020126490AF6058A19002C00D0FF
:10039000524220214F1B1146B9402A411018C20D6C
:1003A0009A4221D0002C17D0012D08DCDA05801AE2
:1003B000D20F8019D207DBB200F0D0FCF8BDDA050D
:1003C000801A012340001B06C01880185A4280186A
:1003D000CA0F1043490007E04908C2071143DA0574
:1003E000801A80194008801800F0B0FCF8BD610048
:1003F0000122511A001BF7E70122D2075140AAE758
:100400000122D2075040A6E7024670B54A40D30FFA
:10041000DB0740002DD04A002AD0010E140E000246
:1004200012020919400A520A8418E501044654438D
:10043000000A120A2E045043A4194219200CC54385
:10044000AA18120C0125AD03521C521912047F394F
:10045000240400D0521C104301D44000491EC2B2F3
:100460000C06C0092018401C4008802A02D003E076
:10047000002070BD40084000002900DA0020184329
:1004800070BD70B502464A40D50F40004A00ED07E6
:1004900040085208002814D0002A12D0C40DD30DF1
:1004A00041020120C0055202490A520AE41A091801
:1004B00012187D34914201D3641C00E04900002CE5
:1004C00001DA002070BD0023914201D3891A034351
:1004D000400849000028F7D100290AD0914202D1F2
:1004E0000121C90705E0914201D2012101E001216A
:1004F000C943E005C018401900F028FC70BD000099
:10050000F0B507460846584087B0C00F0490480031
:100510000E46590040084908BC1A884105D23846A1
:1005200031461E4617460B46024658004008104307
:100530004CD0300D039040055900400D490D0590F9
:10054000401A0290402872DA18030121000B0905B5
:100550000843019004980092002805D00199524266
:100560000020884100920190029840210A1A0199C6
:10057000009800F0EDFA05460C466B4607CB00F0FC
:1005800008FBC0197141039A0E0D0023D71756407E
:100590001A467A40164344D0049A002A2DD0029A73
:1005A000012A039A15DC1205C01A9141012636056D
:1005B000001C7141D20F059ED20700930192029652
:1005C0002A46234600F010FC07B0F0BD38463146FD
:1005D000FAE71605224A0F46B218C01AB7410121A0
:1005E0000905001C4F4100187F4111461818794138
:1005F000E20F10436D19644113E0E2076D081543E3
:100600006408C2071443039A01261205C01A9141D7
:100610003605001C7141CE07400830434908C01818
:1006200051412A46234600F0D2FBCDE7FFE704986C
:1006300001224000C117121A00238B410498314651
:10064000C417381AA141EEE730B40124E40763402F
:1006500030BC55E730B40124E407614030BC4FE7BB
:100660000000E0FFF0B51FB488B00B990998002492
:1006700048400999C00F490049080991C0070B99E2
:100680000090490049080B9109990898A64608432B
:100690001CD00B990A98084318D0099801244000EF
:1006A000420D4800410D099824050003000B20432A
:1006B00009900B980003000B20430B9050181C4925
:1006C0004018002201901446104605E00020014623
:1006D0000DB0F0BD032801DA034600E003239C4679
:1006E000C11A0AAE0AE05F0008ADED5B4F00F75B90
:1006F0007D430027AA187C41491C5B1E6145F2DD41
:10070000410004AB5A522104120C0A43240C401C31
:100710000828DFDB01980290009970460191009053
:10072000059B049A0799069800F05EFBD0E700004D
:100730000DFCFFFFF0B50C465C4085B0E40FE4070C
:1007400003944C0000266408590094464908024668
:100750000296224321D062460A431ED06200570D02
:100760004A000E032303550D012402462C4924059B
:10077000781B1B0B360B4018234326436146009021
:100780001C46501AB44103D30098401C009002E06C
:10079000921800985B41002803DA0020014605B05A
:1007A000F0BD0020012109050746864611E0644698
:1007B0001D46141BB54106D36546521BB341744612
:1007C00007430C43A646CD07400849082843921822
:1007D0005B4105460D43EAD11046184313D06046ED
:1007E000194650407140084306D06046101AB34184
:1007F00006D20122002306E000220123DB0702E0EB
:100800000122D2435310009874460105381C6141FF
:10081000029C039D0019694100F0D9FABFE700006E
:10082000FD0300000122D207002800DB101A002976
:1008300000DB511A814201D8012070470020704727
:100840000122D207002800DB101A002900DB511A10
:10085000814201D201207047002070470122D20757
:10086000002800DB101A002900DB511A814201D355
:1008700001207047002070470122D207002800DBCA
:10088000101A002900DB511A814201D9012070475A
:10089000002070470122D207002800DB101A00292F
:1008A00000DB511A814201D10120704700207047BE
:1008B00010B5002904DB0C460121C9074042A141C3
:1008C000002B04DB1C460123DB075242A341801AA4
:1008D000994101D3012010BD002010BD10B50029A1
:1008E00004DB0C460121C9074042A141002B04DB77
:1008F0001C460123DB075242A341101A8B4101D34E
:10090000012010BD002010BDC217C10F504010B50E
:100910004018CA079623002100F020FA10BD10B538
:1009200000229623114600F019FA10BD0EB5C21729
:10093000C10F5040CA0740180021054B0293019295
:1009400000910A460B4600F04FFA03B000BD0000CC
:10095000330400000EB505490291002100910A46BA
:100960000B46019100F040FA03B000BD33040000D3
:100970003EB5CA17CB0F002450405140C01861410A
:10098000DA07054B0293019200942246234600F0B9
:100990002BFA03B030BD000033040000C20F410049
:1009A00040020123400ADB05D207090EC0187F2947
:1009B00001DA00207047962903DC9623591AC840B3
:1009C00001E096398840002AF4D040427047410047
:1009D00040020122400AD205090E80187F2901DA5F
:1009E00000207047962903DC9622511AC8407047B0
:1009F000963988407047000070B5CD0F4A00090352
:100A00000123090B1B0519430B4BED070024520D65
:100A10009A4201DA002070BD074B34339A4203DC5E
:100A20009A1A00F0A5F802E00449511888402C43B6
:100A3000F1D0404270BD0000FF030000CDFBFFFF7E
:100A400070B5CD0F4A0009030123090B1B0519439B
:100A50000D4BED070024520D9A4202DA00200146A8
:100A600070BD094B34339A4203DC9A1A00F080F8C7
:100A700003E0064BD21800F06BF82C43F0D00022B4
:100A800040428A41114670BDFF030000CDFBFFFFCD
:100A9000C20FD207400040080BD0C10D0723DB0175
:100AA000C91840020905400A1143C2084007114312
:100AB0007047002001467047CB0FDB07490010B597
:100AC000490802460A4307D00A0D07240903E40136
:100AD000090B121B002A01DC002010BDC900440FC5
:100AE0000C43C100E018D205801800F02FF910BDAA
:100AF000F0B51FB40646002082B00546402401919F
:100B000000901BE0019922460F46304600F030F875
:100B1000049A059B801A994110D310461946224623
:100B200000F016F8361A8F41019722460120002165
:100B3000009F00F00DF838184D4100902046641ECB
:100B40000028DFDC019B00982946324607B0F0BD43
:100B500010B5202A04DB0146203A9140002010BD48
:100B6000914020239C1A0346E3401943904010BD56
:100B700010B5202A04DB0846203AD040002110BDE1
:100B80000B46D340D0402024A21A91400843194676
:100B900010BD10B5202A06DBCB170846203A1041BD
:100BA000C1170B4306E00B461341D0402024A21A84
:100BB00091400843194610BD02681378511801602E
:100BC0001846704710B5D16004495161044911625B
:100BD00000211161114600F0ADF910BDB90B000004
:100BE000210F00004268002A08D001680B78491CD8
:100BF000002B03D0521E06C0184670470121C16069
:100C0000881E70474268002A0BD0C3680168002B19
:100C100007D183688B4204D0491E521C06C00020B5
:100C200070470020C04370470FB400B589B00A4632
:100C30000DA9009100230C99002ACB60234B069349
:100C4000234B079301D0042300E00023214A0292A2
:100C5000214A0892019302466B46002000F095FB62
:100C600009B008BC04B01847F0B585B007460020AD
:100C7000C04301901E46002015460C46009102918B
:100C800004903B466A46314604A8FFF7CDFF04991D
:100C900002466018002D05D0002901D0034600E06F
:100CA00023462B6000290ED0002A02DD00998142E4
:100CB00009D0001B019000943B466A4631460294DD
:100CC00004A8FFF7B1FF05B0F0BD0000E50B000080
:100CD000050C0000FFFFFF7F210F0000F7B5009C0F
:100CE0000F4600262578641C002D05D000F014F96D
:100CF0000068405DC007F5D12B2D02D02D2D18D0F6
:100D0000641E39462046029A00F06AFC002F04D087
:100D10003968A14201D10099396071050224002986
:100D20000BDA4042002803DD10F0D6FB0460A00778
:100D3000FEBD012080020643E3E70028F8DA10F048
:100D4000CBFB04600048FEBDFFFFFF7F002904DAF3
:100D5000401C490001D140084000704770B4002495
:100D6000050C05D11024000402D1002921D0112442
:100D7000050E01D100020834050F01D10001241D28
:100D8000850F01D18000A41C002801DB4000641CF9
:100D9000002908D020252E1B0D46F540A14000D08B
:100DA00001212943084301061B1B000ADB1D02D554
:100DB000002070BC7047DB05181880180029F8DA8D
:100DC000401C4900F5D170BC40084000704710B588
:100DD000002B08DA0024401C614192185B411A4341
:100DE00001D14008400010BDF0B51FB482B00546E7
:100DF0000C0003D0084610F057FB02E010F054FB43
:100E000020300246009021462846FFF7A1FE049BB1
:100E1000059A04460F4618431143084314D0184658
:100E200010431BD0009840210A1A18460599FFF775
:100E30009FFE05460E46009A05990498FFF788FE26
:100E4000084305D0012004E02046394607B0F0BD34
:100E50000020C11705430E432C43374300990E98D9
:100E60006305401A7905E40A00220C43FD0A0A30A2
:100E700002D500200146E9E70105101969410C9CE3
:100E80000D9D00196941FFF7A2FFDFE74A00090342
:100E90000123090B1B0519430A4B10B5520D9A4249
:100EA00002DA0020014610BD064B34339A4203DCBF
:100EB0009A1AFFF75DFE10BD034BD218FFF748FEEC
:100EC00010BD0000FF030000CDFBFFFF10B500299F
:100ED00004DB0124E40740428C412146002B04DB63
:100EE0001C460123DB075242A341994200D19042A4
:100EF00010BD0000064C0125064E05E0E36807CC56
:100F00002B430C3C98471034B442F7D3FFF7DCF87E
:100F1000504801007048010000487047741E0100ED
:100F200010B50446FFF7F8FF0068005DC007C00F6A
:100F300010BD0000F3B58DB000200A9001200B9089
:100F4000002608460C300C46099062690121099878
:100F50009047051E2ED0252D2DD0216A88470028C8
:100F600018D06269012109989047216A88470028B2
:100F7000F7D1411E62690998904700E0761CA1698B
:100F80000D988847216A88470028F7D1E1690D98B4
:100F90008847DAE7A1690D9888470746A84201D13A
:100FA000761CD2E7E1690D9888477F1C02D10A9828
:100FB000002877D049E1002762693D463946099803
:100FC00090472A280CD16269012109989047012590
:100FD00006E00A214F433F18303FEBD41020054371
:100FE0006269012109989047014630390A2903D2E4
:100FF0009B498F42DEDCECE7E90600D4994F6C2870
:101000000AD04C2810D0682824D06A282ED0742802
:101010000CD07A280AD00DE0626901210998904726
:101020006C2823D004211CE02020054362690121A3
:1010300009989047A760656065284FD026DC58283E
:1010400039D01ADC452849D012DC252834D0412873
:10105000B0D143E06269012109989047682802D025
:1010600008210D43E6E70120C002DEE70220DCE7AD
:10107000462833D047282CD130E05B2870D0612837
:101080002CD063286CD0642823D161E06F284FD026
:1010900009DC662822D0672820D0692826D06E284F
:1010A00017D12EE0CDE070284DD073286FD0752871
:1010B0004ED078280DD154E0A1690D988847054697
:1010C000252800D16CE7E1690D9888476D1C00D197
:1010D0006DE7BAE00A224CE00A2252E001202346E2
:1010E0006A46C0430D9900F050F9A3E0284640211C
:1010F00008436060A807234601D5002239E000229A
:101100003FE0E80700D020E72068011D216000686B
:10111000290501D5067018E7290701D5068014E7CF
:10112000A90703D5F117066041600EE706600CE7DA
:101130002846402108436060A807234601D50822BD
:1011400017E008221DE0484928460840606016E084
:101150002846402108436060A8072346BCD5B9E76C
:1011600015E02846402108436060A80707D52346BC
:1011700010220120C0430D99C046C0465AE02346C4
:1011800010220120C0430D99C046C04652E0002104
:101190000C910B460091632802D05B2807D043E0F6
:1011A000E80601D40120A060012000903CE06269C3
:1011B0000121099890475E2805D101200C90014635
:1011C0006269099890472169002906D10B4601AA56
:1011D0008F00491CD3510829FADB002835D021693A
:1011E00000290ED1C117C90E09184A11930001AA8E
:1011F0009A1849094901411A01201368884003439C
:10120000136062690121099890475D28E5D10C9827
:10121000002808D0002001AB81005A58401CD2435E
:101220005A500828F8DB01AB01202246C0430D9933
:10123000FFF710F800280ADA401C06D10B980028A6
:1012400003D00020C0430FB0F0BD0A98FBE7E907C8
:1012500002D10A99491C0A91361800200B9074E6B5
:10126000CCCCCC0CFFFFFF7FF1F7FFFFFFB5087878
:1012700089B01546FF2805D0491C2D2804D000222E
:10128000002407E000240BE00122F9E70A235C4375
:101290000419491C0878FF28F8D1002A00D06442BC
:1012A000002004902A7801462D2A01D02B2A0FD144
:1012B0006D1C2D2A02D00022049209E00122FBE7D6
:1012C00000260A2233466D1C00F0DDF93818714102
:1012D0002F78FF2FF4D10C9AA218069202460A43E7
:1012E00004D0FF23069A9133DA4205DA00210998E7
:1012F0000A4606C00DB0F0BD0024B74AB54D2646DB
:10130000079200F00DFA029006980391002801DA86
:10131000474200E0074639050020AF4A001C514112
:101320000191009012E0F80707D022462B46304684
:101330000799FFF797F90646079122462B46104674
:101340001946FFF78FF904460D467F10002FEAD1AA
:101350000698019B0028009A0399029806DAFFF785
:10136000E9F93246079BFFF7E5F905E0FFF77AF95F
:101370003246079BFFF776F9049A002A02D0012231
:10138000D2075140099A03C2B4E7FFB591B00020DB
:1013900009900025ED432E209E685C681F46019051
:1013A000B9696D1C129888470090396A88470028EF
:1013B000F6D10098401C0AD00D20C0018443002EB5
:1013C00012DD00982B2809D02D280DD103E0002034
:1013D000C04315B0F0BD012080020443B9696D1C03
:1013E00012988847761E009003A9600501D52D202C
:1013F00000E02B206A461073491C0CA80F91029044
:101400000AE0B9696D1C12988847009001204002DB
:1014100004431398761E0560002E02DD00983028E4
:10142000EFD001990098884245D18020044308E01C
:101430000998401E09900120400204431399681C3A
:101440000860B9696D1C761E129888470090302894
:10145000EED030E00199884205D1200603D48020E7
:101460000443761E1DE0009810F004F9002825D0F2
:10147000012149020C43009807AA0F990332303822
:10148000761E914208D208700F98401C0F902006DB
:1014900007D50998401E03E0200602D40998401C95
:1014A0000990A00502D51399681C0860B9696D1CE4
:1014B000129888470090002ECCDC59E0002E57DDB2
:1014C0000098652801D0452852D1A00550D50320A9
:1014D00000028443B9696D1C761E129888470090FB
:1014E000002E0CDD2B2804D02D2808D1FF20013040
:1014F0000443B9696D1C12988847761E0090E00578
:1015000001D52D2100E02B21029801700298401C8A
:101510000290019025E00120400204430EA90298A8
:101520000131761E88420ED20098029930380006AA
:10153000000E087003D10299019881420AD90298DD
:10154000401C029006E0E00501D5244801E0234854
:1015500040420990B9696D1C129888470090139811
:101560000560002E04DD009810F084F80028D2D128
:10157000F969129888470F99FF200870029903AA09
:10158000087000200A900B900CA90AA8099BFFF78D
:101590006DFEA00502D40120C0431AE724200442B6
:1015A00009D0E00713D138680B9A0A99031D3B60F4
:1015B000006806C00BE00B990A98FFF77DFA014618
:1015C000E00704D13868021D3A60006801602846CF
:1015D000FFE60000000014400000F03FF1D8FFFFDC
:1015E000F7B582B0029C00272078641C154601974D
:1015F000302802D0002D15D015E020780127641C7A
:10160000782804D0582802D0002D09D00BE0002DF6
:1016100001D0102D07D1002710252078641C02E08E
:10162000082500E00A250026009610E00099012711
:1016300069430818020C294680B2714300908E1845
:101640003804864201D3012001902078641C294689
:1016500000F056F80028E9DA0398002805D0002F9A
:1016600001D0641E00E0029C04600198002806D0AE
:101670000FF032FF02210160C81E05B0F0BD0099D5
:1016800030040843F9E7F0B51FB486B0002000909D
:10169000019002900698069980B204900798090C70
:1016A00002040014114307900027089D0998069131
:1016B0003E463C4603900398A9B20204000C0390F6
:1016C00004982D0C1543484300212246FFF740FAA9
:1016D000C719714110340E46402CECDB3846029A93
:1016E000FFF736FA009A019B801800905941029842
:1016F0000191103002904028CCDB00980BB0F0BD77
:101700003A2800D23038202302469A43412A01D396
:1017100010463738884201D30020C043704700008C
:101720000EB5054A02920022009213460192FFF77D
:101730005BFB03B000BD00003304000070B58C18E3
:101740000578401C6B075B0F01D10378401C2A1100
:1017500006D10278401C03E006780E70401C491C3C
:101760005B1EF9D12B0705D40023521E0DD40B703C
:10177000491CFAE70378401CCB1A921C03E01D7841
:101780000D70491C5B1C521EF9D5A142D8D3002014
:1017900070BD000010B52148016A8A0715D44A07B8
:1017A00015D4C90732D01E498A89002A15D0531E84
:1017B0008B8182688C6904C48C610A691B040DD01A
:1017C000002A22D10121016010BD022100E0042184
:1017D000C16113488021416110BD0A69012A09D104
:1017E000026801239A430260C361FF206830993088
:1017F0000C4A106001204861CA69002A05D0886936
:1018000009898B00C01A904710BD10BDFF226832B5
:10181000054806A109A30DF0C1FAC04608D0014051
:10182000A095010280E200E0C82D01004144435F21
:1018300049525148616E646C65720000556E65785E
:101840007065637465642041444320696E746572F9
:10185000727570740D0A000070B582B00023019398
:10186000444801688A6A4C6813252540132D02D12B
:10187000CB689B07DB0F4361930772D453070AD4ED
:10188000D30711D1130724D5048F838E1C1B102C72
:101890000EDD102310E0042088620220032142A202
:1018A0000EF0D8FA02B070BD0120886202B070BD9F
:1018B000048F1B1B1C0610D0DBB20024058FC66AE8
:1018C00075192D5D0D74641CA342F7D1048FE318C4
:1018D0000387D20607D400212FE04B6A0824A343D4
:1018E0004B62D206F7D5CB68C28E448F141B5B04C3
:1018F000DB0EA34201D3438FD31ADAB2002A16D0EB
:10190000097D438F046BE1540199012A10D0012312
:101910001C46890145582D7D41184E8F9B19096B36
:10192000CD54641CE3B201999A42F2D800E0002140
:101930008B01C3185C8FA2185A878A0181184B8FBC
:10194000CC8EA3420BD301230B618058002242624C
:10195000CA6B002A03D03A31098801A8904702B027
:1019600070BD02208862044804A1084A08A30DF053
:1019700015FAC04674900102E12D01004145535F04
:1019800049525148616E646C65720000CE020000DD
:1019900041455320696E707574206F766572666C70
:1019A0006F770D0A00000000414553206F75747079
:1019B000757420756E646572666C6F770D0A000031
:1019C000F0B581B001243F2900D993E00346806837
:1019D000456B2D688E0001A7BE59B7461B1B000042
:1019E000371B0000131B0000131B0000F51A00003A
:1019F000F51A0000F51A0000F51A0000F51A0000AB
:101A0000F51A0000F51A0000F51A0000F51A00009A
:101A1000F51A0000491B0000651B0000F51A0000C4
:101A2000F51A0000F51A0000F51A0000F51A00007A
:101A3000F51A0000F51A0000F51A0000F51A00006A
:101A4000F51A0000F51A0000F51A0000F51A00005A
:101A5000F51A0000F51A0000F51A0000F51A00004A
:101A6000F51A0000F51A0000F51A0000F51A00003A
:101A7000F51A0000F51A0000F51A0000F51A00002A
:101A8000F51A0000F51A0000F51A0000F51A00001A
:101A9000F51A0000F51A0000F51A0000F51A00000A
:101AA000F51A0000F51A0000F51A0000F51A0000FA
:101AB000F51A0000DD1A0000DD1A0000DD1A000032
:101AC000DD1A0000DD1A0000DD1A0000DD1A00003A
:101AD000DD1A0000DD1A0000DD1A0000434800692D
:101AE0000024022809D001280DD0002802D103CA01
:101AF00004F0ACFF204601B0F0BD03CA04F098FF2B
:101B0000204601B0F0BD03CA04F0B6FF204601B084
:101B1000F0BD022931D0022430E0344D00242C6184
:101B20006C619849354A01F065FE6869401C68613E
:101B3000204601B0F0BD01F097FE284602F004F9FE
:101B40000024204601B0F0BD284909690C234B430D
:101B50002749CA58C918496801F04CFE002420469C
:101B600001B0F0BD0024204604F03EFF0128C1D1A1
:101B70001E483030204900241CE001241B490F6915
:101B80000C26314679431A4A51188968214208D0F7
:101B900000247D1C15490D614C61042D10D315499D
:101BA00006E012494869401C4861032812D32949BC
:101BB00000241846224602F077F8204601B0F0BD16
:101BC0006E430B498A598919496801F013FE204672
:101BD00001B0F0BD0E20009000240A2228462146C4
:101BE00002F052F8204601B0F0BDC046AC990102A7
:101BF000781E0100782501005825010046390100B2
:101C0000B0B504290FD804468068C04679440979E4
:101C100049008F44020A0E1C1700104910A201F05F
:101C2000E9FD0020B0BD0120B0BD01F01DFE002087
:101C3000B0BD00250321284604F0E6FE06492046F3
:101C40002A4602E003490022204602F02DF8002037
:101C5000B0BDC04668250100E825010088130000DA
:101C6000415445300D0A0000B0B582B001240A2964
:101C700010D883687944097949008F440E290505F5
:101C80000B0B0B0B0B0B1A00194909680024224699
:101C900002F00AF8204602B0B0BD5068144908604E
:101CA000144915A2184601F0A5FD0024204602B0F3
:101CB000B0BD0024019403CA09A201AB02F012F9DD
:101CC0000228E7D1019804F0F3FE204602B0B0BD2F
:101CD000184601F0C9FD0024204602B0B0BDC04640
:101CE0002B4353513A2025642C252A0D0A0000006D
:101CF000C89A01028813000041542B4353510D0A26
:101D000000000000B0B582B00546002404F0CAFE11
:101D100001280DD108498C60E86B426853684B601C
:101D2000009401926A4601F0BFFF204602B0B0BDA8
:101D3000E443204602B0B0BDC8930102B0B50546E9
:101D4000881E02280AD3A868012913D0002915D1BA
:101D50000C490DA201F04EFD0020B0BD022001464D
:101D600004F052FE064900242846224601F09CFF5A
:101D70002046B0BD01F078FD0020B0BD0120B0BD0F
:101D8000382501008813000041542B4346554E3D31
:101D9000300D0A00B0B5E0B00324E1016D462846DD
:101DA0000FF06AFB204621462A460EF053F8002029
:101DB00060B0B0BDF0B597B00820149064201390C7
:101DC0002548109002200E904B20C0011690234D04
:101DD00028461430129001270F97B8021190032063
:101DE0000EA906F081F90026F443002802D020460F
:101DF00017B0F0BD0C35284601F0B4FF0028F6D12D
:101E000080200C9016490B910A90164809901648AC
:101E100008901648079016480690392005901548F6
:101E20000490154803900D95144D03A9284601F020
:101E30004BFD0028DBD1009501970F4C104911A2F2
:101E4000124B204601F0E4FE1149204601F014FF38
:101E50003446204617B0F0BD48C001022497010265
:101E600048C40102C8C401024D2F00009D2F00008C
:101E70001D2F0000F8260100DC99010258C901025B
:101E8000D82401004149523738304500F825010077
:101E9000951D000010B50348002404700EF066FF85
:101EA000204610BDE09E010280B501F057F90020E8
:101EB00080BD0000F0B58DB00E4600270C970B9743
:101EC0000A970997089707970697059702908068E1
:101ED0000490406B0068019004F080FD04465BA113
:101EE00005220392FEF788F95A4D00281ED05AA108
:101EF00005222046FEF780F9002817D058A10522B8
:101F00002046FEF779F900280FD059A10522204676
:101F1000FEF772F9002809D057A105222046FEF7E6
:101F20006BF9002807D156A500E04FA505A8202190
:101F30002A4602F0A9F801203F2E00D936E0C0461B
:101F40007E4436797600B7443340474A57313131C1
:101F5000313131313131653031313131313131313E
:101F60003131313131313131313131313131313161
:101F700031313131313131313131313131311F1F75
:101F80001F1F1F1F1F1F1F1FBE48416A04290CD19E
:101F9000039A426287620C2050433D490A58081850
:101FA000416805AB049801F025FC38460DB0F0BD42
:101FB000B44C00206062A062CD49364A049801F01A
:101FC00019FCA06A401CA062EFE7049801F04CFCE9
:101FD000019801F0B9FEE8E7AA48406A05E0A9497E
:101FE000486A01220243032A1CD1A649421C4A62C4
:101FF0008F62062ACFD30BE0A2494A6A012013461A
:102000000343052BD2D1501C48628F62062803D3AC
:102010001E490DE09B48406A0C2141431C48425830
:102020004018BDE7886A401C8862032805D316491A
:102030000022029801F038FEB7E70E200090002140
:102040000A220198029B01F01FFEAEE734363030C1
:10205000300000006E3901003436303032000000AC
:102060003436303031000000554E494E45540000A2
:102070003436303036000000343630303300000063
:1020800043544E4554000000D82401002825010087
:10209000A81E0100EE38010070B5022956D30F29A1
:1020A00007D1784C217A012905D1002222728F496B
:1020B0004AE0012070BD866801F07AFE002004F03D
:1020C0009BFC012803D10020032104F09DFC002586
:1020D000284604F089FC012804D130346A490022E2
:1020E000204631E0304600F0EFFD00282ED030468B
:1020F000FFF708FE002829D004F090FC012807D142
:102100005F498D60F06B4268E26252684A601AE093
:10211000022004F069FC012808D159498D61F06B57
:102120004268E26252684A6110310CE0022004F019
:1021300063FC01280AD152498D62F06B4268E26269
:1021400052684A6220312A4601F0AEFD002070BD7F
:1021500010B582B003460120272931D87944097986
:1021600049008F442C132D2D162D2D2D2D2D2D2D69
:102170002D2D2D2C2D2D2D2D2D2D2D2D2D2D1C2DA1
:102180002D2D2D2D2D2D2D2D2D2D2D2905F034F816
:1021900015E0DF490022184601F086FD0FE000201F
:1021A000019003CA08A201AB01F09CFE012806D1F0
:1021B000019805F03DF902E002480121017200207A
:1021C00002B010BDAC9901022B51495552433A203F
:1021D00022636C6F736564222C25640D0A00000075
:1021E000B0B502294AD30F2914D18568002004F024
:1021F00003FC012803D10020032104F005FC002486
:10220000204604F0F1FB012806D1D94830301E49A0
:10221000002231E00120B0BD2846FFF773FD002801
:102220002CD004F0FBFB012808D115498C60E86B29
:102230004268CF4BDA6252684A601CE0022004F028
:10224000D3FB012809D10E498C61E86B4268C84B69
:10225000DA6252684A6110310DE0022004F0CCFBD2
:1022600001280BD106498C62E86B4268C04BDA62E8
:1022700052684A622031224601F016FD0020B0BDAE
:1022800040900102AC9901025825010080B5022955
:1022900005D3042905D19E49002201F005FD002047
:1022A00080BD012080BDC046B0B50546881E02280D
:1022B0000AD3A868012913D0002915D10C490DA211
:1022C00001F098FA0020B0BD0220032104F09CFB2D
:1022D000064900242846224601F0E6FC2046B0BD0F
:1022E00001F0C2FA0020B0BD0120B0BD7825010088
:1022F0008813000041542B4346554E3D310D0A00D2
:1023000010B50F290BD001291DD000291DD1FFF7D1
:10231000C1FD0020022104F077FB002010BD04461F
:10232000002004F061FB012803D10020022104F009
:102330006BFB002004F060FB012804D1044900225B
:10234000204601F0B1FC002010BD012010BDC046A8
:1023500068250100F0B581B00124322928D805464E
:102360008768786B0668C0467944097949008F44CC
:102370002F3F1919191F1F1F1F1F1F1F1F1F221F4C
:102380001F1F1F1F1F1F1F1F1F1F1F1F1F1F1F1F5D
:102390001F1F1F1F1F1F1F1F1F1F1F1F1F1F1F1F4D
:1023A0001F1F26001E4900242846224601F07CFCFF
:1023B000204601B0F0BD1B48017800291FD0184904
:1023C00000242846224601F06FFC204601B0F0BDF3
:1023D0000024FC623969384688470028FAD0114841
:1023E0000470FC62FFF756FD0E20009001220EE003
:1023F000304601F0A9FC0024204601B0F0BD0121C7
:102400000170FFF751FD0E20009000240522304698
:1024100021462B4601F038FC204601B0F0BDC046F5
:10242000F8240100CC9A010210B586B003460120C1
:102430003B2900D956E0C0467944097949008F44C8
:10244000505051513351515151515151515151519C
:10245000515151515151515151515151515151516C
:10246000515151515151515151515151515151515C
:102470005151515151391D1D1D1D1D1D002005902B
:1024800003CA02AA009218A205AB01F02BFD022894
:1024900027D1039A029817A1FDF7AEFE002820D19C
:1024A000059804F0C5FF1CE0B5490022184601F06C
:1024B000FBFB16E0002002900590049003CA05AAD9
:1024C000019204AA00920DA202AB01F00BFD0328B9
:1024D00007D1049A0599029805F04CF8029804F087
:1024E000EBFF002006B010BD25642C2025700D0ADE
:1024F00000000000434C4F53454400002B5245431D
:10250000454956452C25642C25643A0D0A2565005D
:1025100048250100012901D800207047012070479B
:10252000B0B50546881E03280BD2104604F07EFA8B
:102530000F48C16A00242846224601F0B5FB204618
:10254000B0BDAC6801290BD000290ED104F048FAC7
:102550000346084908A2204601F04CF90020B0BD0E
:10256000204601F081F90020B0BD0120B0BDC04679
:10257000AC9901028813000025730D0A00000000C9
:1025800070B582B001240F293DD803468568686B79
:102590000668C0467944097949008F4407141E34FF
:1025A0003434342F373434343434434E66480024C2
:1025B00004708461C461012101716649664A28463C
:1025C00001F018F91FE0284601F04EF9304601F0FD
:1025D000BBFB0024204602B070BD5B4800240471A0
:1025E0008269042111430278002A2ED0052958D18E
:1025F000016A491C016259D2624961E0524B187864
:102600000024002831D0204602B070BD4E4B18780F
:10261000012816D103CA183351A201F063FC00202F
:1026200002B070BD48480024846101210171007826
:102630004849002812D1484A11E0434E3079002819
:102640001BD00024204602B070BD052932D10024E1
:10265000012101708461C46101713E493F4A2846ED
:1026600001F0C8F8204602B070BD03CA183340A27A
:1026700001F038FC204602B070BD002004F0BCF927
:10268000012803D10020032104F0BEF900242046D4
:1026900004F0AAF9012816D130362D49002430461D
:1026A0004BE000210162C169491CC1610E2000900C
:1026B00000241CE0C169491CC161652915D330495A
:1026C0000024184639E02846FFF71CFB00289AD062
:1026D00004F0A4F9012812D11C4900248C60E86B95
:1026E0004268F26252684A6027E00E20009002229F
:1026F0003046214601F0C8FA204602B070BD0220E3
:1027000004F072F9012809D1104900248C61E86BAA
:102710004268F26252684A6110310EE0022004F011
:102720006BF9012800D06EE7084900248C62E86B41
:102730004268F26252684A622031224601F0B4FADD
:10274000204602B070BDC046AC9901024090010223
:1027500058250100881300000A39010015390100CD
:102760002B43475245473A20252A2C256400000078
:102770002B435245473A20252A2C256400000000AF
:102780004825010008250100B0B584B001243B298B
:1027900000D937E0134605468068C0467944097978
:1027A00049008F444B5532322F2F2F2F2F2F2F2F91
:1027B0002F2F2F2F2F2F2F2F2F2F2F2F2F2F2F2F29
:1027C0002F2F2F2F2F2F2F2F2F2F2F2F2F2F2F2F19
:1027D0002F2F2F2F2F2F2F2F2F2F1D1D1D1D1D1D75
:1027E0000024039403CB01AA00921C4A03AB01F01E
:1027F00079FB022806D1029A019819A1FDF7FCFC89
:1028000000280FD0204604B0B0BD1848006804F07E
:102810000FFE174900242846224601F045FA2046BB
:1028200004B0B0BD1148006804F002FE1049002257
:10283000284601F039FA204604B0B0BD0B490B60C0
:102840001E210CA200F0D6FF0024204604B0B0BD2B
:1028500001F00AF80024204604B0B0BD6E3A010031
:10286000434C4F5345204F4B00000000D09A0102CB
:102870001825010041542B434950434C4F53453DCB
:1028800025640D0A00000000F0B589B0044601205F
:102890003B2900D9AAE01646A7687A6B1568C0469E
:1028A0007944097949008F44536AA071A1A1A1A17B
:1028B000A1A1A1A1A1A18AA1A1A1A1A1A1A1A1A11F
:1028C000A1A1A1A1A1A1A1A1A1A1A1A1A1A1A1A1F8
:1028D000A1A1A1A1A1A1A1A1A1A1A1A1A1A11D1DF0
:1028E0001D1D1D1D0027089703CE06AA0092414A10
:1028F00008AB01F0F7FA022877D13F48056808983D
:10290000854272D1079A069E3CA130460592FDF79A
:1029100073FC002847D03DA13046059AFDF76CFCBA
:10292000002840D03CA13046059AFDF765FC002800
:10293000314E5AD1284604F095FD7068401C7060F5
:1029400003283CD303207060306804F013FD36E0A8
:1029500029480660304604F061FD0590264800686D
:1029600004F030FD04902448006804F037FD049919
:10297000019102900598012827D02EA026E0384624
:1029800000F072FF284601F0DFF92EE01A4D2868AA
:1029900004F068FD6868401C686003280FD30022BB
:1029A0006A6022490DE0144E7760284604F070FDFD
:1029B000306804F083FE002801D01B4900E00C4978
:1029C0000022204601F070F90FE019A000901A498A
:1029D0001AA23846334600F00DFF0E200090002169
:1029E000B4222846234601F04FF9002009B0F0BD7B
:1029F000182501006E3A01009C970102414C524596
:102A000041445920434F4E4E45435400434F4E4E90
:102A1000454354204F4B0000434F4E4E45435420F6
:102A20004641494C00000000B8250100D8240100AF
:102A300054435000554450008813000041542B4328
:102A4000495053544152543D25642C222573222C65
:102A5000222573222C25750D0A000000B0B582B026
:102A600014468A1E022A12D38568012917D000292C
:102A70001CD1204604F098FC00901E210EA228468E
:102A8000234600F0B7FE0024204602B0B0BD09493D
:102A90000024224601F008F9204602B0B0BD2846C5
:102AA00000F0E2FE0024204602B0B0BD0124204622
:102AB00002B0B0BDC825010041545E4845415254A2
:102AC000434F4E4649473D312C25642C25750D0A50
:102AD00000000000F0B583B014468A1E022A1CD301
:102AE0008568012921D0002926D1164F3C60204657
:102AF00004F04CFCFDF76CFB0646386804F046FC1D
:102B00007108009101901E210FA22846234600F073
:102B100071FE0024204603B0F0BD0949002422467E
:102B200001F0C2F8204603B0F0BD284600F09CFE3C
:102B30000024204603B0F0BD0124204603B0F0BDC0
:102B400018250100D49A010241545E48454152546F
:102B5000424541544845583D25642C25752C257324
:102B60000D0A0000F0B585B0044601203B2900D9CC
:102B700088E0A5687944097949008F444257825E0C
:102B80008383838383838383838383836383838335
:102B90008383838383838383838383838383838305
:102BA00083838383838383838383838383838383F5
:102BB00083831D1D1D1D1D1D0020049003CA02AA34
:102BC0000092314A04AB01F08DF9022859D12F4807
:102BD00085680498854254D1039E029F2CA13846F3
:102BE0003246FDF709FB00283DD02BA1384632467E
:102BF000FDF702FB002844D1284604F019FC2949BE
:102C00003BE0224CA260104604F0F4FB002838D0D0
:102C100001F0D1FAE060002833D0A368406800904A
:102C2000234924A2284600F0E5FD2AE017480021A8
:102C3000C160284600F018FE23E01448806804F0C4
:102C4000F7FB19E000F080FE012804D10F48C168AD
:102C500003C900F081FF0D48C0680CC8134928461D
:102C600000F008FE0DE0284604F0C4FB00280749E8
:102C700007D0C96801F075FA0B490022204601F01F
:102C800013F8002005B0F0BD6E3A01009C970102D8
:102C900053454E44204F4B0053454E442046414936
:102CA0004C0000004825010018250100204E0000BE
:102CB0008813000041542B43495053454E443D2551
:102CC000642C25750D0A0000F0B583B0074601F0AD
:102CD0006FF80026304604F097FB032835460BD1E9
:102CE0000421284604F0DCFCF86B51492A4600F028
:102CF000DBFF304603B0F0BD02970024204604F00D
:102D000083FB0428254609D10298C06B49492A460D
:102D100000F0CAFF2646304603B0F0BD0027384613
:102D200004F072FB05283D4609D10298C06B40496A
:102D30002A4600F0B9FF3E46304603B0F0BD019789
:102D40000125284604F060FB0328029FC8D0012516
:102D5000284604F059FB0428D6D00125284604F063
:102D600053FB0528019FE0D00225284604F04CFBC8
:102D70000328029FB4D00225284604F045FB04280E
:102D8000C2D00225284604F03FFB0528019FCCD085
:102D9000254C2068401C0321FDF7B2F90D4608467A
:102DA00004F032FB0628029F08D1284604F022FBDB
:102DB000002803D001F0FFF900282AD1681C032164
:102DC000FDF79EF90D46084604F01EFB062808D1C3
:102DD000284604F00FFB002803D001F0ECF900288E
:102DE00017D1681C0321FDF78BF90D46084604F046
:102DF0000BFB0021CE43062800D07AE7284604F0DA
:102E0000F9FA002800D174E701F0D5F9002800D1C3
:102E10006FE72560F86B05492A4600F045FF00265C
:102E2000304603B0F0BDC046D89A0102D825010053
:102E300098250100A825010080B58AB0062004214C
:102E400008F01EFE4B20C001099008200790642066
:102E50000690B44814300590064803900220019073
:102E60000120029080020490032001A905F03CF9A2
:102E70000AB080BD48C00102B0B582B001220F295E
:102E80003ED803468068446B2468C046794409797B
:102E900049008F44071F25273435353535353535FD
:102EA00035350A152749002204E02649CA68092A4F
:102EB00020D8521CCA601649164A00F09BFC1EE03E
:102EC000002003F091FD012819D11E4830300E4931
:102ED000002212E000F0C8FC204600F035FF0EE0B2
:102EE0000D4908E00E20009000210122204600F04C
:102EF000CBFE04E005490022184600F0D5FE002272
:102F0000104602B0B0BDC04658250100382501006A
:102F10008813000021390100E824010080B5032056
:102F200005F0CAF880BD00000648416B002000296A
:102F300005D0054A914203D049680029FAD170476B
:102F400001207047AC99010228250100B0B5144654
:102F50000D460846114600F0ACFF012816D1285D49
:102F6000002813D1002C0BD06019401E00780A28CD
:102F700006D10320084A01462B460CF06BFF05E002
:102F80000320054A01462B460CF064FF0320294626
:102F9000224605F07DF9B0BDB7380100F0B585B027
:102FA000054604A800240470E743002D12D0EA6807
:102FB000002A0FD0686A00280CD0A86A002809D01F
:102FC000401EE96A814200D38EE004A9284690475A
:102FD000002803D03C46204605B0F0BD514EE86ABB
:102FE000411CE962696A049A0A54E86A696A002223
:102FF00002920A54E86A092806D1696A09224848F7
:10300000FDF7EDF800283ED03078411E022908D89F
:1030100000F0CEFEB168401A4349884264D8414E60
:1030200030780A2820D0012823D16E6A3A21304610
:10303000FDF7C4F8002847D0019002980390E96A90
:1030400003AB304639A200F04DFF02284CD1039863
:10305000002849D00A21334A117001990818696A79
:10306000401AC01C50602FE07068E96A81422BD181
:103070003AE004A800780A280FD00D2814D10120C6
:103080002863E86A1AE00120307000F091FEB06019
:103090003078411E0229BBD9C3E7296B012904D12D
:1030A00002202863E86A03E0296BE86A022905D157
:1030B000022817D10298E862286305E0012803D1AD
:1030C000686A00783E280FD0A86AE96A401E8142EB
:1030D0000AD2EA6804A9284690470028114E00D178
:1030E0007DE777E702982863E96A686A00F0E1FE05
:1030F00001280FD16B6AE86A002806D0C018401E6C
:1031000000780A2801D10DA200E010A20320014698
:103110000CF0A0FE03480470204605B0F0BDC04688
:10312000FA31010024970102DC0500002B524543CF
:10313000454956452C252A2C25643A005B415420EC
:10314000526563765D202573000000005B415420CA
:10315000526563765D2025730D0A000010B5064C9C
:103160002078002108F048FC044806F0EDFC2078A7
:10317000012108F041FC10BDAE96010260E316008B
:10318000B0B50F2001F0DEFB194D687028703328B0
:103190002AD120243721204601F020FC21200321C0
:1031A00001F01CFC2220402101F018FC2320082102
:1031B00001F014FC3020AA2101F010FCA2480221E9
:1031C0000187322001F00AFC3320012101F006FCC6
:1031D0005F21204601F002FC0F2001F0B3FB2870B4
:1031E0000A2006F0B1FCB0BD97480021C187B0BDF0
:1031F00004960102F0B581B0364C21210091617234
:10320000354909886170354FFA886271BD6ABD61C0
:10321000334B1B782370090AA170110AA171B97888
:10322000814207D10AF012FE6421FCF753FF398175
:10323000B978BD6A2B4848432B4940180A21FCF74E
:1032400049FF4519FD620AF097FD40190BF0F0F9AE
:1032500006460D462548007B0BF076F82449098880
:103260002222A15482B2D20B801802B2D01752107F
:10327000B2186841130E009D6355130C2025635549
:103280003B6DA3761D0AE5761D0C25771B0E637733
:1032900023462233090A5970A277BA64F864BA65E2
:1032A000F865100AE0770AF0D1FDF861FB6A282181
:1032B000012220460EF066F80AF0C8FD786108F099
:1032C000A3FF0028FBD1042008F056FB002001B02A
:1032D000F0BDC04606D40102AC980102309901024B
:1032E00086980102800A1B0040C20C00B6900102C1
:1032F0009098010270477047F0B587B04F4800685A
:10330000FDF714FB04460D464D48406AFDF7C0FB2F
:1033100002460B4620462946FDF70CFA02460B46AC
:10332000002448492046FDF78FF9049003910620B8
:103330004549085EFDF7FAFA0190009101200690D8
:1033400040020290414F05E04F4908517F1C241D67
:10335000642C70D0387805283D48F5D105973D4854
:1033600001593D4E31613D480359B3603C48005915
:10337000B0613C4A1259326200275D1A35637369A5
:10338000F1689941069B00DB3B46002B01D0029B74
:10339000C918314E7163F369716A101A9941069A1E
:1033A00000DB3A46002A01D0029A8918FDF7E0FABC
:1033B00002460B4604980399FDF754F9FDF740FBCC
:1033C000254A9062D162401BC10F40184010106026
:1033D0001546FDF7ABFA244A244BFDF743F9A863E1
:1033E000E963234A234BFDF73DF93A46224BFDF7AB
:1033F00039F93A46214BFDF783F805460E46164843
:103400000564416428463A461D4BFDF751FA0028F1
:10341000059F9BD10022284631461A4BFDF75EFAE4
:10342000002893D128463146019A009BFDF768F8A1
:10343000FDF7E2FA88E707B0F0BDC046F09601025A
:10344000D41F01000000F03F32A9010200980102E0
:10345000FFFF0100949F010218960102F89F0102EC
:10346000F4DF010258E00102699006699006903F7E
:1034700052257997532ED33F0000594000003E401B
:1034800000408FC0006AF84020D20102B0B582B07F
:10349000194C2068056801A90020087007E09047D2
:1034A0000198401C01A90870C0B2082822D201224C
:1034B00011048140294209D02268516080002018FF
:1034C000826A002AECD001A80121E8E713028340B8
:1034D0002B4201D0022104E082402A42E0D00321A5
:1034E000134622685360800020188268002AD7D0D3
:1034F00001A8D4E702B0B0BDD4920102FEE70000FB
:1035000010B509480168CA6920231343CB610269D9
:10351000032A08D1012293050C689C430C605102D8
:10352000C26E0A43C26610BD4893010281B010B555
:1035300081B00393002807D0C16A002904D003ABEF
:103540000093C46A0021A04701B010BC01BC01B0C7
:103550000047000080B5024608480068002807D0F0
:1035600091B2120C03889A4203D040690028F9D125
:1035700080BD002200F0F4FA80BDC04654C90102AB
:10358000F0B581B05C4C2068856BE80707D0E16836
:10359000002904D000208847206801218163A80702
:1035A00007D52169002904D001208847206802211D
:1035B0008163680707D56169002904D00220884724
:1035C000206804218163280707D5A169002904D058
:1035D00003208847206808218163E80607D5E16950
:1035E000002904D004208847206810218163A806A0
:1035F00007D5216A002904D00520884720682021AA
:103600008163680607D5616A002904D006208847CF
:10361000206840218163280607D5A16A002904D0CB
:10362000072088472068802181630126E80507D5A7
:10363000E16A002904D037020820884720688763A0
:10364000A80507D5216B002904D0770209208847F7
:1036500020688763680507D5616B002904D0B7022D
:103660000A20884720688763280507D5A16B0029B1
:1036700004D0F7020B20884720688763E80407D549
:10368000E16B002904D037030C208847206887634A
:10369000A80407D5216C002904D077030D208847A2
:1036A00020688763680407D5616C002904D0B703DC
:1036B0000E20884720688763280407D5A16C00295D
:1036C00004D0F7030F20884720688763E80307D5F5
:1036D000E16C002904D037041020884720688763F4
:1036E000A80307D5216D002904D07504112088474F
:1036F0002068856301B0F0BDD893010202480068DC
:10370000411E88417047C046A0980102F0B58DB0B7
:10371000002862D00446406800285ED0A068402897
:103720005BD8E56A002D58D0074620464030002679
:10373000039003E0019E4AE0039848E04021012203
:103740000691FCF729FDAE4202963ED2002031469A
:10375000019009900398069B3E46002EEAD0606ACD
:103760000491405C07900998401C059000210427B3
:1037700008916518EA5C012A17D10A966268D31984
:103780001B1F1B68099E9E5D0798864208D1059DF8
:103790005B5D002B0A9E22D00898401C089003E035
:1037A000403500222A70A668069B0837491CB142A2
:1037B000DFD308980028BFD00499491CE06A8142F1
:1037C000059809900398C8D301E003983E46374610
:1037D000E56A029E761CAE42B0D30DB0F0BD616AC0
:1037E0000B91E16A0C91D1590BAA204600F09CF88C
:1037F0000DB0F0BD81B0B0B583B00D46044607935F
:1038000007AB02938069E1690DF036FE20626548DE
:103810000078002803D1216AA06900F09FF963694C
:10382000A169226A204698470146A06B002905D06D
:1038300069460C600021224B0A460CE000F084FA35
:103840007D2081002846FCF745FC0246A06B6946B6
:103850000C6000211B4B00F0D3FA002003B0B0BC79
:1038600002BC01B00847C04680B5806B00F06CFA1E
:10387000002080BD70B582B00D46044646691146F1
:103880001A46B0470146A06B002907D069460C6074
:1038900000210B4B0A4600F0B3FA0EE000F054FA98
:1038A0007D2081002846FCF715FC0246A06B694686
:1038B0000C600021034B00F0A3FA002002B070BDA1
:1038C000AD390000C339000070B50D4604468021B3
:1038D00000F0C0FA2868E06368686060A868A060CB
:1038E000E868E0602869206168696061A869A06192
:1038F000E86900262662E061286A6062686A2663D9
:10390000E662A062A86A60632046383000F02AFAB6
:10391000002802D0F643304670BD2148016821607E
:103920000460304670BDC04670B514460D4606466C
:10393000881E032802D8B06B00F006FAF06B294607
:10394000224600F00DF970BD16480178012048406C
:103950007047C04670B512480468002C1FD0114E45
:1039600011A5216920468847002815D13078002804
:103970000DD1E16A606A00F09CFA0146606A012993
:1039800003D0E16A00F0E8F8284600F0E3F82046AA
:10399000FFF7BCFE0020E0622468002CE1D170BD7E
:1039A00050C9010248C901020D0A000010B50446C1
:1039B000806B00F0C9F9E06B0521002200F0D0F81F
:1039C00010BD10B50446806B00F0BEF9E06B042119
:1039D000002200F0C5F810BDF0B581B00091064698
:1039E000C7680468A01C3946FCF774FB00257068A2
:1039F000814201D1ED430BE0601C3946FCF76AFBC4
:103A0000316032695143B06808180099FCF7B2FB85
:103A1000284601B0F0BDB0B5012400250560446022
:103A200008300EC0B0BD70B50E460446C1680068CF
:103A3000401CFCF74FFB00256068814202D1ED433A
:103A4000284670BD22695043A16841183046FCF7F2
:103A500091FBE1686068401CFCF73CFB6160284614
:103A600070BDB0B5002400280DD00546006888421E
:103A7000FDD3401A286068684018E968FCF72AFB03
:103A800069602046B0BDE4432046B0BDB0B5002417
:103A900000280ED00546006840182860EA68904269
:103AA000FDD8A86840181146FCF714FBA960204611
:103AB000B0BDE4432046B0BDF0B583B01646024623
:103AC0000027F843002E22D01C46002B1FD00D46A5
:103AD000D168136899421AD9CB1AAB4217D39268AE
:103AE000019252198A423A4607D9019A8A1A0292D9
:103AF000029A52199342029A09D30292019810181D
:103B0000FCF7E8FA3160029840192060384603B0AB
:103B1000F0BD406870478068704702460020002A68
:103B200004D0106050609060D1607047C04370470F
:103B3000002803D00168484248417047012070477F
:103B4000002805D00168C068411A484248417047C2
:103B50000120704700207047002070470020704708
:103B6000F0B583B014460D4606464088012818D1AA
:103B7000306900280CD0A900405801782D2910D0B8
:103B8000F368716809686A461160506010A205E028
:103B9000F36870680068694621C115A23046FFF7D6
:103BA000C5FC7768FB6830462946224698470128BD
:103BB00008D00AE0C36830462946224698477F6805
:103BC000012802D178680028F4D103B0F0BDC046C6
:103BD00046534D3A252D38732053544154453A25C8
:103BE0002D323873204556454E543A25730D0A0040
:103BF00046534D3A252D38732053544154453A25A8
:103C00002D323873204556454E543A25750D0A001D
:103C1000F0B581B0002828D01E460C460546079B0B
:103C20000698009000206862A862E862104909883E
:103C30006B8029800F4B1F686C60009BAB602B462C
:103C40000C33C4C3A861E8612862481C0849088095
:103C500008480560002C08D06C60002128460A4600
:103C6000FFF77EFFA468002CF6D101B0F0BDC0467E
:103C7000D8CC010254C9010202460020002A01D01A
:103C8000D1627047C043704710B582B004AC24883D
:103C90001B881B041B196C462360024B00F0B0F814
:103CA00002B010BD55350000F0B597B01646029130
:103CB00005464268002A30D001966A60012100243E
:103CC000284616462246FFF74BFF3046029FBE426B
:103CD00032D003A85021FCF766FA32467268002FF2
:103CE0000CD003AF029811C74068083F824209D048
:103CF000394608313C4600280F46F4D1002A019E7F
:103D0000DBD10AE0019E386868600021284632460F
:103D1000FFF726FF7F68002FF5D102988468002CFA
:103D200008D06C60002128463246FFF719FFA468CE
:103D3000002CF6D117B0F0BD00212846019E324676
:103D4000FFF70EFFE9E70000014600201F2901D917
:103D5000C043704718224A43344901238B508918C5
:103D60008860704710B50021CC4300280BD00A4A68
:103D70001368002B09D01832491C2029F8D306D12A
:103D800006A0FFF7E7FE204610BD01231360016087
:103D90000024204610BDC046D8C9010274696D6573
:103DA000722049442069732066756C6C0D0A00000E
:103DB000264800687047C04670B520241B4D234E2E
:103DC0002868022817D13068A968EA68401A90422A
:103DD00011D96969002907D02879002807D0022065
:103DE00028603068A86004E00120286003E001201A
:103DF0002860286988471835641EE1D170BDC04627
:103E0000F0B5044600201F2C01D9C043F0BD059D2C
:103E100018266643054C0227A751A41921710B49A6
:103E200009682646083626C66361F0BDD8C9010276
:103E300006480168491C0160054841680268002382
:103E4000521C02604B4143607047C0468CAD01027A
:103E500090AD010280B5FCF7A6F980BDB0B502783F
:103E6000002A24D0441C0021084601E0573A08E00B
:103E700023460001D5B2302D0C4611D3392D02D87E
:103E8000303A14460CE0412D0C4609D3462D01D89A
:103E9000373AF6E71446613CE4B2062CE6D3002438
:103EA000E2B280185C1C1A78002AE1D1B0BD002073
:103EB000B0BD10B50246012000290DD00023D45C0E
:103EC000202C02D37F2C04D307E00D2C01D00A2C28
:103ED00005D15B1C8B42F2D310BD002010BD002029
:103EE00010BD000081B0F0B584B0099300230393A6
:103EF000002800D1C2E0002A00D1BFE009AB039343
:103F00001678002E00D1A8E05623DB43009300234F
:103F10001D46002900D1A2E0252E3FD1971C5278E2
:103F20001446643C0023142C43D8C0467C442479B6
:103F30006400A7440A99A3A3A3A3A3A3A3A3A3A331
:103F40004CA3A3A3A3A3A3A35F000297039A131DEB
:103F50000393126801920122002317461E4604783B
:103F6000FF0703D02D2C01D1164607E02746303F2E
:103F7000092F09D80A275F433B19303B491E401CD3
:103F800000270029EBD13946029A019C002C03D06E
:103F9000012E00D15B4223606B1C06E00378B34224
:103FA0005BD1491E521C401C2B461678002EAFD107
:103FB00064E02A2A62D13A780378934204D0491EF9
:103FC000401C0029F8D100216B1C3A46EDE7039A0A
:103FD000131D03933E7812680023C45CB44233D0AF
:103FE000491E5B1C0029F8D13C46C7180021002A55
:103FF0002ED12EE00297039A131D0393126800231B
:10400000009E0778302F18D33A2F02D23446273437
:104010000BE0612F03D3672F344606D30DE03C46F7
:10402000413C052C09D8344620341B011B19DB19EF
:10403000491E401C0029E4D10021029C002A00D026
:1040400013606B1C2246B0E73C46C718002A00D01C
:1040500009C26B1C22463846A7E700230EE0252E36
:104060000BD15178652908D103990A1D039209687B
:10407000002900D008606B1C00E02B46184604B0F5
:10408000F0BC02BC01B0084781B010B581B00C464D
:10409000039303AB00930DF0EFF9A04200D3601E31
:1040A00001B010BC02BC01B0084770B50446002046
:1040B000002A1BD0002C19D0002B17D0146001202F
:1040C000022B13D32578002D10D0641C01208D42C3
:1040D00005D1651E00262E7085005451401C984263
:1040E00004D2661C2578002D3446F0D170BDB0B5E1
:1040F00004467821FCF762F8002805D158212046B3
:10410000FCF75CF8002828D04278002A23D0841CD1
:104110000021084623460001D5B2302D0C4613D3AA
:10412000392D01D8303A0EE0412D0C460CD3462DE6
:1041300001D8373A07E01446613CE4B2062C01D3BB
:10414000002401E0573A1446E2B280185C1C1A7849
:10415000002ADFD1B0BD0020B0BD2046FCF7EEF84C
:10416000B0BD70B504460026F043002C0DD00D46BE
:1041700000290AD0204610300121FFF772FCA968FF
:1041800020342046FFF76DFC304670BD70B5044604
:104190000026F043002C0DD00D4600290AD0204601
:1041A00010300121FFF772FCA96820342046FFF788
:1041B0006DFC304670BD70B50024002814D0054653
:1041C000064610363046FFF7B3FC01280CD02846CF
:1041D0002030FFF7ADFC012806D02C683046FFF7F1
:1041E00098FC0C2141436418204670BDF0B583B0A3
:1041F00000250295019500281FD00C46064607466B
:1042000010373846FFF79CFC002816D13046203086
:1042100002AA01AB2146FFF74FFC00280DD13568FB
:104220003846FFF778FC0C214143B068029A101819
:1042300068506D186C600198A860284603B0F0BD06
:1042400070B505460C2058430024904211D2121A32
:10425000461829606860AE60EA602846103019464A
:10426000FFF75BFCE96820352846FFF756FC20463F
:1042700070BDE443204670BD04217046084204D05E
:10428000EFF30983EFF3088203E0EFF30883EFF322
:1042900009829BB004A8F0C044464D4656465F468E
:1042A00008A8F0C01846F0C86846F0C018690C901D
:1042B000202018440D9058690E9098690F90D86985
:1042C0001090EFF310801190EFF3148012900949D1
:1042D0000868139008490868149008490868159000
:1042E0000749086816901793189270461990684607
:1042F0000AF06EFF04ED00E00CED00E010ED00E0D0
:1043000014ED00E0F0B581B00326002430462146CC
:1043100007F0B6FB04252846214607F0B1FB01272C
:10432000304639463A4607F03FFB30462146324692
:1043300007F0CEFB284639463A4607F035FB022106
:104340002846224607F0C4FB01B0F0BDF0B589B0A5
:1043500008900425284607F00FFB0A27384605F089
:10436000F3FB284607F018FB0324204607F00CFB5C
:1043700007900526304605F0E7FB284607F0FCFAD3
:10438000384605F0E1FB284607F006FB204607F01B
:10439000FBFA0690304605F0D7FB284607F0ECFA0A
:1043A000384605F0D1FB284607F0F6FA204607F01C
:1043B000EBFA0590304605F0C7FB284607F0DCFA1B
:1043C000384605F0C1FB284607F0E6FA204607F01C
:1043D000DBFA0490304605F0B7FB284607F0CCFA2C
:1043E000384605F0B1FB284607F0D6FA204607F01C
:1043F000CBFA0390304605F0A7FB284607F0BCFA3D
:104400003846019705F0A0FB284607F0C5FA20467C
:1044100007F0BAFA0290304605F096FB284607F0FE
:10442000ABFA384605F090FB284607F0B5FA20466F
:1044300007F0AAFA0746304605F086FB284607F043
:104440009BFA019805F080FB284607F0A5FA204664
:1044500007F09AFA0446304605F076FB284607F046
:104460008BFA0699481E81410A460799481E8141E8
:10447000480080188000059A511E8A41510040185A
:10448000049A511E8A4180188000039A511E8A4165
:1044900051004018029A511E8A4180188000791EEE
:1044A0008F4179004018611E8C4106190898002838
:1044B00003D0032007F060FA02E0032007F06CFA53
:1044C0000A24204605F040FB0425284607F064FA3C
:1044D000204605F039FB284607F04EFAF0B209B045
:1044E000F0BD70B50446042007F046FA60B200281B
:1044F00003D4032007F040FA02E0032007F04CFA4F
:104500000A25284605F020FB0426304607F044FA29
:10451000284605F019FB304607F02EFA284605F02C
:1045200013FB600603D4032007F026FA02E0032001
:1045300007F032FA0A25284605F006FB0426304625
:1045400007F02AFA284605F0FFFA304607F014FA79
:10455000284605F0F9FAA00603D4032007F00CFA68
:1045600002E0032007F018FA0A25284605F0ECFAC5
:104570000426304607F010FA284605F0E5FA3046E2
:1045800007F0FAF9284605F0DFFAE00603D4032025
:1045900007F0F2F902E0032007F0FEF90A252846A9
:1045A00005F0D2FA0426304607F0F6F9284605F061
:1045B000CBFA304607F0E0F9284605F0C5FA2007A7
:1045C00003D4032007F0D8F902E0032007F0E4F950
:1045D0000A25284605F0B8FA0426304607F0DCF92B
:1045E000284605F0B1FA304607F0C6F9284605F02E
:1045F000ABFA600703D4032007F0BEF902E0032002
:1046000007F0CAF90A25284605F09EFA0426304626
:1046100007F0C2F9284605F097FA304607F0ACF9E2
:10462000284605F091FAA00703D4032007F0A4F967
:1046300002E0032007F0B0F90A25284605F084FAC5
:104640000426304607F0A8F9284605F07DFA3046E2
:1046500007F092F9284605F077FAE00703D1032026
:1046600007F08AF902E0032007F096F90A242046B1
:1046700005F06AFA0425284607F08EF9204605F071
:1046800063FA284607F078F9204605F05DFA70BD18
:10469000F0B581B003260025012430462946224684
:1046A00007F082F9304607F077F90626304605F024
:1046B0004BFA042007F070F9304605F045FA032064
:1046C00007F062F900281BD0681CFA2D0546F6D3C6
:1046D0000425284607F050F90326304607F04CF928
:1046E0000A27384605F030FA284607F055F93046D3
:1046F00007F052F9384605F027FA204601B0F0BD20
:10470000032001210A4607F04FF9042007F034F98D
:104710000024204601B0F0BDB0B50446C00703D167
:10472000032007F029F902E0032007F035F90825F6
:10473000284607F031F9284607F01EF9A00703D4F0
:10474000032007F019F902E0032007F025F90825F6
:10475000284607F021F9284607F00EF9600703D430
:10476000032007F009F902E0032007F015F90825F6
:10477000284607F011F9284607F0FEF8200703D471
:10478000032007F0F9F802E0032007F005F90825F7
:10479000284607F001F9284607F0EEF8E00603D4B2
:1047A000032007F0E9F802E0032007F0F5F80825F8
:1047B000284607F0F1F8284607F0DEF8A00603D4F3
:1047C000032007F0D9F802E0032007F0E5F80825F8
:1047D000284607F0E1F8284607F0CEF8600603D433
:1047E000032007F0C9F802E0032007F0D5F80825F8
:1047F000284607F0D1F8284607F0BEF860B2002836
:1048000003D4032007F0B8F802E0032007F0C4F84F
:104810000824204607F0C0F8204607F0ADF807242A
:10482000204607F0B9F8204607F0A6F8B0BDF0B56D
:1048300081B0032700243846214607F011F9384695
:10484000214607F01DF9012538462946224607F082
:10485000ABF8052638462946324607F039F90827CD
:104860003846214607F00CF938462946224607F01B
:104870009BF838462946324607F02AF9072738467A
:10488000214607F0FDF838462946224607F08CF805
:1048900038462946324607F01BF901B0F0BD00004A
:1048A00080B50B2007F070F812490A78002804D070
:1048B000002A12D003F022FB80BD012AFAD1002089
:1048C00008700F49C8830C4908700C480121017019
:1048D0000BF0FCFB03F012FB80BD074801220270C5
:1048E0000A700648002101700BF010FC03F006FB73
:1048F00080BDC0461C90010218900102199001026F
:1049000032A9010202484069811E4842484170476D
:104910006896010280B5FDF74DFA002801D000200D
:10492000C04380BD80B5FEF7FFFA80BD10B50448D6
:104930000F2100242246FFF713F9204610BDC04680
:10494000DC990102F0B581B007460324204607F048
:1049500023F80425284607F01FF8204607F00CF836
:104960000A26304605F0F0F8284607F005F8322010
:10497000FFF7B7FDFFF78CFEF8B2FFF7B2FDFFF7C8
:1049800087FE204607F008F8284607F005F820467D
:1049900006F0F2FF304605F0D7F8284606F0ECFFA7
:1049A0003320FFF79EFDFFF773FE0020FFF7CEFCDC
:1049B0000746284606F0E0FF204606F0DDFF3046B9
:1049C00005F0C2F8284606F0E7FF204606F0E4FFAF
:1049D000304605F0B9F8384601B0F0BDF0B581B009
:1049E000009107460324204606F0D6FF04263046F1
:1049F00006F0D2FF204606F0BFFF0A25284605F044
:104A0000A3F8304606F0B8FF3220FFF76AFDFFF743
:104A10003FFEF8B2FFF765FDFFF73AFE0098FFF79B
:104A200060FDFFF735FE304606F0A6FF204606F093
:104A3000A3FF284605F088F8304606F0ADFF204673
:104A400006F0AAFF284605F07FF8284605F07CF816
:104A500001B0F0BD80B50748012101700648026829
:104A60000A43026005480268002A02D0002001467D
:104A7000904780BDDECC01021C100050E0CC01024A
:104A8000F0B599B0F548017BC67A427B0E92F44CA2
:104A9000221F1368F34A1268069242780C92027938
:104AA0000592C76A04931F4001200F907A0200D537
:104AB000BCE03A0200D5BFE0FA0102D50F98020629
:104AC0002260502508968A191826BB0102D50F9836
:104AD000430623604123079569430A9635465543AB
:104AE0001426FC0210D50F98040538463746DC4ED4
:104AF0003460DA4CA469B464D84CE4697464DA4C68
:104B0000241D34603E46074690000B90D8040D905B
:104B1000681809900E9B73430F988203B902D04D19
:104B200022D50F9841052960CC480E9616460246BC
:104B300081692965C169696509990D9801430898DA
:104B4000000108180B994018C018C84909889279C3
:104B50004A4380180A301C4605F0D6FA23463246EE
:104B60000E9EC04988672A600F98C404380300D598
:104B70002C60F80302D50F98000428600F984104B8
:104B8000B80300D52960380400D4E4E1039402910D
:104B90000E9308920D980B990C180A980C994143A2
:104BA0000C910F98C0030B90286008F0E1F80028E2
:104BB00001D005F08BFA0C98005B410B43D10998AA
:104BC00000190E9940180599090140180E90E74DFB
:104BD000287B079B4343E97A0A010D9C2243D218A4
:104BE00041188B00D2180A9B4B43D1186A7B56435D
:104BF00089190E9E2A791018DF4A128842438818B4
:104C000016903068C000800D10A9C882002511954B
:104C10007079C0077ED110A80F998182069C0094FC
:104C20000020E8A2049B0BF015F978E00F988205AC
:104C300022603A0200D43FE70F98C2052260FA01D1
:104C400000D53BE73DE7072149030840032149031D
:104C50008842089A00D07EE1069707F0FDFC00200C
:104C6000169009901590C14CE07A217B08180A999A
:104C7000414380000D9A10434118627B0E967243A7
:104C80008A186178A379079E7343D718FA683F267C
:104C9000324063789A420C976ED105960A9A4A433D
:104CA00080580F210A0702400398401EC04B1B6822
:104CB000DB090340981810900F98C0020B90B86859
:104CC000800767D42C46283C0AF03AF8054620684D
:104CD000000609D5C3208401786A400704D40AF08D
:104CE0002FF8401BA042F7D905980002B96849087F
:104CF0000140B34803688268B868C40C2020204093
:104D0000DB0700D095E0002310221D461C460E9EB6
:104D10000B9FB1E010A88582B0681190069C701DB1
:104D2000924B1979E20707D1491C1971D97A1A797E
:104D30008A4202D31D7100E0D970017842781202D4
:104D40005118827812048918032291430170357139
:104D50005878401C5870D87A197B081859788842BE
:104D600000D85D70D879401ED871596B002901D0E8
:104D700010A888477E4DEDE010A80B998182F86855
:104D800030406378009000207CA20F990BF062F80D
:104D90000E9E94E0388A874A024010A8C2822022E0
:104DA000BA5C9307DB0F3C68C3720F9B1A40827298
:104DB0006205D20C0D9B1A431692FA68130E037209
:104DC000BB69FC697C4D2D682D0C05745204920F53
:104DD000427211931394654CA07B002809980E9E93
:104DE0000B9F5FD075480068007A0328099859D056
:104DF0000C98007D08400928099853D1C3208401EC
:104E000009F09EFF05460C98406A41070BD45949AA
:104E100009680906890F06D109F092FF401BA042DC
:104E2000F1D90C98406A41030898884310A98882F8
:104E300037E0D2070E9E0B9F03D1082300221546B0
:104E400019E00C9B9A68029C224211D19A68520C7C
:104E5000022494430022134615460DE0E4D10102DA
:104E600028A000503CA10050FC1F0000E0D101022E
:104E700004250022134614460843104318432843D0
:104E8000204310A9888238420BD10C9B198A494AC9
:104E90000A4010A9CA8219684905C90C0D9A114324
:104EA0001691324C2921615C002908D03037B84274
:104EB00005D010A908461130123109F05BFAE77AE3
:104EC0002A48047BE519294800790E902748407844
:104ED000401C2946FBF7FEF888000D9A10431890F5
:104EE000079961433801104340182049497B4E43DC
:104EF00080191C21694340180E9909191B4B1E4A41
:104F000012884A4380181790099A0C998A60987BF6
:104F1000002800D04A629879401C9871187B9979D2
:104F20008142069F00D39A715978491C5970D97AE9
:104F30000818597888420E4D00D85A70187A401EC9
:104F400018722820185C002804D0996B002901D021
:104F500010A88847089A174202D00F9800032860CB
:104F60001C480449486019B0F0BDC046E4D10102B4
:104F700028A000503CA10050E0D101024857204534
:104F8000542069647820256420616E642045542093
:104F900069647820256420696E2052582064657306
:104FA00063206D69736D617463680D0A0000000011
:104FB00038200040FF030000943000404494010278
:104FC000604000404D41432045565420257820251F
:104FD000780D0A00FFFFFF03F0B5A5B01E460C9246
:104FE00008910024239422A90C8016A90C8024A9DE
:104FF00009250D80598C0D91FBF76CF82A99012930
:1050000000D0DFE03189012900D0DBE0318C0129BB
:1050100000D0D7E00D99002900D1D3E022460796B1
:105020002C990B912B99069180B205900F9415A89D
:10503000058090000E900C990C582E4600252046B5
:1050400029461746FBF7EEFB0028119636D12C2097
:105050000A9778430899081817A90A4668C868C2C9
:10506000E8C8E8C2E8C8E8C2079F119880B280008B
:105070000E5822AD019523A8009020463946059A86
:10508000069B04F06FFD0F98401C0F9028880028A5
:105090002DD03B8A239913AC039416A8029014A830
:1050A000019015AE009617A824AA04F035FF2588B4
:1050B000308811900120149E0A9A05E013A80580FB
:1050C00014952E4628463A460E9F51000B9B119C84
:1050D0005C52591808830D84D81986600F9818857A
:1050E000521C0D9882426DD024A805889FE709962E
:1050F00016A800250580149524A8068823981290E8
:105100002F46109503E06D1CA8B2B04213D8A8B288
:10511000800017A90C5820461299FBF791FB002834
:10512000F1D1002FEFD115A8058016A8012707801F
:1051300014941094E7E715A80288B01A012805D145
:1051400015A80680099F1497119628E0102007994A
:10515000095E0129119221DB551CA8B20C18109F81
:105160000E9B099403E06D1CA8B2844218DDAAB21C
:10517000B242F8D8800017AA105810903946344629
:105180001E46FBF74FFB33462646099C0028EAD112
:1051900015A80580109F14971195E4E7109F0E9BAA
:1051A0001C463E4638461299FBF76BF9FBF7F6FBB7
:1051B0000546052800D3052513A8058001200A9A75
:1051C000274682E725B0F0BDF0B58BB00243159AB3
:1051D000149C139E2BD0054601A856C0129CD8697A
:1051E000196A09900A911E469F6B0123009309A832
:1051F00007AA0146059306F091FC716C3846FBF74F
:1052000040F90746E06A616BFBF73BF9002D069613
:1052100013D0044611980199012924D10921081AB3
:105220000421069A515E884229D16425B1E000200C
:105230003080207010700BB0F0BDB0880022642563
:10524000002829D0059269493846FBF715FB00284C
:10525000049C039E6FD166493846FBF70DFB00287E
:105260001DD05A2567E03C25082800D191E05F4910
:105270002046FBF701FB002819D0502589E00A29B8
:105280001DDB1D293BDC59493846FBF7F5FA0022A6
:10529000002854D05A253AE03346049C39E0554959
:1052A0003846FBF7E9FA002821D0502543E0504961
:1052B0002046FBF7E1FA00282ED0462569E03C2580
:1052C000012866D049492046FBF7D6FA0028D4D1F8
:1052D00047492046FBF7D0FA0028EED14549204641
:1052E000FBF7CAFA002854D1434920466EE04249F0
:1052F0003846FBF7C1FA00281CD128251BE03B49A2
:105300003846FBF7B9FA0022002832D05025049C19
:10531000069B0299039E41E036492046FBF7ACFA12
:10532000002836D134492046FBF7A6FA00282FD1B1
:1053300014252EE037250299059A069B2EE005924A
:105340002B493846FBF798FA002896D12949384668
:10535000FBF792FA0028B0D127493846FBF78CFAC0
:105360000028049C069B0299039E059A3BD11E25AA
:1053700014E005921E493846FBF77EFA00289CD1BE
:105380001C493846FBF778FA00281DD03C2500E080
:105390002325049C069B0299039E059A2580327062
:1053A00000200870307800280CD118681349FBF7EA
:1053B00055FA002806D12088102803D30F38208002
:1053C0000BB0F0BD0BB0F0BD0B493846FBF754FAFB
:1053D0000028049C069B0299039E059A01D114257E
:1053E000DCE72325DAE72D25D8E7C046CDCCCC3D38
:1053F000CDCC4C3DCDCCCC3C0AD7233C000020404A
:1054000070B588B00C4606464088002820D0FBF7CF
:1054100086FA059005A804A901252A4606F0E8FDAC
:105420003088B188081AFBF76FFA0390049903A833
:1054300007AA2B4606F09CFD5249079D2846FBF71C
:105440001BFA002808D0BF200006206008B070BDFD
:105450000020206008B070BD4B492846FBF7F0F9EA
:10546000002804D03F200006206008B070BD4749E6
:105470002846FBF701FA002801D0002010E00021A7
:105480002846FBF7F9F9002801D0022008E040493E
:105490002846FBF7F1F9002801D0042000E006209F
:1054A00001957F21C905029180003A49091801A898
:1054B00006AA022306F010FD0698206008B070BD11
:1054C000F0B587B00C460546476800263846314699
:1054D000FBF7E0F9002802D0266007B0F0BD049782
:1054E00004A803A90126324606F082FDA8682968AF
:1054F000FAF782FF0290039902A806AA334606F043
:1055000037FD2049069D2846FBF7B6F9002804D050
:10551000BF200606266007B0F0BD1B492846FBF7F2
:105520008FF9002804D03F200606266007B0F0BDA2
:1055300016492846FBF7A0F9002801D0002010E00A
:1055400000212846FBF798F9002801D0022008E046
:105550000F492846FBF790F9002801D0042000E00D
:10556000062000957F21C90501918000094909188D
:10557000684605AA022306F0AFFC059E266007B028
:10558000F0BDC046CDCC0C3F295C0FBFCDCC4C3E0E
:10559000CDCC4CBE4C940102F0B587B00C4606460B
:1055A0007F270088002801D0FD0503E0B08800288F
:1055B0002ED0334DFBF7B3F903907088FBF7AFF9AA
:1055C000049003A802A90126324606F011FD0299B3
:1055D00004A806AA334606F0CBFC2A49069E3046AC
:1055E000FBF74AF9002802D03F20010641E0264996
:1055F0003046FBF725F9002802D0BF20010638E02D
:1056000022493046FBF738F9002805D0002024E075
:105610000020206007B0F0BD1D493046FBF72CF993
:10562000002801D0022018E01A493046FBF724F97F
:10563000002801D0042010E017493046FBF71CF980
:10564000002801D0062008E014493046FBF714F981
:10565000002801D0082000E00A200096F9050191F9
:1056600080000F490918684605AA022306F034FC99
:1056700005992846FAF7C8FE206007B0F0BDC0467D
:10568000000080BF000038433333733F0000C8423E
:1056900000007042000020420000A0410000C04015
:1056A0006C940102F0B59DB015460B917F210391DA
:1056B000C9051C9102911B9119A900248C80199491
:1056C00018941794598C0691198C0F91DE8B998B35
:1056D0000791997805911F882B21CA4327999142F8
:1056E00001DB7F0015E04022D243914211DC4922C8
:1056F000D243914202DB7908CF190AE05322D24308
:105700009142EEDA5D22D243914201DBBF0000E01C
:10571000FF000A971396269E597E00290BD0002180
:1057200032460F46D170917051701170121D7F1C5E
:105730005C7EA742F6D30C9311952599149122997A
:105740000D91159041088C4211D2FD4A2346A000CC
:1057500084583454270A451C7755250C871CF55569
:10576000240EC01C34545B1C9CB2A142EFD8239879
:10577000109001200990009030463146149A159FF0
:105780003B4606F0D9F90D9800060890400E139D8F
:1057900000D186E068000490002F3FD00022104620
:1057A0001146144606E01C461146159F401C82B265
:1057B000BA420ED283B2AB42F8D09200149B9A5EEA
:1057C0000FB2BA42034600DC2346BA42EBDC0A467B
:1057D000E9E7002F25D0002210461146129206E07C
:1057E00012931146159F401C82B2BA4214D283B262
:1057F000AB42F8D0A5B2AB420CD09200149B9A5E9B
:105800000FB2BA42034600DC129BBA42139DE7DC9A
:105810000A46E5E7139DE6E7129903E000242146D6
:1058200000E00021129110980183C4828582049FB8
:10583000F057FBF769F87921C9050E91FAF7E4FDF5
:105840001099C86109980743F057FBF75DF80E9966
:10585000FAF7DAFD109F38622004C40B3057FBF7CB
:1058600053F80E99FAF7D0FD7862601C3056FBF7BA
:105870004BF80E9C2146FAF7C7FDB8621298000457
:10588000C70BF057FBF740F82146FAF7BDFD109C17
:10589000E062781C3056FBF737F80E99FAF7B4FD42
:1058A0002063119805800C98407E410000278D42AE
:1058B00028463A46149E1ED30A9880B28AB29300B4
:1058C000F45E84420BDA491C8AB2AA42F6D9002758
:1058D00028463A4681B2691A012910D01BE0F01817
:1058E000119B1980078808040FD0500040008019D0
:1058F000001F0288084681B2691A01290BD1A8004D
:10590000301811990D80078826E00020024681B2E8
:10591000691A0129F3D00A9989B2079B4B43BB420C
:105920001AD306998A4217D80599002914D0401C29
:1059300082B2891803E0401C82B291420CD983B232
:10594000AB42F8D89200B35EBCB2A342F3DDB2180A
:10595000119B18801788EEE712970B980580119815
:1059600000882B1A002B16DD02210F9A1143032900
:1059700042D10E93411C421E10B281420EDA0E98A3
:10598000032824DB0C98808C012820D019A818A9A2
:10599000FFF736FD1FE0002018902BE00026F443AF
:1059A000374608E0B8B2400019AD2B527F1C521C9C
:1059B00010B28142E3DB13B2A3423346F2DD159B02
:1059C00098423346EEDA8000149B1B5AEAE719A886
:1059D00018A9FFF7E1FD149E139D0F9A012A13D019
:1059E000032A11D0022A04D111980088281A02280B
:1059F0000ADA0020179034E0022A01D1022BB8DA2B
:105A000000201890012AEBD1681C691E0FB2B84221
:105A100008DA0C98808C01281DD119A817A9FFF766
:105A2000BBFD1CE00022D343144608E0A5B26D0084
:105A300019AF7E53641C491C0FB2B842E9DB0DB2AA
:105A40009D421646F2DD159DAF421646EEDABD00C8
:105A5000149E765BEAE719A817A9FFF7D1FC149EFC
:105A6000139D249F189C17992046FAF7C5FC0F999F
:105A7000012900D8204638600D98002800D1CBE0DD
:105A800011990888109FB8860888281AB88012983B
:105A900080B2FAF744FF7921CC052146FAF7B4FC2D
:105AA0002146FAF7B1FCB863119F3888002849D025
:105AB00081008919091F0988129C0C1915998842BF
:105AC00003D2800080198088041915984300534937
:105AD00016AA304606F00EFA169810994864FAF79E
:105AE00076FFA4B2A04201D14D480FE0001BFAF7A7
:105AF00016FF1C901CA81BA9012206F079FA20466B
:105B0000FAF70DFF01461B98FAF77EFC1099086022
:105B10003988491B4A1C92B2032A02D20021159FE0
:105B200017E009B20229159F12DB3F210906FAF797
:105B3000A3FE002802990CD10998810709E0C0460C
:105B4000402100400020129C15998842B9D3BCE73F
:105B50003449109801610898800E5DD0002F1CD048
:105B600000221146144610464B1B1DB2ED135B1963
:105B70006B40139D1BB29200B25E53431818A418D9
:105B8000491C8AB2BA42EFD3FAF7C9FE064620464C
:105B9000FAF7C5FE002C03D100E000260398C005EB
:105BA0001C901CA81BA901252A4606F021FA1B9C63
:105BB00020463146FAF728FC014610988160002FF4
:105BC000119422D000242746264613951291B8B28C
:105BD000FAF7A5FE1299FAF70FFC0546A0001499F2
:105BE000085EFAF791FE01461398C00785432846E0
:105BF000FAF70AFC01463046FAF7ADFB06467F1C71
:105C0000BCB215988442E2D300E0002611983146D8
:105C1000FAF7FAFB1099C8601DB0F0BD30A7010279
:105C20000000204100004040F0B58FB00692F74AD6
:105C300009AF70CA70C770CA70C70328079320D80D
:105C40008800F3A10858F649FAF785FB0446F549A0
:105C5000FAF781FB0D90F4492046FAF77CFB0C9093
:105C6000F2492046FAF777FB0B90F1492046FAF704
:105C700072FB0A90EF492046FAF76DFB0990EE4956
:105C800069E0042822D0062820D88800EBA1085813
:105C9000EE49FAF760FB0446ED49FAF75CFB0D901C
:105CA000EC492046FAF757FB0C90EB492046FAF7EF
:105CB00052FB0B90E9492046FAF74DFB0A90E84960
:105CC0002046FAF748FB0990FD4944E008380228CD
:105CD00021D88800FBA10858D149FAF73CFB0446BB
:105CE000FC49FAF738FB0D90FB492046FAF733FBE5
:105CF0000C90FF2081052046FAF72DFB0B90F74909
:105D00002046FAF728FB0A90CA492046FAF723FBF7
:105D10000990FE491FE08800F1A10858F449FAF7FC
:105D20001AFB0446F349FAF716FB0D90F249204698
:105D3000FAF711FB0C90F1492046FAF70CFB0B9097
:105D4000EF492046FAF707FB0A90EE492046FAF79A
:105D500002FB0990EC4900942046FAF7FCFAEC4962
:105D600009680E90EB480468EB4801684808EB4F5F
:105D700005463D400022002D08922DD0CA01120E8A
:105D800007D0280CE90D12D14000E649085AE6492F
:105D90000AE0C903090E0CD0280AE90B10D1400013
:105DA000E049085A8F2189004018E4300DE0DC49B1
:105DB0000AE081B27F2905D84800DA49085A04E090
:105DC000D94901E08F218900401800B2FAF79CFD03
:105DD000D649FAF719FB02460292039507252606D3
:105DE000D34B1A68002A089840D0791C8A420BD2FB
:105DF0001102090E13D0110C1F46D00D1FD14800FF
:105E0000C849085AC84907E01F46110E002A13D492
:105E10004800C449085AC2494018E4301FE0110440
:105E20001F46090E0ED0110AD00B12D14800BD49F1
:105E3000085A8F218900EFE7BE4808180FE0B848DC
:105E400008180CE091B27F2906D84800B549085AD5
:105E500005E0B548081802E08F218900501800B20B
:105E6000FAF752FDB149FAF7CFFA3B460590159F74
:105E70002C40F50E5B69B0491940089810D0DA0241
:105E8000D20E34D0C80B3E210140A648405AA64944
:105E90004018E43000B2FAF737FDA449FAF7B4FA33
:105EA0000490149E6800A5A1085EFAF72DFD014636
:105EB000A00009AA1058FAF74EFA0146B8B2012814
:105EC000089F019102D1022C0AD9A74F052C24D199
:105ED000189808900C2D20D80B2D16D3A44918E043
:105EE0000027022C089718D08120C70515E01A0456
:105EF000120E00D1CAE0080AC90B00D0CDE0400064
:105F00008849085A8F218900C2E7092D00D2C7E0CD
:105F100096490898FAF71FFA089001200021B54227
:105F2000034600D30B46052C00D308461799169A52
:105F30001A9C199D1843069B012B12D1079B402BDD
:105F400022D1002840D03846FAF705FA01460198D8
:105F5000FAF701FA01460098FAF74EFA059A049901
:105F60008AE0079B402B1FD1002838D03846FAF72B
:105F7000F2F901460198FAF7EEF901460098FAF7AE
:105F80003BFA059A049977E0002833D03846FAF7AF
:105F9000E2F901460198FAF7DEF901460098FAF7AE
:105FA0002BFA059A049967E000285BD03846FAF787
:105FB000D2F901460198FAF7CEF901460098FAF7AE
:105FC0001BFA059A049957E002981146FAF714FA59
:105FD0000399002900D16748059A04994CE002987A
:105FE0001146FAF709FA0399002900D16148059A88
:105FF000049941E002981146FAF7FEF90399002945
:1060000000D15C48059A049936E0C046F01E0100B4
:10601000000068C1000088C166665EC1000084C1DE
:10602000000084410000B4410000484100002040CD
:106030000000F0C0000084C10000F841333323C1E8
:10604000000050C19A9929C19A9949C19A99494128
:106050003333CB4166667641CDCCAC40333393C00D
:106060009A9949C102981146FAF7C6F9039900298D
:1060700000D14048059A049928601046FAF7BCF907
:106080000899FAF7B9F920600FB0F0BD99B27F29ED
:1060900011D848002349085AFCE623494018F9E67C
:1060A000C12001060898FAF756F90890062D00D984
:1060B00033E7002030E78F2189005818EAE6C04610
:1060C0003333F341000058C19A9961C19A9969C16B
:1060D000000084C10000AC4100003841000008C14C
:1060E000CDCC80C1CDCC88C133338FC1333397C180
:1060F00033339741CDCC8C413333F3409A9919C057
:10610000666646C1333397C1CDCCB4410000D4415B
:106110000C0000405030004068400040FFFFFF008E
:106120007C080000FC2201005C050000919AF63C0E
:10613000642000409C0B0000FFFF1F00FAFFFCFFE3
:10614000FEFF000002000400060008000A000C0028
:106150000E00100012001400160018001A001C0097
:106160001E00200022002400000080BF0000A0C00C
:10617000000040C00000DCC2F0B5FFB0ECB0174634
:106180000E460D900021E991E891DC91999198914A
:10619000979196911491139112919AA8F49DF39C62
:1061A000F29A002E00D1E6E10B938030F09B118033
:1061B000099529602546DBAC218095AC21800C95A2
:1061C0002980DA917F24E405B994B894B794B69401
:1061D000B594B494B394B294B194B094AF94AE9493
:1061E000AD94AC94AB94AA94A994A894A794A694C3
:1061F000A594A494A394A294A194A0949F949E94F3
:106200009D949C949B949A94046644668466C466A8
:10621000046744678467C467046444648464C46432
:10622000046544658465C465046244628462C46232
:10623000046344638463C463046044608460C46032
:10624000046144618461C461B0090B250B2800D34B
:10625000AE011095012B0B9D00D070E12B89012B15
:1062600000D06CE1298C00290E9200D18BE16B8C5F
:10627000002B00D1FAE1AA8C3021695C002900D101
:1062800088E10892109F5F431196304639460F937C
:10629000F9F720FF0590FAF737FB01462046FAF799
:1062A000F0F88321C905FAF7AFF8064696A8021D53
:1062B000119887420A9200D879E155A811909AA9BD
:1062C000069196AF15463A46059C234605F004FE16
:1062D00015A80F9006992A46234605F0FDFD0223D6
:1062E0000D93384631463A4605F042FE01230893A5
:1062F0000093E8AA10923846394605F00FFCE8985A
:10630000DD901198069D29463A46234605F0E4FDA6
:106310000F9829460A9A234605F0DEFD3846314695
:106320003A460D9B05F024FE089B009338463946FB
:10633000109A05F0F3FBE898DE9011982C46294658
:106340003A46059D2B4605F0C7FD0F9821460A9A4F
:106350002C462B4605F0C0FD384631463A460D9B8B
:1063600005F006FE089B009338463946109A05F062
:10637000D5FBE898DF901198069D29463A462346BA
:1063800005F0AAFD0F9829460A9A2346254605F0EE
:10639000A3FD384631463A460D9B05F0E9FD089BC2
:1063A000009338463946109A05F0B8FBE898E0901B
:1063B0001198069C21463A462B4605F08DFD0F9814
:1063C00021460A9A2C462B4605F086FD3846314672
:1063D0003A460D9B05F0CCFD089B009338463946A4
:1063E000109A05F09BFBE898E1901198069D2946CC
:1063F0003A46234605F070FD0F9829460A9A23462F
:10640000254605F069FD384631463A460D9B05F0B4
:10641000AFFD089B009338463946109A05F07EFB85
:10642000E898E2901198069C21463A462B4605F0E2
:1064300053FD0F9821460A9A2B4605F04DFD38462C
:1064400031463A460D9B05F093FD089B0093384674
:106450003946109A05F062FBE898E39011982146BE
:106460003A462B4605F038FD0F9821460A9A2B46EE
:106470002C4605F031FD384631463A460D9B05F075
:1064800077FD089B009338463946109A05F046FB85
:10649000E898E4901198069D29463A46234605F06F
:1064A0001BFD0F9829460A9A2546234605F014FD40
:1064B000384631463A460D9B05F05AFD089B00933D
:1064C00038463946109A05F029FBE898E59011986E
:1064D000069C21463A462B4605F0FEFC0F982146C5
:1064E0000A9A2B4605F0F8FC384631463A460D9B91
:1064F00005F03EFD089B009338463946109A05F09A
:106500000DFBE898E690119821463A462B4605F097
:10651000E3FC0F9821460A9A2B4605F0DDFC38462D
:1065200031463A460D9B05F023FD089B0093384603
:106530003946109A05F0F2FAE898E7907AE0108868
:106540000C9A108099919891DA9E08460F46099D01
:10655000F59CF9F751FF2860DC9827606060A66021
:106560000C34DDA80EC80EC42EC82EC42EC82EC4EE
:106570007FB06CB0F0BDFF2010800021296020802A
:106580007FB06CB0F0BD002201233021695C00298E
:1065900000D076E6DDAA1ACF1AC23ACF3AC23ACF75
:1065A0003AC20B213046F9F795FD054642E000203E
:1065B0000690059D0796089F1190069801460D9C30
:1065C0000F9A4A43D219109B5A43119BD218D200FA
:1065D000A35889002E4655AD6B503546121DA25862
:1065E00015AB5A50401C01B28E42E9DC55A89AAE58
:1065F00096AC314622462B4605F06EFC15A8314676
:106600000A9A2B4605F068FC022320460799224689
:1066100005F0AEFC01230093E8AA2046214605F0D0
:106620007DFA119B9800DDA9E89A0A505B1C0B2BA0
:106630001846C1D1F19EDDA89AA9DCAA0B2305F06A
:106640004BFC09210E980F9101800B98C168DC9CCE
:106650002046F9F7D9FE0146A8B2E69F0F281BD8BD
:1066600008280DD30846F9F776FE14E0FF201080C5
:106670000021099A11600C9908807FB06CB0F0BDC0
:10668000042803D381220846D10502E041220846AE
:106690001106F9F7B9FE01462B20C04386420D973B
:1066A00004DB0846F9F757FE014603E04020C043EB
:1066B000864244DD0E9A0C9C0B98408A002811D02B
:1066C0000B98038A95A80390DBA80290DAA80190A2
:1066D0000094DDA80D4603F01FFC29462488DA9EAD
:1066E000099D68E011910F98208000273D46109782
:1066F00005E00E9804887F1CB8B2A04211D8B8B249
:106700008000DDA90C5820461199FAF799F8002865
:10671000EFD1002DEDD10C98078001250F97109433
:10672000E7E7DBA805800F9A90B2201A012811D163
:106730000C9804800D9FDA973E46099D3AE0492067
:10674000C043864200DA8BE0FF2208469105F9F744
:106750005BFEA9E710200B990E5E012E00DA90E097
:10676000551CABB21846A1B2AAB28A4217D805E0AE
:106770000E990C88A1B2AAB28A4210D88000DDA975
:106780000C58204610991F46FAF74CF83B46002853
:1067900005D10C9805800B98068A0F95109430B29D
:1067A000C1186D1CA8B28142E2DC109EDA960F9CE3
:1067B000099D0D9F11993046F9F763FEFAF7EEF83F
:1067C000052800D3052095A90880A0B20E99098854
:1067D000814218D9401C611E0CB2A04218DA12A8DE
:1067E00098A9FEF76DFE0E980188481C491E0CB250
:1067F000A04221DA12A899A9FEF762FE9999989809
:10680000099D0D9FA4E600219891999108469FE665
:106810000022134608E09CB2A40012AF3D515B1C5D
:10682000491C0CB2A042DADB8DB20A2D1546F2D813
:10683000A400DDAD2D59EEE70022134608E09CB21E
:10684000A40012AF3D515B1C491C0CB2A042D1DB2D
:106850008DB20A2D1546F2D8A400DDAD2D59EEE714
:106860005320C043864200DB1BE70E460B9881692C
:106870002046F9F7D7FF00280C9C08D10B98808B95
:1068800007E01446099D0D9F1199109E93E70B9800
:10689000C08BFAF744F801463046F9F7B5FD119080
:1068A00021E70000F0B58BB01C4609930E46034665
:1068B00000200A9040480088224F05970AA90491B9
:1068C00003940292109C0194012500950B214143F1
:1068D00089B230331C4A3046FFF74EFC38680790C7
:1068E00078680890B868069033480088334F009560
:1068F00001940297324E30363249334A3346FEF71E
:106900006BFB0698F86207983863089878630998D3
:1069100000882E4905912E4904912E490391029732
:10692000019000962C4B284629462A46FEF74CFC3F
:10693000432001060A98F9F767FDFAF72FF80BB024
:10694000F0BDC046F8A60102B0DF0102F0B589B083
:106950000F9F0E9C002815D01098079016480088AD
:10696000164E01250095019102960893144B303381
:106970001449154AFEF730FB089BF762079830630D
:10698000746303E00D484763C462002518880F490B
:1069900005910F4904910F49039108490291019013
:1069A00007483030009001210B4B28460A46FEF77D
:1069B0000BFC09B0F0BDC0469CAD010274D40102CD
:1069C0005CA00102E49E010284D2010228A401021B
:1069D00098AD010238AD010240AD01023048704768
:1069E00000487047DCAD0102800037490918C86BC8
:1069F0000022CA637047C046800033490918886C7A
:106A000000228A647047C04680B52F4AD369002BA4
:106A100001D0126A9847002080BDC046024908781C
:106A200000220A707047C0464CC90102002070471E
:106A300080B5182905D803468A1E03481946F9F778
:106A400099FB002080BDC046A0AD0102B0B5024652
:106A50000020022901D2C043B0BD8C1E0F2C07D8E4
:106A6000044D284611462246F9F784FB002028559C
:106A7000B0BDC046BCAD0102B0B50246002002293F
:106A800001D2C043B0BD8C1E0F2C07D8044D284640
:106A900011462246F9F76EFB00202855B0BDC046CE
:106AA000CCAD01020849087800220A707047C04640
:106AB000B0B50446044DAA68002A02D0E968204611
:106AC00090472C610020B0BDAC970102F0B581B0B9
:106AD000DF4C206A0025002828465ED0324E3278EE
:106AE000012A11D1D948808A30490968012281429E
:106AF0000ADA0020E0706178002905D0E07060704B
:106B0000022002F0F7F83278D04FB98A274800689F
:106B1000884201DC002A0ED1E278531CE370152A6A
:106B200009D36278002A06D10120607002F0E2F8F1
:106B3000B98A1E48006888420DDA2078002801D002
:106B4000002020700020A070606219490870307821
:106B500000280CD118E00121A170626A531C636205
:106B6000FB8A9842132A04DA307800280CD001B04E
:106B7000F0BD2078002800D12170002060620C4810
:106B8000017030780028F2D12078002801D101204E
:106B90002070F3480549086001206562A07004492F
:106BA000087001B0F0BDC04630990102549901024D
:106BB000AD96010280B5124801681F220A400260AA
:106BC00003200840022812D10E480268D30D02D0DB
:106BD000FF231B06D2180C4B1A600C4A12680C4B90
:106BE0001A6080680B4A1080000C0B4A10801A480B
:106BF0008268002A02D082680020904780BDC0468B
:106C0000742000406440004098D201027830004077
:106C10009CD20102C0A001026AD4010280B50D48D5
:106C2000016889070FD5052101600B48C17800294B
:106C300008D00021C170C168002903D0C268416832
:106C40000020904780BD054805A10B4A0BA308F022
:106C5000A5F8C0462C04004034940102603C0100B9
:106C60005048595F54494D45525F49525148616EF1
:106C7000646C6572000000008D0A0000556E657836
:106C800070656374656420696E7465727275707482
:106C90000000000070B50446401E012814D80320EF
:106CA000084011D13F2040030818050B28198028FF
:106CB0000AD8164E317801204840294604F086F85B
:106CC000641E6D1C002CF5D170BDC04680B500203F
:106CD000014603F0C3FD002800D080BD0B48012110
:106CE000017080BD70B516460C460546FF22F9F7C7
:106CF00053FA0548311805480278012050402A46C9
:106D0000234603F00BFF70BD00E0070430A9010229
:106D1000012000037047012040037047F0B585B0A3
:106D200048484949016005F077FF484DE98A4A2201
:106D300047488152AA8A4823C252AB88C362AC7AC0
:106D40008471AC89048242828182A98D0187049377
:106D500083864A1E914149000162A88B3B2801D8D5
:106D60003C20A8830020E883288B3A490880FF2034
:106D70000A3068806C8C0F20224602407D21C900B9
:106D8000260B4E43B6182205170F64225743F619F7
:106D90002406270F0A246743F6192F4F3E80AE8C36
:106DA000374607402B46350B4D43ED1937053F0F4E
:106DB0005743ED193606360F6643AD19274E358019
:106DC000DD8C2E4606402F0B4F43BE192F053F0F7B
:106DD0005743F6192D062D0F65437519204F3D8039
:106DE0001D8D28402E0B4E4330182905090F5143A5
:106DF00040182906090F614340181A4E30800324B9
:106E000019A220462146049B09F024F80F48408827
:106E1000C1B20091030A18A22046214609F01AF8CF
:106E20000D4803880D48008839883288094D2D881F
:106E300000AE27C619A22046214609F00BF805B07E
:106E4000F0BDC04600960102B584000032A90102DF
:106E500080980102749601026C9601026E960102FE
:106E60007096010272960102C9E8B1B849443A200D
:106E70002578202E0D0A0000B9CCBCFEB0E6B1BECC
:106E80003A5557422D3447B3B5D4D8CAD6BBB720EC
:106E90005625642E25642E200D0A0000B7FECEF183
:106EA000C6F7B5D8D6B73A2025642E25642E2564BA
:106EB0002E25643A25642E0D0A000000F0B581B03D
:106EC000254E3378002B0CD0244D24350022144657
:106ED0002F8887420AD0AD1C641C521C9A42F7D3FB
:106EE00001E0002422469C4203D006E0D4B29C423A
:106EF00003D1172B01D8631C3370B318602400250D
:106F00001D555200154B9A189084746A002C02D0BB
:106F10001348844202D1716201B0F0BD0846F9F70E
:106F200005FD00250F4B2A46F9F79CFB074600910B
:106F30002046F9F7FBFC2A460A4BF9F793FB024679
:106F40000B4638460099F9F7DBFAF9F755FD01468B
:106F5000716201B0F0BDC046309901020C9A010285
:106F6000FFFF01000000E03FF0B583B0304800684B
:106F7000C16B0901890F01D003B0F0BDC16BC06BBB
:106F80002C4D05404800400F0826029686400227F7
:106F9000384602F009FD01907043C10B4A1B264898
:106FA0005043F9F7ADF8044607F03AFE032123A257
:106FB00038461F4F0091234608F04CFFF88A0028FE
:106FC00017D0019840012946F9F784F84643182262
:106FD000324001200F2A014600D8002173095B18B6
:106FE0001B4CA3420DD8194DED1A6D050F2A0CD874
:106FF0000CE038680021C160112002F0C5FC03B02C
:10700000F0BD5D1C6D050F2A00D956422A0C029D69
:107010002E4009018919A34202D80098000400E01B
:107020004004081880183968086303B0F0BDC046F2
:10703000C4940102FFFF1F0040420F0052434F3330
:10704000324B2070706D2025640D0A00FF07000090
:10705000FE7F0000B0B582B0154908688269D2078A
:107060000CD00122C2610D69002D07D000686C466A
:10707000214607F075FB00212046A84702B0B0BDAD
:10708000B0B582B00A490868026C92070ED5026C4E
:10709000012313430364CD68002D07D000686C46BC
:1070A000214607F05DFB00212046A84702B0B0BD95
:1070B000C4940102064801680322914301600168FB
:1070C00001220A43026000F017FB07F0CBFDC04627
:1070D0002800004080B50D490868002810D52248D6
:1070E00002680423032A01D01A4300E01A460A600A
:1070F0001E490A68002A02D041680020904780BDDE
:1071000003A00CA19E2211A307F048FE2C10014001
:10711000696E636C7564652F647269766572732F2E
:107120006D6B5F736C6565705F74696D65722E63FE
:1071300000000000534C4545505F54494D45525F97
:1071400049525148616E646C65720000556E6578F5
:1071500070656374656420736C65657020696E7416
:1071600065727275707400000C90010270D4010297
:10717000B0B582B004460078002811D0094D01A9AD
:1071800008702868416A0029FCD101A90122002069
:10719000034609F021FC611C607800280C46EED102
:1071A00002B0B0BDFC94010270B50C784D782D0290
:1071B0002C198D78C9780902491909040919800028
:1071C000094C21509178D47815785278074E335075
:1071D000074B069E1E501202521923025918090429
:1071E0008918044A115070BD949F010258E00102B1
:1071F000F4DF0102F89F010210B5DD4C2168062979
:107200000FD8012002468A4058210A4209D0206046
:107210000020A0602369002B03D0626900200221B6
:107220009847D2482258062A12D801210B4693408B
:10723000582213420CD0215020180021816003698C
:10724000002B05D0AD20C000225801200221984714
:1072500047482258062A11D801210B46934058224C
:1072600013420BD021502018002181600369002BAC
:1072700004D003482258022001469847002010BD40
:10728000BC0A0000F0B581B00024022803D9E44311
:10729000204601B0F0BD17460B46094E464309484B
:1072A0008519284618302A2107A2FCF7EDFE422056
:1072B0002F52032003498851204601B0F0BDC0463B
:1072C000540500005CAE010225730000F0B585B0E6
:1072D000CB4D2C68002C0CD0C84FC94CE659002E61
:1072E0000CD0234FE659002E0DD00020C04305B02E
:1072F000F0BD01AC0FC400272E4608E001AE0FC65A
:10730000E619012703E001AE0FC6E6190227DB4CA0
:1073100030462146FCF79EFD022030607C4329194F
:10732000029D4D60CF60039808610498486108464B
:107330004430CC310122560210233246FCF780FF44
:10734000DD480019B32189004118012D05D1B8305D
:1073500001233246FCF75FFB04E074301023324611
:10736000FCF76EFF01980760002005B0F0BDC04635
:10737000A80A000001460020022901D9C043704735
:10738000D44A4A43D44988507047C046022806D898
:10739000D0494143D04840180249401870474B201B
:1073A00080007047D4040000022802D94B208000DE
:1073B0007047C8494143C84840184D210901405809
:1073C0007047C046032801DB03487047C149414369
:1073D000C1484018183070476D3A0100022806DC99
:1073E000BC494143BC4840184221405A70470020E4
:1073F0007047C046032801DB00207047B549414370
:10740000B548401844307047022804DCB149414374
:10741000B1484058704700207047C046022805DC3C
:10742000AC494143AC484018406870470020704761
:10743000B0B50024E14302280FD8A64A4243A64B28
:107440009D58042D09D0991801220A600B69002B60
:1074500005D04A690221984721460846B0BD20461A
:10746000B0BDC04610B50024022801D9E04310BDCC
:1074700098494143984A0723535051180B69002BF0
:1074800003D04A69002421469847204610BDC046D3
:1074900010B50024022801D9E04310BD8D494143B5
:1074A0008D4A0623535051180B69002B02D04A69AC
:1074B00001219847204610BD10B50024022801D9AB
:1074C000E04310BD83494143834A51180B69002BA7
:1074D00002D04A6903219847204610BDF0B583B019
:1074E00017460024E24302281AD8002B18D00D4674
:1074F000784941437848461870680128029312D1B0
:10750000002F0AD0B836002429193046FCF78BFA30
:10751000002825D1641CA742F6D1029807600022FA
:10752000104603B0F0BD019274363046FCF743FEBE
:10753000002811D003464268BA4209D21968284689
:107540001D46F8F717FE2B466868029908600194FB
:1075500030461946FCF705FE019A104603B0F0BD0F
:10756000029804600022104603B0F0BD54050000EC
:107570005CAE0102F0B581B004460020C343022C8A
:1075800002D9184601B0F0BD15460E461B4A6243AB
:107590001B498F187968012910D1002D28D01C466D
:1075A0000090B83738463146FCF716FA002821D14A
:1075B000761C6D1EF6D1009801B0F0BD00907437B6
:1075C00038462946FCF712FE00280CD00446006815
:1075D00031462A46F8F7CEFD38462146FCF7D6FD5F
:1075E000009801B0F0BD07A02146FCF7B3FA00985F
:1075F00001B0F0BD204601B0F0BDC046540500000A
:107600005CAE0102536F636B65745B25755D205240
:10761000656376204275666665722046756C6C0DF2
:107620000A000000F0B583B0154607460022D0439B
:10763000022F19D8002D17D000AB07C30F4878438D
:107640000F490E18443630462946FCF7CFFD002876
:107650000CD00446006801992A46F8F78BFD3046A5
:107660002146FCF793FD029803B0F0BD05A0394612
:10767000FCF770FA009803B0F0BDC0465405000056
:107680005CAE0102736F636B65745B25645D207390
:10769000656E64206275662066756C6C0D0A00006C
:1076A00002460020022A04DC0A4B53430A4AD15006
:1076B0007047C0437047C0465CAE0102022801D942
:1076C000002070470349414303484018034940588C
:1076D0007047C046540500005CAE0102CC040000B7
:1076E00080B504480168491C01600069002800D089
:1076F000804780BDDCDF010201480249016070471C
:10770000709001020026B80310B5C34800244461FC
:1077100010300221024A2346FFF7D8FD204610BD53
:10772000CD77000070B584B0FDF7FCF8012814D1C6
:10773000FCF73EFB1F4D6969022914D0002909D1CD
:10774000297800291FD0A969411A062902D30021EE
:107750002970A861002004B070BD16480021416165
:10776000002004B070BDE969421A13490E2A02D8FC
:107770000A78002AEED0E8610020087000F004F9D1
:10778000002004B070BD01266E61AB88E8882989AD
:107790006A8900AC07C4B102084C09A22046FCF774
:1077A00073FC2869AA892146FFF76CFD2E70002022
:1077B00004B070BD689601024493010248C50102FD
:1077C00025752E25752E25752E257500F0B58DB0E5
:1077D000032909D87944097949008F4401070F1515
:1077E0005948416901290AD00DB0F0BD5648416998
:1077F0000129F9D1022141610DB0F0BD52480021AB
:10780000416101700DB0F0BD002500954E4C20691E
:107810004E494F4A6B46FFF761FE0028E4D1032032
:107820004CA2014608F016FB48484DA10A22F8F781
:10783000D6FC002812D045484CA10F22F8F7CFFC07
:107840000028D1D141482C2101AA0C23FCF72DFCA2
:107850000298FCF703FB60870DB0F0BD3B482C217C
:1078600001AA0C23FCF721FC0498FCF7F7FA6087C7
:1078700080B2684EB1888142B6D10298FCF737FCDD
:10788000E062039801794279120251188279C37932
:107890001B029A18120451188278C378077840782E
:1078A0000002C0191B029A181204101820626162AB
:1078B0000598FCF7D3FAA0870698FCF718FCE08738
:1078C0000798FCF714FC4027E0530898FCF70FFCDE
:1078D00042216054E16A491E062901D80122A270A2
:1078E000062926D87944097949008F440318111CC8
:1078F000221E1500E08FB082E05BF082A08FB18D78
:10790000814216D01E4902220A60B0851D4800E05F
:107910001A48012101700CE00120B08709E01848E5
:107920000560B58505E0B58703E0C0B23C21414361
:10793000B1830120A07000F027F807F0F5F8256268
:107940006562A5700DB0F0BD6896010248C50102E0
:10795000FF030000CAD5B5BDCAFDBEDD0D0A00009B
:1079600024696E7374727563742C0000246D6573E2
:10797000736167655F7265706C792C00AC9601026B
:10798000A098010238900102F0B5C7B0214CA08840
:107990001490214D68781390FBF7B0FE1290A08DE3
:1079A0001190687810901D4800780F90A08A0E9072
:1079B000E08A0D901A48C0C81A490A684968AB782D
:1079C000194C24682035089209910A950B930C9460
:1079D0001298009011980190109802900F980390BF
:1079E0000E9804900D9805A9C1C11398012801D0E3
:1079F0000F4A00E00D4A15ADC8212846149B09F036
:107A00001FFD0246044800692946FFF70BFE47B0F8
:107A1000F0BDC04632A90102689601028A980102AF
:107A200010990102089901025499010238310100AC
:107A30007931010080B582B00E4908680022C26029
:107A40000192CA68002A02D0016801A8904702B0DA
:107A500080BDC04680B582B0064908690022C26078
:107A600001220192CA69002A02D0016801A8904748
:107A700002B080BD1C930102F0B582B0144C207896
:107A8000009000281DD0134B24330025019504E0FD
:107A90009B1C6D1C0098854215D262196026905D72
:107AA000471C97550928F3D80199C8B222181C8899
:107AB00097554000074A10188484054C491C0191D1
:107AC000E6E7002001900198207002B0F0BDC046AA
:107AD000309901020C9A0102F0B589B009F0D4FB8B
:107AE000E94C607809F076F9E8498A8807A882802D
:107AF0000A88498809048918079105F00FF9607808
:107B0000052804D00222E249092804D104E0012218
:107B1000DF49092800D0891849792078621C09F0CA
:107B20001DFA607A06F022FCDA48DB4904F0FAFB21
:107B3000DA4C20780026002806960AD0D8491A3157
:107B4000D84A034610CA0C80891C5B1EFAD1460035
:107B5000D24CD54DA872D54800886871D4490978AF
:107B600029706178E970000AA871481C6070284685
:107B70000B30CB4F39464C3103913246F8F7FAFAC5
:107B800070190B3039461A313246F8F7F3FA2020D3
:107B9000687206982071E0886870000AA870C32097
:107BA0000690840106F052F90319BC48C362BB4831
:107BB000007881000D3101222846059209F0E2FB90
:107BC000B6498862B548C46A06F0D6F80019B34CC5
:107BD00006F02EFD05460E46AB48007B06F0B4FBD2
:107BE00081B2C90B401800B2C11740102818A06517
:107BF0007141E16506F02AF9A06104F005FB002857
:107C0000FBD106F023F9E0617D200601002738460C
:107C10003946324609F06AFBA0626771254606982C
:107C2000040206F013F9297861434118A2480818A4
:107C3000421C01D19F480818984C206306F006F9B1
:107C40006063216B884204D39C4A8918884200D81B
:107C500097E006F0FBF8606306F0F8F8E06104F0E6
:107C6000D3FA0028FBD106F0F1F8206260790228EF
:107C70004FD001287DD100206071914D697A212972
:107C800071D16979AA7912025118884A12889142F1
:107C900069D1874909782A788A4264D16978AA78B3
:107CA00012025118A181E278002A40D02278002ADD
:107CB0000BD07B4B4C3300201C888C4204D09B1C87
:107CC000401C8242F8D11046744CC0B2E081236E51
:107CD000A16BA26D7A4D2C46223400946F4C019119
:107CE000029229461A311E352A46FFF75DFAE089CD
:107CF000E178884208D34100694A5118A2894C238F
:107D0000CA522178491C21700521654A11546C48DA
:107D100024E0002060710146324609F0E7FAA062D3
:107D200006F094F8206206F091F8A06121E04C2062
:107D30005B4A11520598207005201070236EA06BCD
:107D4000A16D2A46223200920190029129461A31F1
:107D50002A461E320020FFF727FA28469621F8F718
:107D600022FA0020208200200146324609F0BEFAA5
:107D7000A062226B606B51495118904200D365E7B5
:107D800067E7A06DE16DFBF7B7FAA77020780028D0
:107D90002FD044484C213D463C46414B05E0891CD0
:107DA000001DFAB26D1C95421AD25E5D002EF6D00F
:107DB000761E5E55A3000693F6B22246414CE6506D
:107DC000374B5E5A5300404CE6527F1C334B9F703A
:107DD00003683E4C069EA3511446314B541CDEE70B
:107DE00005922E48C77007700497F8B2022806D291
:107DF00028E0E77805970497F8B2022822D305987F
:107E0000441E0021069403E0491C069CA14219D09F
:107E10002E4A10682C4B2B4F0FE0156050605D8888
:107E20001E885E801D8060CF083F3E607D60641EBE
:107E3000121D9B1C3F1D002CE6D05568A842ECDCAF
:107E40002846F4E704980006059C10D062001E49FD
:107E50000398F8F78FF9A20012481C49F8F78AF93D
:107E60000F4A184802C81170521C641EFAD10B4800
:107E700083890C4800680090032015A2014607F092
:107E8000E9FF09B0F0BDC046C4900102081F01001F
:107E9000C4A001028D000100A5EA0000B096010215
:107EA0000098010220D20102CEE90102AC98010241
:107EB0008698010201CF030000CF03000026B8031B
:107EC00070D30102D4E801029CE9010238E9010201
:107ED000BBF9D5BE4944A3BA25582CBEE0C0EB3A45
:107EE0002025640D0A00000080B5002008F02CFA5F
:107EF00080BD80B5012008F027FA80BDF0B581B0C3
:107F000003F0C2FC164CE060A178002901D001B05A
:107F1000F0BD21790029FAD10121217100281BD05F
:107F20008D02281AA168814216D0614E2F46A068A2
:107F3000305C21698847A068401CA060681EA16869
:107F4000814201DD0020A060E168A068022F03D318
:107F5000691A7F1E8842EAD10020207101B0F0BD6D
:107F6000F0950102B0B5294C2368002B07D0022BF5
:107F70000DD0012B39D109F053F900F00FFC09F0B5
:107F80002DF92368022B1FD0012B18D02DE0204D96
:107F9000287800282FD003201EA2014607F05AFFA0
:107FA0000020287009F03CF900F02CFD1C4D2870D1
:107FB00009F014F928780028E3D00120206019483E
:107FC00000214181012310E011480178002909D1E5
:107FD00014494A89531C4B81152A03D3012202708C
:107FE0000020488108F0C2FE2368032014A2014645
:107FF00007F030FFB0BD0B48408914210B1A032055
:1080000009A2014607F026FFBBE7C046A09801027F
:1080100038900102BFAAC6F4CBD1CBF70D0A0000FD
:108020008798010230990102B5C8B4FDBDF8C8EBCC
:10803000CBD1CBF7C4A3CABDA3BA25640D0A0000F7
:10804000555742D7B4CCACA3BA25640D0A00000042
:1080500080B505480068022805D809F0E1F8FFF767
:108060003BFD09F0BBF880BDA098010270B50E255C
:1080700000242846214603F003FD0D20214603F08D
:10808000FFFC0124204608F067F804262846314604
:1080900003F0F6FC0920314603F0F2FC204601F023
:1080A000C9FAA2020249034B204608F053FB70BDF7
:1080B000E0CD01028D09010080B5032810D8002908
:1080C0000ED07C224243BF488018C268012A07D1E3
:1080D0002030FBF7A8FC002801D00020C04380BD61
:1080E0000020C04380BDC046F0B589B00022D54312
:1080F000032800D9ABE00C46002900D1A7E0009589
:10810000216A0727534DA9420EDC574DA9421ADDBB
:10811000564A91422FDC4B22D501A9423ED0120291
:1081200091424BD1042246E04B4A914217DD4B4A23
:1081300091422ADCE1221203914231D0494A914214
:108140003CD10C2237E04B252E01B14233D06A01DD
:10815000914227D0AA01914230D102222BE0E122A4
:108160005502A94220D09502A9421FD0D2029142C5
:1081700024D109221FE04B225202914218D0E12261
:10818000120291421AD1062215E0E12252039142D5
:1081900010D0334A914211D10D220CE003220AE0A3
:1081A0000A2208E0012206E0072204E0082202E099
:1081B000052200E00B22D1002D4A57587C21414373
:1081C000804A505056182068B0606068F060A1681E
:1081D0003161E268726100250595032304930395DC
:1081E000029501970695079501231B020893012824
:1081F00007D000280AD18818009A8018B161F06170
:1082000004E0304620300123FBF705FC2069706351
:108210006069B063E069B067A069F063706801A944
:1082200008F0C4F92068012806D8304640302346BB
:1082300010330ECBFCF704F86068012807D1301D1D
:108240007036006801220B4B314608F083FA28464D
:1082500009B0F0BDFFC10100FF0F0E00FF1F1C00A1
:1082600080841E0040420F007F250000FF95000023
:10827000381F0100A5090100B0B50C467C21484318
:10828000504A15182846FBF7E5FD6C600020B0BD8C
:10829000F0B583B00024E743032800D98EE00E46F2
:1082A000002900D18AE01546002A00D186E07C2111
:1082B0004143444841188868022832D001283AD006
:1082C00000282BD1EFF31080C00702D1EFF310800C
:1082D00072B602910846403001902946FBF786FFAE
:1082E000002863D0014601980F46FBF74FFF38681E
:1082F00031462A46F7F73EFF0198FBF75CFFEFF3A4
:108300001081C90703D1EFF3108172B662B60299EA
:108310004D6806C82C4B284608F05EFB204603B08B
:10832000F0BD4868002431462A46234608F054FB35
:10833000204603B0F0BDEFF31080C00702D1EFF389
:10834000108072B602910846403001902946FBF732
:108350004DFF00281ED0014601980F46FBF716FF7F
:10836000386831462A46F7F705FF0198FBF723FFE7
:10837000EFF31081C90703D1EFF3108172B662B633
:1083800002994D6806C8104B284608F025FB204688
:1083900003B0F0BDEFF31080C0070FD1EFF31080F2
:1083A00072B662B63C46204603B0F0BDEFF31080D3
:1083B000C00703D1EFF3108072B662B63C46204688
:1083C00003B0F0BD58BE0102A90C0100B0B582B0E7
:1083D000602833D0622843D0642854D101A82F49A3
:1083E0000180EFF3108072B600242046214602F08F
:1083F00035FA2B4D002805D1012002030020294623
:1084000002F086F9103501AA02232046294602F01F
:108410005DFE62B623A0FEF7ABFE64201B490C5242
:1084200006F082FB1A4801F08FFBBFF34F8F19480B
:1084300019490160BFF34F8F00BFFDE7602013496A
:1084400000220A5206F070FB114801F07DFBBFF3D9
:108450004F8F104810490160BFF34F8F00BFFDE7F9
:1084600062200A4900220A520A8006F05DFB084891
:1084700001F06AFBBFF34F8F064807490160BFF365
:108480004F8F00BFFDE702B0B0BDC04632A9010268
:10849000A08601000CED00E00400FA05AAAA000085
:1084A00000D00204BDF8C8EBC9FDBCB6C4A3CABD68
:1084B0000D0A0000F0B5D1B0A74EA8490A78002AED
:1084C00025D0F28B002A22D1A54FBA68082A00D9FC
:1084D00090E0930001A4E3589F46C0460185000048
:1084E000F5850000F5850000058600002F86000058
:1084F0003986000043860000138600004D86000088
:10850000552800D0BBE00120B86051B0F0BD4978DB
:10851000002900D1B7E0924D6A7996498854A9792B
:10852000A871E971521C6A710A2800D0ABE00D29CC
:1085300000D0A8E003A8019037A800902C46303462
:108540008C488D491DAB2246F7F766FEE8608BA18B
:1085500005222046F7F743FE00282AD1F08B002899
:1085600005D0032087A2834B014607F073FC1DA8AA
:108570000024214609F02DFCA861E961824B2246C6
:10858000F8F796F9002814D1804800F079FF1DA86B
:108590000024214609F01DFC2862696237A82146A3
:1085A00009F017FCA862E96203A8F7F7C7FE286183
:1085B00000E0286900266E71002806D07448067015
:1085C000744801210170744806806A489621F7F7C3
:1085D000EAFD1DA864242146F7F7E5FD37A82146EA
:1085E000F7F7E1FD03A82146F7F7DDFD6E71EE8098
:1085F00051B0F0BDAA2838D1012A36D10220B86086
:1086000051B0F0BD0421B9600021B970787051B04B
:10861000F0BD3979534A5054481C38717978491F54
:10862000C0B281422FD10820B86051B0F0BD052200
:10863000BA60887051B0F0BD0621B960B87051B011
:10864000F0BD0721B960387051B0F0BD7A78062AC4
:1086500002921AD3531F0025424A2C46565DA41994
:10866000A4B26D1C9D42F9DB10E0032807D1022A59
:1086700005D10120F8700320B86051B0F0BD002092
:10868000B870B860787051B0F0BD00242018029A1C
:10869000821888781118BD7849193C780919FA7838
:1086A000002A00D0C91C2C4EC9B2FF2935D101289F
:1086B00009D0022831D11E2D36D1FFF7D7FC012079
:1086C000F08351B0F0BD284A94710320107190706E
:1086D000AA2050705520107068085071651DD57023
:1086E000400031181646D01D2246F7F743FD301DD5
:1086F000E11CEAB2D21C037892B2D218401C491E87
:10870000F9D1A019D143C171090A017209340120BC
:1087100000233146224608F05FF90020B870B860A7
:108720003871787051B0F0BD70190E4E3146224646
:10873000F7F720FD3078012802D12846FFF746FEE2
:1087400006F0F2F9BFF34F8F084809490160BFF303
:108750004F8F00BFFDE7C04632A901021890010209
:10876000E89801027CCD0102DC9A01020CED00E0E8
:108770000400FA05E4CC0102D5300100474E47471A
:1087800041000000257300000000F03F99AD010298
:108790002C940102AF9601029AAD0102F0B585B0AA
:1087A00008F072FD7B487C4903F0BCFD7B4C002542
:1087B0002571E57005F04AFBE061042003F0ECF858
:1087C000774E726828460495294608F08FFD05F01B
:1087D0003DFB0546206327204101706848430A217C
:1087E000F7F778FC60634119481C00D00846A06385
:1087F00005F02CFBE063A16B6A4D884202D3491956
:10880000884233D9684E694F05F020FBE06303F0DE
:10881000FBFC00280AD0FCF743F805F017FBE063E7
:10882000A16B8842F3D949198842F0D2E078012837
:108830000FD130783978814211D1707A20280ED149
:108840007079B179090208185949898D884206D191
:1088500033E0534842680020014608F047FDA16B11
:10886000E06B8842D0D349198842CDD801252846EB
:1088700001F06AF9284608F063FD2079002816D136
:108880004C4806F0D1F94E4E3378032056A20146EB
:1088900007F0E0FA3078411C3170062807D35848B9
:1088A000022101600498307060813D480570042009
:1088B00003F062F8002005B0F0BD012020713D48B2
:1088C000623006F0B1F905F0C1FAA061B27A039204
:1088D000A2707079B17909020818E08031460B3135
:1088E0005500354F384602912A46F7F743FCA9193F
:1088F0000B31384632302A46F7F73CFC039A002AFF
:10890000049834D000262D4D03E0BF1C761C9642FF
:108910000FD2388829688142F7D125488089798E1D
:108920000818788601B2E0880022FEF7C7FAA2781C
:10893000EBE7002A10D029680020029D16462A780D
:108940006B781B029A18914209D0AD1C401C32462C
:108950008642F3D1104608E00020024605E0C5B289
:108960002846FAF747FC2A46A078824202D1C0B2D4
:10897000FAF740FC124800210170052020560C49EE
:108980008B8D616A0091019003200EA2014607F0D1
:1089900061FA6BE765000100FDE900003099010212
:1089A00038900102007C3125D8D20102869801025C
:1089B00032A901021A3F0000649A0102AC98010238
:1089C000D6D20102B1EAC7A94944A3BA25582CBEA0
:1089D000E0C0EB3A20256420D0C5BAC5C7BFB6C8F1
:1089E000A3BA25642E0D0A00B2E2BEE0CAA7B0DC2D
:1089F000A3ACBCC6CAFDA3BA25640D0A00000000E2
:108A0000A0980102F0B585B008F03EFC744C607887
:108A100008F0E0F973498A8803A882800A884988A7
:108A200009048918039104F079F96078052804D0C5
:108A300002226D49092804D104E001226A4909286B
:108A400000D0891849792078621C08F087FA607A8A
:108A500005F08CFC6548664903F064FC654F002412
:108A6000FC7005F0F3F9F861042002F095FF624D07
:108A70002046029421462A4608F038FC05F0E6F923
:108A80005E49386379634118481C00D00846B863D2
:108A900005F0DCF9F863B96B594E884202D38919A5
:108AA000884234D9574C03F0AFFB00280AD0FBF7BB
:108AB000F7FE05F0CBF9F863B96B8842F3D9891951
:108AC0008842F0D205F0C2F9B861F87801280FD1D8
:108AD00020784D49097881420AD1607A202807D14F
:108AE0006079A179090208184849898D88421CD00B
:108AF00005F0ACF9F861002001462A4608F0F6FBC3
:108B0000B96BF86B8842CED389198842CBD801253E
:108B1000284601F019F8284608F012FC029C0420AF
:108B200002F02AFF204605B0F0BD394806F07CF877
:108B300005F08CF9B861A27A0292BA706079A179D5
:108B400009020818F88021460B315600314D28469D
:108B500001913246F7F70EFB31190B3128463230BE
:108B60003246F7F707FB029A002A24D000242A4E47
:108B700003E0AD1C641C94420BD22888316881420A
:108B8000F7D13220295EF8880022FEF797F9BA78EB
:108B9000EFE7002A11D031680020019D14462A78A1
:108BA0006B781B029A18914210D0AD1C401C2246D3
:108BB0008442F3D102E0002203E0002214469442F2
:108BC0000BD1D0B2FAF716FB0124A8E7C4B22046B5
:108BD000FAF710FBBA789442F3D001249FE7C0461D
:108BE000B69001020E1F0100C4A001026500010041
:108BF000FDE900003099010280841E000098E00E1B
:108C0000007C3125D8D201028698010232A90102E6
:108C10005C3F0000649A0102AC98010280B582B00A
:108C2000002001900448C268002A02D001A8002157
:108C3000904702B080BDC0468C950102F0B583B06C
:108C400000242046FEF742F8FEF765F8274EB06094
:108C5000FEF75EF87060264F0BE001A8C18880889F
:108C6000084319D101A8408824180834B068844208
:108C700035D201AD082128462246FEF733F8288870
:108C80000028EAD0B8422AD001AD0421284600F0DD
:108C900045FFA9888842E5D03460B06884420CD290
:108CA00001AD022128462246FEF71CF82888B8426A
:108CB00003D0A41CB0688442F2D370682118491E06
:108CC0004042084030600DD000242546012029464E
:108CD000FDF7E0FF03CE4D19083E8542F6D3346020
:108CE00003B0F0BD0024346003B0F0BD189701025A
:108CF000FFFF000010B5054C6070FEF745FE607880
:108D0000022801D10020607010BDC04668960102A3
:108D1000F0B585B01F4604920646C8170C184440AB
:108D20000A2C039114D301250A212046F7F7D2F922
:108D30006D1C632C0446F7D804998D4200D3294654
:108D40000A9C002F09D00398002808D4002207E0CD
:108D5000012504998D42F2D2F2E7002205E00122BA
:108D6000042323409B081343FA1A02232340049848
:108D70000028029412D1002B10D0F468002C62D489
:108D80000398002825D40298400734D57068B56848
:108D90006F1C87422FD830682B2423E0E407ECD1E6
:108DA000002A0AD1E9E7376820203855B560F06815
:108DB000441CF460521E002CDFD49142DDD277684F
:108DC000B468651CBD42EED9F468521E002CF4D57F
:108DD000D3E7404203907068B5686F1C87420AD899
:108DE00030682D244455B760F068441CF4600025B9
:108DF000ED43A84227DB002B1CD00120029B18402A
:108E0000049B184316D1002A03D113E0521E002CF4
:108E10000ED491420CD27068B3685D1C8542F5D8BF
:108E200030683024C454B560F068441CF460EDE749
:108E3000002C08D40092029801900A22304603992F
:108E4000049B00F003F805B0F0BD0000F0B587B05A
:108E50001F4615460290012406919142009407D3C3
:108E6000012406982946F7F735F9641CA842F9D27F
:108E70000D980C9ABC42039700D3039400990140CB
:108E8000002A009109D00029029C25D120218007C9
:108E900005D40846002F11D004E0029C1CE03020CD
:108EA000002F0BD0084609E023685854A260E168FF
:108EB000491CE1603246721E00290DD4039991428B
:108EC0000AD216466368A1684A1C9A42ECD9E16846
:108ED0003246721E0029F1D5E068002859D4059069
:108EE000012401E07F1E6C43022FFBD2069821462D
:108EF0001646F7F7EFF83246A842F4D20298806897
:108F00000490069F0195069738462146F7F7E2F848
:108F1000049D691C029F7A68914206D9069F059AB2
:108F2000019D0592002A0ED516E01B4A125C3B6893
:108F30005A55B960FA68521CFA600491069F019D67
:108F40000592002A08D460433F1A20462946F7F7C5
:108F5000C1F8AC420446D6D200980028029C059B7A
:108F6000049D16D0002E14D0701C01E0002B10D4EC
:108F7000401E039981420CD2691C62689142F5D867
:108F8000226820235355A160E268531CE3600D461C
:108F9000ECE707B0F0BDC04614220100F0B583B085
:108FA00001900291002923D00025124F2E460AE09D
:108FB00013480818410F4018C010B872761CB0B2A0
:108FC0000299884214D2019800884B24210100B2F2
:108FD00000F018F8400061014018388301B20648DB
:108FE00081422846E9DB05488142E1DD6420E4E76F
:108FF00003B0F0BD80980102E40C000004100000F2
:109000001CF3FFFF074A904201DD054A801800B2B9
:109010004143C817400D0818C00A00B27047C04647
:1090200000F0FFFFFF07000010B50078012819D1FC
:10903000AC480269012A04D1614A13680124A343A0
:109040001360032905D080214161C269002A05D13E
:1090500007E001214161C269002A02D001898069CB
:10906000904710BDFF222E32024803A107A305F04E
:1090700095FEC046C82D01006164635F646D615F49
:1090800063616C6C6261636B00000000556E657813
:1090900070656374656420646D61206368616E6EE1
:1090A000656C0D0A00000000F0B58DB00D4601247E
:1090B000EFF31081214002D1EFF3108372B6894E95
:1090C00073690F2B06DD102B37D0402B2FD0802B50
:1090D0002DD005E0002B2AD0012B01D11023736184
:1090E000B5813581B061F261002900D162B6317974
:1090F000002929D00294304C05A90A460495039012
:10910000E8CCE8C2E8CCE8C2029C204600F08CFD26
:109110002A4800902A4D294608312046039A049B8C
:1091200000F0F2FD2C60002420460DB0F0BD0029B7
:10913000FAD162B620460DB0F0BD02240029F3D169
:1091400062B620460DB0F0BD3178002907D01C482A
:10915000072181610460002420460DB0F0BD326912
:10916000B3891749002B15D0B5693089012A02D07F
:10917000002A03D003E09FB2874200D10C604F6801
:10918000FF07FCD08F6880C55B1E1F04EED1002353
:10919000B381B561012A02D10A68A2430A607461F1
:1091A000F2690024002ABFD0B36931898800181AF7
:1091B000904720460DB0F0BD5422010029900000D8
:1091C00008D00140F0B581B0002856D00446424E88
:1091D000F068800754D41325284600F0DDFB2846AC
:1091E00005F0B0FA27686168012538462840CA07AB
:1091F000920F1018227C1207120E8018627C120740
:10920000120D8018A27C1207120C8018627D1307C1
:109210001B0AC01812091206801830607D20060251
:109220000029304600D12D48E3681A0A7D2A1A46E3
:1092300029D22B4EB3422AD200292BD0002A29460C
:10924000254E00D01146F6F745FF401E80B27060F3
:1092500024480761E27C0270237D0371224F3E683F
:109260006902A468012C1BD02C0226433E60002B0F
:109270001ED00121184A116329E0012001B0F0BD80
:10928000022001B0F0BD3246154EB342D4D333466E
:109290000029D3D11A46002A29460F4ED2D1D2E74F
:1092A0003F242401A6437618F0363E60002BE0D11F
:1092B000002A0CD0FF2212020C4B1C68944301229E
:1092C000D203A2181A60304A1160304A116001219D
:1092D0004161002001B0F0BD00D001400026B8037C
:1092E00080841E00A09501022C06004008E400E0E6
:1092F00070B5002801D0012070BD0C461625284607
:1093000000F04AFB284605F01DFA002C05D01B484A
:10931000183014222146F6F72DFF28211748415C0A
:10932000002915D04168002916D403220B46934327
:10933000144A9C588D07ED0EFF26AE40B4439C5056
:109340001F220A40012191400F4A11600F4A11600B
:1093500001210161002070BD8A07D20EFF239340D6
:109360000F220A40083A03218A43054954589C4376
:10937000545001210161002070BDC046749001026B
:109380001CED00E000E400E080E200E000E100E02D
:1093900080B568480021017061480078C0016149CA
:1093A00009788901014360480078400108435F491A
:1093B0000978090101435E480078C00008435E490E
:1093C0000978490001435D4800780843C0B2FBF7C3
:1093D000A3F980BD80B5574801210170514800783C
:1093E00080014F490978C90101434F480078400185
:1093F00008434E490978090101434D480078C000EF
:1094000008434D490978490001434C480078084316
:1094100004210143C8B2FBF77FF980BD5A21014AFC
:10942000505270475CA00102F0B581B013490A7830
:10943000002A13D0052A01D104220A709300CD1806
:10944000561C00231C462F686F60F917DB194C412E
:109450002D1F761E012EF6DC084902E0002213467D
:1094600014464860521C0A70C11718186141D2B2E4
:109470000023F6F759FE01B0F0BDC046C0950102C9
:10948000F0B581B004460078414241412170244842
:109490000078C001234909788901014322480078F6
:1094A0004001084321490978090101432048007817
:1094B000C00008431F4F3978890001431E4D2878AA
:1094C000400008431D4E31780143C8B2FBF724F930
:1094D0007D20C00000F038FB2078414241412170DE
:1094E0000F480078C0010F490978890101430E48EF
:1094F0000078400108430D490978090101430C48EF
:109500000078C0000843397889000143287840007A
:10951000084331780143C8B2FBF7FEF801B0F0BD53
:10952000E09E0102AE9601021D90010264EA010272
:1095300099AD0102E19E010224A3010225A30102CB
:10954000B0B5094D28600224002120460A4602F0E9
:109550002BFA01210522204602F0BAFA2A680321DB
:10956000204602F099F9B0BDDC9E01025C219D48C5
:109570000022425282847A2141840284C28302837F
:10958000C2820282114941608260C2603D21490469
:1095900041834182090C8183818270475C2191481B
:1095A0000022425282847A2141840284C28302834F
:1095B000C2820282054941608260C2603D21490445
:1095C00041834182090C8183818270474C37373750
:1095D00070B585484C21016001252C02601C00F00B
:1095E0005BF9322000F0B0FA00F044F9284600F0B0
:1095F0004BF9284600F05AF800F036F90C4800F014
:109600004BF900263046314600F056FA28463146DE
:1096100000F052FA204600F03FF9022000F03CF939
:109620004834204605F032FB05F090FB70BDC04683
:109630000102000010B50446072106F069FA01484E
:10964000046010BD6096010270B505200424214617
:1096500002F016FA0620214602F012FA0A202146EC
:1096600002F00EFA0920214602F00AFA0024012134
:10967000204602F005FA022520462946224602F03D
:1096800027FA0B2630462146224602F08DF9304655
:109690002946224602F01CFA70BD0000024801680B
:1096A00001229143016070475800004002490A6856
:1096B00002408242FBD1704704600040B0B5494D82
:1096C00028688107484C0ED528797F2108402268F8
:1096D0008A431018206023680B4002200321434A6C
:1096E00006F0B8FB286880040ED55E20285C7F2138
:1096F000084062688A431018606063680B4002206B
:1097000003213B4A06F0A6FB172000F045F9394833
:10971000016802220A4301218A4302603648374920
:10972000016037480021C17181791F25294081716D
:10973000817A427C837C1B029A18C37C1B04D2185A
:10974000037D1B06D2182F4B9A4218D1427B837B94
:109750001B029A18C37B1B04D218037C1B06D21869
:10976000294B9A420BD1C27A037B491E122906D893
:1097700019028918254A914201D1202101720178EC
:10978000CA0602D11022114301701C3C206820211E
:10979000884320601E481F49016041680029FCD5AC
:1097A00003F020FA0446022003211BA2234606F000
:1097B00051FB0A20C441032C05D8022003211DA21D
:1097C00006F048FBFEE71848C1680F229143C160CC
:1097D0000168164A0A4002601920000114494860D5
:1097E0000D60B0BDC4A0010248000040102E010071
:1097F000FA2D0100040200400C060040AF6B100A75
:109800006B0001404D383650312E3236073400009F
:1098100000600040FE1C0080436869702049443AA3
:1098200020253038780D0A00C8600040FEFFC3FFD5
:109830000C0400404F6C642063686970206D6F6495
:10984000656C206973206E6F7420737570706F7211
:1098500074656420627920746869732053444B21D5
:1098600021210D0A0000000080B5172000F08CF8BF
:10987000002080BD10B51724204600F08DF820464A
:1098800004F060FF002010BD0121C9070143014819
:10989000016070470060004010B5C1B2000AC2B25A
:1098A00002290CD0012913D0002930D1911E7F4804
:1098B00002291BD20121032A2AD0490429E07B482E
:1098C0004168002A1FD00246203A1143416010BD72
:1098D00076480168D31E022B10D3012A29D0002A12
:1098E00041D1012292079143016010BD002A16D197
:1098F0000121490702688A43026010BD0123042A3E
:109900001FD05A041EE0012292079143416010BD0E
:109910000904194A7F32C36A13405918C1621749B2
:109920008A699207FCD50121490702680A4302604F
:1099300010BD0522120791430246203A0A430260F5
:1099400010BD1A04836A0C4C1C40A21882620B4A98
:10995000131F00241C600A4B0A4C1C600D235B0281
:1099600014681C431460054A93695B06FCD5052204
:1099700012071143016010BD80FFFCFF140200407C
:1099800004010040FF0F00000121814047480268A8
:109990008A4302607047C046012181404348026803
:1099A0000A4302607047C04610B5052811D8C0466A
:1099B0007844007940008744020E192434393B4929
:1099C0000A680868C0003CD53A4820390A425DD090
:1099D0003BE0002010BD35490A680868C00035D555
:1099E00034480B46203B1A4237D134E02F490A68ED
:1099F0000868C00036D52F480B46203B1A424CD190
:109A000035E02A494C680120C0030A680B46203B18
:109A10001C421AD00C68E4003BD5264C1A423CD0BC
:109A20003AE0224800680120C00310BD1F490A68BF
:109A30000868C0001ED51F480B46203B1A4220D1A3
:109A40001DE01B4820390A4220D010BD18480B46A3
:109A5000203B1A4201D10120C00349688900890FC7
:109A6000C84010BD12480B46203B1A4215D10120B8
:109A7000C00312E00E480B46203B1A4201D10120E0
:109A8000C00349680903890FC84010BD0120C00305
:109A900010BD074C1A4200D020464A689200920F2F
:109AA000D04049680901890FC84010BD200000401E
:109AB000006CDC020026B80304282CD8164AC046E5
:109AC0007844007940008744020A121A21000320DA
:109AD0000007136883438807800818181AE00320DA
:109AE00080061368834388070009181812E00320D2
:109AF0008004136883438807000B18180AE0FF20CE
:109B00000002136883430802181803E01068FF235B
:109B1000984340181060704724000040B0B5002200
:109B200000290CD0074B047895B22D0A65406C00D3
:109B30001C5B12026240491E401C0029F3D190B206
:109B4000B0BDC0461420010000280AD030B407255B
:109B50002C02CD256419604340091238001FFDD83E
:109B600030BC7047F0B583B01F4616460D4601461F
:109B7000E8680291F6F748FC04460F2E11D8082E2B
:109B800004D320462146F6F7E6FB09E0042E02D373
:109B90008120C10501E0412001062046F6F734FC92
:109BA00004460999089E2B20C043874205DB2046C6
:109BB0000F462146F6F7CFFB0DE03F20C04387421A
:109BC0000BDA4920C04387420CDBFF200F4681059A
:109BD0002046F6F719FC39460446688A0880346046
:109BE00003B0F0BD01915320C043874206DB2046FD
:109BF0002146F6F7B0FB0446688A10E0A86902998E
:109C0000F6F72CFE002801D1A88B00E0E88BF6F7D0
:109C100086FE01462046F6F7F7FB04460020019930
:109C20000880346003B0F0BDF0B581B00546012076
:109C3000072D66D80C46002963D04A4F3868016961
:109C4000C90736D105263046FFF7A6FE304604F098
:109C500079FD03CF0369012213430361002918D45E
:109C600003200B4683438E481E588807C00EFF27EB
:109C70008740BE4340278740374389481F501F20F5
:109C80000840824087480260874802603548006883
:109C90000FE08A07D20EFF2696400F230B40083BA9
:109CA00003218B437D495F58B743402696403E438E
:109CB0005E5069014018012109024218E369DB0680
:109CC0009B0CA569ED00EDB2EB185360626852077A
:109CD000520B23685B075B099A18A3685B079B0C10
:109CE000D218E3685B075B0DD21823695B01DBB216
:109CF000D21863699B07DB0ED218802313434350AD
:109D0000002001B0F0BDC046F0B581B0002A23D0DC
:109D100005460835134C2668F668EE40F50702D074
:109D2000022001B0F0BD069D8600A619B560400175
:109D300024682018009301231D0246197768072420
:109D4000A7437760F16032610099B16041591943CE
:109D50004151002001B0F0BD03A00AA174220DA35F
:109D600005F01CF8D4920102696E636C7564652F6E
:109D7000647269766572732F6D6B5F646D612E63BB
:109D800000000000646D615F7472616E73666572DD
:109D900000000000496E76616C6964207472616E27
:109DA00073666572206473742061646472000000DD
:109DB00000015849085840687047C046F0B581B066
:109DC00005460120012D4CD80C46002949D0002D14
:109DD00003D0012D04D10F2000E00E20FFF7DCFDA1
:109DE000A668012E04D0002E4FD1E08900284CD166
:109DF0002901294843580020D860F507AD0F27688E
:109E00006668B607360F76192569EA07920EB61806
:109E1000022F04D0012F03D10122164300E0403667
:109E20001D4F9E60E2681A6079188D606269CA6091
:109E30004968002917D403220B469343184A9C58BB
:109E40008D07ED0EFF26AE40B4438026AE4026437C
:109E50009E501F220A4001219140124A1160124A6D
:109E6000116001B0F0BD8A07D20EFF2494400F2389
:109E70000B40083B03218B4308495D58A5438024D0
:109E800094402C435C5001B0F0BD08A00FA14922C2
:109E900012A304F083FFC0461C9301021CED00E0F6
:109EA00000E400E080E200E000E100E0696E636C45
:109EB0007564652F647269766572732F6D6B5F646C
:109EC00075616C5F74696D65722E63006475616C99
:109ED0005F74696D65725F6F70656E00636F6E664B
:109EE000696720697320696E76616C69640000009F
:109EF0000001084A10580160816880220A4382608C
:109F00007047C04600010349085881688022914388
:109F1000816070471C930102F0B58DB00193154626
:109F20000E460A901298002408900480149F3C80EA
:109F3000139809900460159804900480FF2081050F
:109F40003046F6F761FA0290304603963146F6F74E
:109F500002FA2B463D460690274607950B9311E0E3
:109F60001180188880002858099908600120079DF1
:109F700028800520049908807F1CBCB21888844280
:109F800000D9A0E028880028F6D1A0000A9D2E580C
:109F900030460699F6F754FC002817D0304603994E
:109FA000F6F74EFC00280B9B079DE5D1089A178019
:109FB000099D2E601888011B012934D11080198851
:109FC00089000A9A51582960059035E0089A17804F
:109FD000099806600B9B1988081B0128C0D00C96B5
:109FE000019825187E1CB0B28542BFD389B2B2B2A7
:109FF0008A420ED880000A990C5820460C99F6F730
:10A0000011FC0B9B002804D1099804600898068075
:10A010000C94761CB0B28542A8D3198889B2B2B22A
:10A020008A42E7D9F5E70C96019962187D1CA9B21E
:10A0300016468A4205972CD2059884B2A5000A9E3E
:10A040007259002C104609D0A819001F016810464B
:10A050000C92F6F780F90C9A062C07D80446A8193A
:10A0600041681046F6F777F90C902046079D029953
:10A07000F6F7F4FB00280B9B07D10C980299F6F732
:10A08000DFFB0B9B002800D076E70120288003200F
:10A0900070E780B2AAB282420FD888000A990C58A1
:10A0A00020460C99F6F7BEFB0B9B002805D10998BA
:10A0B00004600898058005950C946D1CA9B28E4229
:10A0C000BAD31888E5E70DB0F0BD00000A490A6868
:10A0D0000A4802400A60FD214900094A1268515CA1
:10A0E000002908D007490A6C02400A6401200006D2
:10A0F0000A6882430A60704700040040FFFFFF7F48
:10A10000449401022000004000207047F0B583B065
:10A110000D4604467C26464350488719F869396A3B
:10A12000F5F7D8FFA84200D892E0019502940121EA
:10A13000EFF31080084002D1EFF3108272B63C4674
:10A1400010343B690025062B0CD80A469A40D306EA
:10A150005B0F06D161231A4275D00D46002803D04B
:10A1600003E00225002800D162B6002D02D0284667
:10A1700003B0F0BD00943C4620343848805910218B
:10A18000C1613E46143604F0DBFD05463868C069FF
:10A19000C00605D504F0D4FD401B31888842F5D9AE
:10A1A0000621029D284600F00BFF206801994143DB
:10A1B000B869091838688160172179563C46173408
:10A1C000002909D5C16920220A43C2610121F9662B
:10A1D000890502680A4302600521284600F0F0FE66
:10A1E000207840B200250028C1D42B4800687D2487
:10A1F000E100F5F76FFF61014143029800F0B2FE04
:10A2000004F09EFD04463868C069C00705D004F01C
:10A2100097FD001B31888842F5D904F091FD044672
:10A220003868C169890706D504F08AFD001B3188AA
:10A230008842F5D938680121009A1160534981613B
:10A24000284603B0F0BD0321216000288CD08CE7A4
:10A25000034804A1084A09A304F0A0FD48930102A1
:10A26000402E0100666C6173685F626C6F636B5FA8
:10A2700065726173650000005D020000626C6F63CF
:10A280006B20696478206973206F76657220726133
:10A290006E67650D0A000000F0DF0102F0B583B0C3
:10A2A00002907C214143934A5418E56EEAB2511E54
:10A2B00002291FD229040126090E18D00196009206
:10A2C000022100F07DFE2746143704F039FD0646D2
:10A2D0002068C169890606D404F032FD801B3988E4
:10A2E0008842F5D92068007DC007019E08D030461D
:10A2F00003B0F0BD032A36D100922804000E36D0F8
:10A3000020466C302D0C0021019101602746143746
:10A3100004F016FD06462068C069C00705D004F0A9
:10A320000FFD801B39888842F5D904F009FD0646E7
:10A330002068C169890706D504F002FD801B3988B1
:10A340008842F5D9206811498161E9B201200029CC
:10A3500011D003290099019E00D006202061226FB0
:10A36000002A0ED1C3E70026304603B0F0BD012617
:10A37000304603B0F0BD0099019E2061226F002A93
:10A38000B5D002A89047304603B0F0BD000093EB73
:10A3900070B5002801D0012070BD7825CD4E705DCC
:10A3A00000280ED000240921204600F009FE0F20CD
:10A3B000FFF7CAFB1520FFF7E7FA74553461204612
:10A3C00070BD042070BDC046F0B581B00C46007869
:10A3D000484EF16881422CD1032C54D1706EB16E7D
:10A3E000884261D900240621204600F0E9FD30684A
:10A3F000F16D81602046214600F0E2FD3546603572
:10A400002CCDF0683168B48C414F00975B1BA342A0
:10A4100000D81C46A3081431FFF776FCB06E001973
:10A42000B066306E00193066F06D0019F06501B04D
:10A43000F0BDB168814255D1032C45D1F08CF16D4E
:10A440000918F165316E09183166B16E0818B066E9
:10A45000716E814238D900240621204600F0B0FDFB
:10A460003068F16D81600121204600F0A9FD316E58
:10A47000B068F38C3268264C009414329B08FFF7C6
:10A4800043FC01B0F0BD30681021C16104F058FCFC
:10A4900005463068C069C00616D504F051FC401B63
:10A4A000B18A8842F5D90FE030681021C16104F00B
:10A4B00047FC05463068C069C00605D504F040FC7D
:10A4C000401BB18A8842F5D90120C1073268136860
:10A4D0008B431360F16E22040A4300021043F066BE
:10A4E00001B0F0BD4D200201034804A1844B04F0EB
:10A4F00055FCC04648930102402E0100666C617312
:10A50000685F646D615F63616C6C6261636B0000C6
:10A51000C9A30000F0B581B000786E4DAA688242F0
:10A5200000D0D0E001263002032942D16A6DAA662C
:10A53000AB6DAC6AA418EB652C66AB6C5B1CAB64B2
:10A540006B6E934235D95E30FFF7FEFA686CA96CEA
:10A5500002293AD3814238D1E88C696D08186865C0
:10A560000020062100F02CFD2868E96D81602F6D28
:10A5700004F0E6FB04462868C069C00705D004F073
:10A58000DFFB001BA98A8842F5D904F0D9FB0446F9
:10A590002A68D069800706D504F0D2FB001BA98A7F
:10A5A0008842F5D92A687420285C012841D0F1043A
:10A5B00040E0F2072B681C6894431C60EA6E0904B3
:10A5C00011430143E96601B0F0BD0229FBD381428A
:10A5D000F9D2E88C696D09186965A96D0818A86534
:10A5E0000020062100F0ECFC2868E96D8160EF8C0A
:10A5F00004F0A6FB04462868C069C00705D004F033
:10A600009FFB001BA98A8842F5D904F099FB0446F8
:10A610002A68D069800706D504F092FB001BA98A3E
:10A620008842F5D92A687420285C012822D0F104D8
:10A6300021E03105334B3B405918012802D0192045
:10A64000400601E00720C00608182F494018506056
:10A65000002F0DD004F074FB04462A68D0698007EF
:10A6600006D404F06DFB001BA98A8842F5D92A683C
:10A670002B6D1FE03105234B3B40C918012802D048
:10A680001920400601E00720C00608181E4940189E
:10A690005060002F0DD004F053FB04462A68D069A7
:10A6A000800706D404F04CFB001BA98A8842F5D928
:10A6B0002A68EB8C296EA868144C00941432FFF7BA
:10A6C00023FB01B0F0BD044804A10C4A0C4B04F07C
:10A6D00065FBC04648930102402E0100666C617321
:10A6E000685F646D615F77726974655F6E627974CB
:10A6F00065735F63616C6C6261636B007204000080
:10A70000272E0100FF3F00000080800015A50000FB
:10A71000F0B587B004460126880E14D01546002AED
:10A7200011D00F468120C004401B88420BD37C20EF
:10A730006043F04908180590818C38460691F5F77A
:10A74000C9FC002902D0304607B0F0BD2846069962
:10A75000F5F7C0FC0029F6D1059880693E1A30460D
:10A760000699F5F7B7FC0746039670190190069E07
:10A770003146F5F7AFFC0546C01B04900598006A0A
:10A7800002903146F5F7A6FC049981420FD20026CB
:10A79000BD42D8D92046394600F018FB2046FFF7C5
:10A7A0007DFD0028FAD17F1CAF42F3D3CBE70090A8
:10A7B0000398029D2946F5F78DFC0646284670430E
:10A7C0000399081A019800D0761C2946009D75430C
:10A7D000F5F780FC0590029941430198401A0390D7
:10A7E0000699F5F777FC0490AF420BD22046394624
:10A7F00000F0ECFA2046FFF751FD0028FAD17F1C4B
:10A80000AF42F3D305988642069D009F0CD22046A6
:10A810003146FFF77BFC2046FFF740FD0028FAD1C8
:10A82000761C05988642F2D30398A84203D20026EC
:10A83000304607B0F0BD059847430025E91920468A
:10A8400000F0C4FA2046FFF729FD0028FAD16D1C5C
:10A85000002604988542F1D375E7C046F0B585B06F
:10A86000002803D00124204605B0F0BD7822A14F76
:10A87000B85C002803D00024204605B0F0BD049247
:10A88000002905D0384614300CC90CC01CC91CC0A6
:10A890000020F86615242046FFF77EF8204603F0D6
:10A8A00051FF38681021C16104F04AFA0446386843
:10A8B000C169C90607D504F043FA001BB98A88426A
:10A8C000F5D9386800E0B98ABA7D1207120B521820
:10A8D000F97DCB07DB08D2188B07DB0F5B05D2189D
:10A8E000CB06DB0FDB05D2184B07DB0FDB06D218DC
:10A8F0008B06DB0F5B07D2180907C90F89071143C5
:10A90000016000240A21204600F05AFB3220FFF7A4
:10A910001BF90821204600F053FB04F011FA05460C
:10A920003868C169890606D404F00AFA401BB98A5E
:10A930008842F5D93868017D0A46C23A53425341EC
:10A9400074257B550904027D12025118007D0B18F5
:10A950000220032668A2314605F07CFA785D0128C2
:10A96000039619D1F87D029000260621304600F0AA
:10A9700027FB0721304600F023FB01210298814389
:10A98000785D012847D13868890101750675752100
:10A99000795C012938D048E00020032100F010FB49
:10A9A00004F0CEF906463868C169890606D404F079
:10A9B000C7F9801BB98A8842F5D93868007D4608F6
:10A9C0000122F87D014631431640C90701D03040CD
:10A9D00036D00295002506212846019200F0F0FAB3
:10A9E00007210095284600F0EBFA019846400298AE
:10A9F000385C012813D13868B101017500990175DF
:10AA00007521795C012910D114307621795C4A4294
:10AA10004A41510008E038680675490003E038688B
:10AA200000990175710014300170374800687D216C
:10AA3000C900F5F74FFB28214143002000F092FAAE
:10AA40007720385C012803D102200021FFF734F879
:10AA500004F076F906463868C069C00705D004F0EE
:10AA60006FF9801BB98A8842F5D904F069F9064666
:10AA70003868C169890706D504F062F9801BB98A74
:10AA80008842F5D93868D0498161172038560028A6
:10AA900029D57868002816D40146039A91431C4AA8
:10AAA0008B588507ED0EFF26AE40B3438026AE409F
:10AAB0001E438E501F210140012088401549086027
:10AAC000154908600FE08107C90EFF228A400F2355
:10AAD0000340083B039883430C481D58954380224C
:10AAE0008A402A431A50012004997854386120463C
:10AAF00005B0F0BD489301026A656465635F6964EF
:10AB00002025780D0A000000F0DF01021CED00E0B6
:10AB100000E400E080E200E000E100E0F0B593B086
:10AB20007C270A9047439348C619980704D0F07DC4
:10AB30004024044000D017E10125880E2ED0002BC0
:10AB40002CD08120C004C01A884227D30992012248
:10AB5000EFF31084144002D1EFF3108072B6304648
:10AB6000103005903069002506280891069310D80A
:10AB7000079414468440E106490F04D161210C4238
:10AB800003D0154604E0022502E00221059B19606E
:10AB9000079C002C00D162B6002D02D0284613B0CD
:10ABA000F0BD344617347348C05910210491C16177
:10ABB0003746143704F0C4F805463068C069C0064B
:10ABC00005D504F0BDF8401B39888842F5D92078B6
:10ABD000400665D40297B78C069C20463946F5F7A7
:10ABE00079FA079039464143601A03903546243577
:10ABF000A74200D894E0039800281CD006210A9CA4
:10AC0000204600F0DDF92888079948430899401844
:10AC10003168886000272046039C394600F0D0F94F
:10AC2000079B099A28885843C0193168097D115437
:10AC30007F1CA742F6D330680499C16104F080F804
:10AC40000446029D3068C069C00605D504F078F856
:10AC5000001B29888842F5D904F072F80446306850
:10AC6000C069C00705D004F06BF8001B2988884232
:10AC7000F5D904F065F804463068C169890706D53E
:10AC800004F05EF8001B29888842F5D9306801215C
:10AC9000059A1160B24981610025284613B0F0BDC4
:10ACA00003200025089FF7650999316606997166AA
:10ACB000B566F0660120C00731680A6802430A6081
:10ACC00006210A9C204600F07BF930688760204608
:10ACD000294600F075F93A4F0BAA0A921BCF1BC206
:10ACE0001BCF1BC2B48CF0680A99FEF79DFFF06879
:10ACF0003168344A0092069A944200D31446A3085D
:10AD00001431099AFFF700F8B06E0019B066306E82
:10AD100000193066F06D0019F065284613B0F0BDDB
:10AD2000002404E0641C0798844200D363E70621F2
:10AD30000A9800F045F9288860430899401831685E
:10AD4000886000270A98394600F03AF928880028D8
:10AD5000099AE7D0604310183168097DC1557F1CFE
:10AD600028888742F6D3DDE7034804A1064A07A3F3
:10AD700004F014F848930102402E0100666C6173E0
:10AD8000685F726561640000C60300005468652056
:10AD9000444D412072656164206C656E6774682063
:10ADA00073686F756C6420626520746865206D75CA
:10ADB0006C7469706C65206F6620340D0A000000A9
:10ADC000B4220100C9A30000000093EBF0B583B0EA
:10ADD0000D4604467C26464351488719F869B98CCC
:10ADE000F5F778F9A84200D894E001950294012182
:10ADF000EFF31080084002D1EFF3108272B63C46A8
:10AE000010343B690025062B0CD80A469A40D3061D
:10AE10005B0F06D161231A4277D00D46002803D07C
:10AE200003E00225002800D162B6002D02D028469A
:10AE300003B0F0BD00943C462434394880591021B9
:10AE4000C1613E46143603F07BFF05463868C06991
:10AE5000C00605D503F074FF401B31888842F5D940
:10AE60000621029D284600F0ABF820880199414355
:10AE7000B869091838688160172179563C4617343B
:10AE8000002909D5C16920220A43C2610121F9665E
:10AE9000890502680A4302600421284600F090F800
:10AEA000207840B22C4600250028C0D42B480068EA
:10AEB0007D21C900F5F70EF920492D314143204687
:10AEC00000F050F803F03CFF04463868C069C00742
:10AED00005D003F035FF001B31888842F5D903F017
:10AEE0002FFF04463868C169890706D503F028FF9B
:10AEF000001B31888842F5D938680121009A116019
:10AF000017498161284603B0F0BD03212160002864
:10AF10008AD08AE7034804A1084A09A303F03EFF48
:10AF200048930102402E0100666C6173685F73658F
:10AF300063746F725F657261736500002B020000BD
:10AF4000736563746F7220696478206973206F760B
:10AF500065722072616E67650D0A0000F0DF010204
:10AF6000000093EBF0B583B001917C220290424344
:10AF700053498C182546143503F0E2FE064602219B
:10AF8000029800F01DF803F0DBFE07462068C16957
:10AF9000890606D403F0D4FEC01B29888842F5D95F
:10AFA0002068007DC00708D06420FEF7CDFD03F0C7
:10AFB000C7FE801B01998842E1D903B0F0BDC046AD
:10AFC000F0B585B0049104467C2060433C490F18DD
:10AFD0003D46143503F0B4FE06463868C069C00724
:10AFE00005D003F0ADFE801B29888842F5D903F017
:10AFF000A7FE06463868C069800705D503F0A0FEA5
:10B00000801B29888842F5D91421049B5943DC20F0
:10B0100060432C4A1018039002914018018A8268FC
:10B02000C47C7426BE5D012E0DD10191012B0299C5
:10B030000CD0012B0DD07526BE5D012E0ED0019EC9
:10B04000072B0ED10EE00E4602990BE00222012BD7
:10B05000F1D138247526BE5D012EF0D10326072BD1
:10B0600000D0019E184B334024069207D20A1219D1
:10B07000D218039B5958C907490C52184168CB078D
:10B080001B0CD218837C5B075B0BD218C06840078F
:10B09000000A10183A685060002E0ED001290CD119
:10B0A00003F04EFE04463868C069800705D403F0FB
:10B0B00047FE001B29888842F5D905B0F0BDC0467F
:10B0C00048930102FC230100FF3F0000F0B59DB052
:10B0D0000D460126890E2FD0002B2DD011928121F3
:10B0E000C9041093C91AA94226D30121EFF3108491
:10B0F0000C4002D1EFF3108272B67C220F904243D3
:10B10000E74814928718384610303B690026062B12
:10B110000DD80A469A40D3065B0F07D161231A4225
:10B1200000D16FE30E46002C03D003E00226002C72
:10B1300000D162B6002E02D030461DB0F0BD0290A4
:10B14000BD650021139179651098401E1290401939
:10B15000B964B9690D916E1A1199B962FD623863CB
:10B160007E63F98C0E913046F4F7B4FF0446B86361
:10B17000129830180E9E3146F4F7ACFF109B011B5D
:10B180004A1CF86339647A64139A0029194608D076
:10B19000704359190D9BC91A0A1A7443581B801918
:10B1A0000119384648300E90384644300D903846E4
:10B1B00040300B9038462630059038465830139072
:10B1C000384654301290F9643A651498B4490858D6
:10B1D0001021C16138461430149038465030049024
:10B1E0003D464C3503F0ACFD04463868C069C006E6
:10B1F00006D503F0A5FD001B149909888842F4D9EF
:10B20000F87D40060C9500D574E201230E9803608A
:10B210000D98016800290F9800D1CDE23A467432AA
:10B220000A92DA0407921A05099219225206069226
:10B230000722D206089216E09A4800687D21C900CC
:10B24000F4F748FF109941430F9C2046FFF78AFE10
:10B2500020460C9D0E9A11684B1C13600D990968CD
:10B260008B4200D9A8E20B9A1268012A55D0002A15
:10B2700000D0A8E02E6812990C6813990D68062179
:10B280001091FFF79DFE386885601198051903F04D
:10B2900057FD04463868C069C00706D003F050FD6A
:10B2A000001B149909888842F4D903F049FD04462B
:10B2B0003868C169890707D503F042FD001B14995E
:10B2C00009888842F4D938680A990A78012A0899C5
:10B2D00000D00699012A099A00D0079A3346724C89
:10B2E000234013430B4371490B434360002EA3D00B
:10B2F00003F026FD04463868C069800706D403F0D1
:10B300001FFD001B149909888842F4D938682978F0
:10B3100001756D1C761EFAD18EE7012B00D0C7E0B7
:10B320002E6812990C6813990D6806211091FFF789
:10B3300047FE386885601198051903F001FD044641
:10B340003868C069C00706D003F0FAFC001B1499E6
:10B3500009888842F4D903F0F3FC04463868C169CF
:10B36000890707D503F0ECFC001B14990988884273
:10B37000F4D938680A990A78012A089900D0069900
:10B38000012A099A00D0079A3346474C23401343B9
:10B390000B4346490B434360002E69D003F0D0FCB9
:10B3A00004463868C069800706D403F0C9FC001B56
:10B3B000149909888842F4D93868297801756D1C78
:10B3C000761EFAD154E0012B00D0C9E02E68129904
:10B3D0000C6813990D6806211091FFF7F1FD38688C
:10B3E00085601198051903F0ABFC04463868C06904
:10B3F000C00706D003F0A4FC001B149909888842FA
:10B40000F4D903F09DFC04463868C169890707D563
:10B4100003F096FC001B149909888842F4D9386817
:10B420000A990A78012A089900D00699012A099AEE
:10B4300000D0079A33461C4C234013430B431B494F
:10B440000B434360002E13D003F07AFC04463868A7
:10B45000C069800706D403F073FC001B14990988A7
:10B460008842F4D93868297801756D1C761EFAD1A6
:10B470000C4800687D21C900F4F72CFE1099414367
:10B480000F9C2046FFF76EFD20460C9D2A68139BFB
:10B49000196889181960129B196889181960D9E60A
:10B4A00048930102F0DF0102FF3F000000808000AE
:10B4B0008B4200D0CEE604990E6812990C6813995D
:10B4C0000D6806211091FFF77BFD386885601198A3
:10B4D000051903F035FC04463868C069C00706D07A
:10B4E00003F02EFC001B149909888842F4D903F05C
:10B4F00027FC04463868C169890707D503F020FC9A
:10B50000001B149909888842F4D938680A990A7886
:10B51000012A089900D00699012A099A00D0079AB1
:10B520003346D44C234013430B43D3490B4343606E
:10B53000002E00D180E603F003FC04463868C069A1
:10B54000800706D403F0FCFB001B1499098888428D
:10B55000F4D93868297801756D1C761EFAD16BE62E
:10B56000129A1268119CA618139A15688B425FD123
:10B5700004990C6806210391FFF722FD3868856065
:10B5800003F0DEFB05463868C069C00706D003F04B
:10B59000D7FB401B149909888842F4D903F0D0FBEB
:10B5A00010900C9D3868C169890708D503F0C8FB65
:10B5B0001099401A149909888842F3D938680A9971
:10B5C0000A78012A089900D006991091012A099A4F
:10B5D00000D0079A2346A7490B40134310990B4309
:10B5E000A5490B434360002C14D003F0A9FB109035
:10B5F0003868C069800707D403F0A2FB1099401A8D
:10B60000149909888842F3D9386831780175761C15
:10B61000641EFAD19A4800687D21C900F4F75AFDEA
:10B62000039941430F9C2046FFF79CFC204611E6FE
:10B6300005990C8806210391FFF7C2FC38688560E4
:10B6400003F07EFB05463868C069C00706D003F0EA
:10B6500077FB401B149909888842F4D903F070FBEA
:10B6600010900C9D3868C169890708D503F068FB04
:10B670001099401A149909888842F3D938680A99B0
:10B680000A78012A089900D006991091012A099A8E
:10B6900000D0079A234677490B40134310990B4378
:10B6A00075490B434360002C14D003F049FB109004
:10B6B0003868C069800707D403F042FB1099401A2C
:10B6C000149909888842F3D9386831780175761C55
:10B6D000641EFAD16A4800687D21C900F4F7FAFCBB
:10B6E000039941430F9C2046FFF73CFC20460599F7
:10B6F0000A88CCE65E4815A90A4678C878C278C898
:10B7000078C20125E8073A68136803431360B868F4
:10B71000FEF78AFA02200026139C2168BA6AF965AE
:10B720003A6610997966BE66F8660C980068129AB7
:10B730001168091811600E9B19684A1C1A6022686A
:10B7400010182060002900D0F6E4109538466030CB
:10B7500013903C465C3438460830129006210F980E
:10B76000FFF72EFC3868216881600C980068119002
:10B7700003F0E6FA04463868C069C00706D003F053
:10B78000DFFA001B149909888842F4D903F0D8FA2B
:10B790000446109D3A68D069800707D503F0D0FAB7
:10B7A000001B149909888842F4D93A687420385CDF
:10B7B00001282DD0E9042CE003F0C2FA04463868D1
:10B7C000C069C00706D003F0BBFA001B14990988B2
:10B7D0008842F4D903F0B4FA04463868C16989078D
:10B7E00007D503F0ADFA001B149909888842F4D9F3
:10B7F00038680121029A1160224981610026304691
:10B800001DB0F0BD04210160002C00D191E491E451
:10B810002905119C174B2340591801280C9D02D073
:10B820001920400601E00720C006081812494018F8
:10B830005060002C0ED003F083FA04463A68D069B9
:10B84000800707D403F07CFA001B1499098888420A
:10B85000F4D93A682B681398016812980068074C6D
:10B8600000941432FEF750FA30461DB0F0BDC046C9
:10B8700074220100FF3F00000080800015A5000039
:10B88000F0DF0102000093EB3920C0000149096894
:10B8900008587047D4920102F0B5032920D8C04659
:10B8A0007944097949008F4401080F15012181402D
:10B8B0004F4B1B685963D96212E0012181404C4B08
:10B8C0001B681963D9620BE001218140484B1B685A
:10B8D000596304E001218140454B1B68196399625B
:10B8E00083004349CB18DA608A68002A29D14A6864
:10B8F000002A16D4032314469C43174BE558960799
:10B90000F60EFF27B740BD438027B7402F43E750CF
:10B910001F23134001229A40104B1A60104B1A60EB
:10B920000FE09307DB0EFF259D400F241440083CD9
:10B9300003229443074AA658AE4380259D403543D1
:10B94000A55001228240086802628868104388601E
:10B95000F0BDC0461CED00E000E400E080E200E045
:10B9600000E100E010B501242046FEF715F820465E
:10B9700002F0E8FE002010BD012181401C48006853
:10B9800042688A4342607047194909680968C140A2
:10B99000012008407047C0460121814014480068DA
:10B9A00042680A4342607047012907D0002910D13C
:10B9B000012181400F4802680A430FE001218140C4
:10B9C0000B4800684368002A0DD00B4343600161B7
:10B9D000704701218140074802688A430260044899
:10B9E0000068416170478B43436001617047C04606
:10B9F000D89301020801004080B5114A1170114A24
:10BA000010708001C90101430F48007840010843CC
:10BA10000E490978090101430D480078C000084328
:10BA20000C490978890001430B480078400008431D
:10BA30000A4909780143C8B2F8F76EFE80BDC046D6
:10BA4000E09E0102AE9601021D90010264EA01022D
:10BA500099AD0102E19E010224A3010225A3010286
:10BA6000012282400548002903D00168114301608A
:10BA700070470168914301607047C0460001004073
:10BA8000124A072809D880000F23834081401940BB
:10BA9000106898430843106070470F280AD8800048
:10BAA00020380F2383408140194050689843084351
:10BAB00050607047800040380F2383408140194018
:10BAC00090689843084390607047C0463400004037
:10BAD000F0B54307DC0E0726A640C3089D000E4BB9
:10BAE000EF187D68B5433E1D002908D0356001225E
:10BAF000824001290CD1186810431860F0BD012163
:10BB00008140186888431860A24015433560F0BD35
:10BB1000186890431860F0BD0C01004010B582B069
:10BB200014460A46014604980093019008202346D3
:10BB300000F092F802B010BDB0B584B014460A46C9
:10BB4000014608980225009501930290072023469C
:10BB500000F052F904B0B0BD70B500285BD0314997
:10BB60000A783149002A03D14A68012313434B6004
:10BB7000428803881B049A180B46183B1A60828877
:10BB800083891B049B180C460C3C23600B46083B26
:10BB900084681C60446903232340057CAD00EB18D6
:10BBA0008569AD072D0D5B19457C2D035B19C569B2
:10BBB000AE07B60A9B19867CB6059B190E1F33602B
:10BBC000036A122B04D107240C60541EA2410AE020
:10BBD000032C05D1012D03D807220A60012202E0BF
:10BBE00006220A600122114C002525700F246401F1
:10BBF0002034C57C6D0225401B069B0BD218C379EF
:10BC00001B07DB0ED21880790007C00D10184019F1
:10BC10001439086070BD064806A1862209A303F006
:10BC2000BDF8C046DCCC010218100050DECC010289
:10BC30001D3B01006C73705F656E67696E655F72B6
:10BC4000756E0000506172616D6574657220697374
:10BC5000206E756C6C000000F0B58BB0109E340443
:10BC60003ED00D46D64C2140012701977F06B942B0
:10BC70003CD111462140B9423FD11C40BC4243D186
:10BC8000119902AC0027E781E78066802780278230
:10BC9000A774E1749908A181A908A1800A90099765
:10BCA00008970797900880B204902046FFF754FF4A
:10BCB000AA480078002801D00BB0F0BDAB4801685D
:10BCC000C90708D10168C90705D10168C90702D1B0
:10BCD0000168C907F3D07F48019901700BB0F0BD2E
:10BCE000B8480D49AF22C14B03F058F80095B5484C
:10BCF0000949B022754B03F051F80092B14806494A
:10BD0000B122724B03F04AF80093AE480249B222C6
:10BD10006E4B03F043F8C046F33A0100F0B58DB026
:10BD20000392139E340446D00A46A54C21400125B7
:10BD300002956F06B94244D103992140B94247D1D7
:10BD40001C40BC424CD11499129D04ACE1742949A9
:10BD500021820027E781E780668027809908A181FA
:10BD60009108A1800B95012D01D16121CF43A774CA
:10BD70000C9002200A9009900398800880B20690E7
:10BD80002046FFF7E9FE75480078002801D00DB085
:10BD9000F0BD76480168C90708D10168C90705D117
:10BDA0000168C90702D10168C907F3D0494802995F
:10BDB00001700DB0F0BD83480D49FB228B4B02F0A2
:10BDC000EDFF00927F480A49FC22404B02F0E6FF5B
:10BDD000039800907B480649FD223C4B02F0DEFFB1
:10BDE000009378480249FE22384B02F0D7FFC04644
:10BDF000003B01008E8E0000F0B58BB0119E340424
:10BE000047D00D466E4C2140012701977F06B9426D
:10BE100045D111462140B94248D11C40BC424CD1C9
:10BE20001299109F02ACE174294921820021E1811D
:10BE3000E180668021809908A181A908A1800997E5
:10BE4000012F01D0712100E06121C943A1740A9042
:10BE5000032008900790900880B204902046FFF7D6
:10BE60007BFE3E480078002801D00BB0F0BD3F4873
:10BE70000168C90708D10168C90705D10168C90768
:10BE800002D10168C907F3D01248019901700BB0C3
:10BE9000F0BD4C480C49D522544B02F07FFF009571
:10BEA00048480949D622094B02F078FF00924548DC
:10BEB0000549D722054B02F071FF00934148024922
:10BEC000D822024B02F06AFF0F3B01003D3B01000C
:10BED00086860000DECC010210B582B014460A4608
:10BEE000014600200093019004202346FFF7B4FE92
:10BEF00002B010BD10B584B014460A4601460020B9
:10BF000000900193029004202346FFF707FF04B03E
:10BF100010BD000070B50D46064604242046FDF70E
:10BF20003BFD204602F00EFC0B4805600B480670F6
:10BF3000002E0ED00A48016880220A437F218A43DE
:10BF400002600120000307490860074908600748AC
:10BF50000460002070BDC046E0CC0102DCCC0102D0
:10BF60000CE400E080E200E000E100E01C10005082
:10BF7000B0B582B0144602461148204001256D0636
:10BF8000A8420DD1180413D0174801600020009377
:10BF90000190062011462346FFF75EFE02B0B0BDB9
:10BFA0000094FF228C320748074908A302F0F6FEEE
:10BFB000FF208C30421C034803490C4B02F0EEFE7C
:10BFC0000300FCFF1D3B0100E53A010044737420AF
:10BFD0006164647265737320257820697320696ECB
:10BFE00076616C6964000000081000505B3B010042
:10BFF00080B582B00B4601460020009201900320DC
:10C000000A46FFF729FE02B080BD0000002801D0DB
:10C01000042100E00221C54A5172411E884180017D
:10C0200003490A6840239A43101808607047C046C5
:10C0300050A00050F0B583B002912E49CD7A0E7B0E
:10C04000771987424FD90899019118254543412610
:10C05000F604BF00BE19745B34490C4057033C1909
:10C060009B07D90C6418324B1B681B7A74537519E3
:10C070006C880326B60326409B079B0C9B193F2424
:10C0800004401819029CA3061B0DC0186880012AE1
:10C09000184E13D8707B14224243307B5023434305
:10C0A00024011B199A18F37AC0181C234343D01893
:10C0B00080081E4A104007430F432F800198686094
:10C0C00001F0C4FEA860E8681A4908403030E86012
:10C0D000286908402721715C4018286100F044FE5F
:10C0E000686103B0F0BDFF228832034803A108A3B2
:10C0F00002F054FEE4D10102AC3B01006D61635FCC
:10C1000063735F636F6E7374727563740000000015
:10C11000435320696E646578206973206F76657279
:10C120002072616E67650D0A00000000FF070000C5
:10C13000449401020000F0FF2820D84900220A544C
:10C140007047C046F0B581B0009314460D460746CF
:10C1500006263046FDF720FC304602F0F3FA262191
:10C160001D48475400210170417081710171817037
:10C170004171C170C17102224272C16201634163A7
:10C18000816304734273C572009A561C134A168069
:10C1900001724120C00401214903F4F704F8502042
:10C1A00060432901081861198A00801818224A433F
:10C1B0008018B2B24A438018094940180949884298
:10C1C00004D200F0B5F8002001B0F0BD064807A188
:10C1D0009A2209A302F0E2FDE4D10102E0D10102BA
:10C1E0002800080201200802AC3B01006D61635F7A
:10C1F000696E697400000000454D206F76657266B7
:10C200006C6F770D0A000000A448C179002901D0A5
:10C2100001207047007A411E88417047F0B583B015
:10C2200002912A494B7B834248D9CB7A0C7BE31895
:10C2300018245C439B00E3184124E4041A191424D5
:10C240000190054665430026565100925519EE8827
:10C250002E4F0B467A1C3240F54E3688497A711AB9
:10C260002B4E0E40B618EE803740997BEF80AA889F
:10C27000284F17404A424A4191007918264A8918A6
:10C28000A980264F0F402D1D029801280AD124496C
:10C290000E400921C902711869800121C90379186A
:10C2A000298000E02F800198444300980019074A34
:10C2B000918C4182118C018203B0F0BD3520C20007
:10C2C000034804A109A302F069FDC046E4D10102BC
:10C2D000AC3B01006D61635F6C696E6B5F6465739D
:10C2E000635F636F6E737472756374004C696E6B19
:10C2F000206465736320696E646578206973206FBC
:10C300007665722072616E67650D0A00FFFBFFFFA4
:10C31000FF03000003D0FFFFE80F0000EF1F000045
:10C32000FF830000BE4A506391637047E4D101026D
:10C33000F0B581B04348CC21016003214160B84988
:10C340000A7BD304404C1B19CC7AA218541E1C4300
:10C350001823534392009A184B7B14255D435219BE
:10C360009201224301246306134343610022826247
:10C37000C262026342638263C26342650267334BF7
:10C380001A605A609A60324B1A601A619A61DC61D5
:10C39000304C1C62304C251D1D6325460C3D5D63F1
:10C3A0002546283D9D632D4EDE631C645C642C4D48
:10C3B0002F461C379F642746143FDF64103C1C65E2
:10C3C000284C5C65284C9C650C369E67274CA56301
:10C3D0004035E563DA651A665A669A66DA661A6760
:10C3E000234DDD6702258561224DC561C325AD035F
:10C3F000CD620A63D2435A601F4A1368FF25AB43DC
:10C4000026254D5DAD072D0EEB1813601B4A10233A
:10C4100013601B4A1360272260238B5419498160E3
:10C42000C160016121607D210901016641661649F3
:10C43000C164164941641649016400F085FC01B0ED
:10C44000F0BDC04604A000500000F8FF94A00050CA
:10C4500034A10050FF185A0030040040041000407E
:10C460001C2000405430004060400040B8A1005003
:10C4700014001400FF3F3FFF04E400E080E200E00E
:10C4800000E100E0DC05DC053F0270020133D0076B
:10C49000D007D0072921C64A50547047E4D1010281
:10C4A000F0B58BB0079208910146C14FB878099159
:10C4B000FFF7B4FE78793A7B79790691824200D809
:10C4C0009FE0FB7A9A181823534392004124E10419
:10C4D00004915218D2187B7B14214B43D21850245C
:10C4E0006043155801230A93DB022E469E431650E3
:10C4F0004E4B2B4005937D7B03914D433E7B744314
:10C50000F97A0B011B195B1971181C240294614301
:10C510005918A84B1B88069C5C430919C904490D8E
:10C52000059BC9181150101807994160387879791E
:10C53000089A00920322099BFFF77CFDF87A397B69
:10C5400009183878814263D983000993049AD45C2E
:10C550000894F7212140D154D1184D788E783602B5
:10C560007619CB781B04F31807900A9886051E43AA
:10C57000330CCB70FB7A387BBC784D709F4D3540C7
:10C58000039E6643C018029B4343981940029C4B8C
:10C5900003405C19200A8870200CC870F023089DA5
:10C5A0002B401B1D3D7B0895FE7A099D5355C87095
:10C5B0000620079A50438019089A801848701F2255
:10C5C000D20222400243100A88707879401C7871A8
:10C5D000387B7979814201D3002179713978491CFE
:10C5E0003970F97A08183978884201D800203870F3
:10C5F00028200A993954387A401C3872387A0BB09E
:10C60000F0BDA7204200D2480649074B02F0C6FB06
:10C61000A72042007A32CE487349744B02F0BEFB29
:10C62000E4D10102CC3B0100753B010000F0FFFFAB
:10C63000E0D101020320000605490A6882430A602E
:10C640000A6802430A600348012101607047C0463E
:10C650001C0000401CA0005080B50120FDF752FCDA
:10C6600080BD0000F0B587B006930646504C607A56
:10C67000504B1B88181A0C9DA84200DC89E00F461D
:10C680000592012E06D156480021C1620169554A22
:10C6900089180160A0783146FFF7C0FDE078E178A5
:10C6A000069A2B4600F0AEF82078E1780097002239
:10C6B00006923346FFF7BEFCE07A217B081821780A
:10C6C00088426ED94120C20404918800815C0391A4
:10C6D000F7250D40029285544549455C4549465C25
:10C6E000360276194449475C3F04F6190127BF0515
:10C6F00037433E0C4654E67A217BA3783C4A855466
:10C700003E4D3D4014275F4389191C234B43D919E3
:10C7100049023B4B0B405D19290A364BC1542E0C84
:10C7200035494654F02703990F400599002900D157
:10C730003F1D217BE37A029A87542F4A86540622B2
:10C74000049E7243D2185118294A81541F22D202E2
:10C7500015400D43290A274A8154E078401CE070B7
:10C76000E07AE178814201D30699E1702178491C91
:10C770002170217B08182178884201D80698207002
:10C78000E079401CE071A07A401CA072E07907B00B
:10C79000F0BD3920C2001632074808A109A302F0F3
:10C7A000FDFA3920C20004480F49104B02F0F6FA96
:10C7B000E4D10102E0D10102AC3B01006D61635F95
:10C7C000747800004D4143205458206C656E2069F8
:10C7D00073206F7665722072616E67650D0A0000C6
:10C7E0000804004090D00300E23B0100933B0100AD
:10C7F000010008020200080203000802FF07C0FF50
:10C8000000F83F00F0B589B00893019204914F4DB4
:10C81000EF7A874200D891E0297B502632464A437E
:10C820004124E3040693D218CC19A1005118182210
:10C83000059254430A19697B1423079359435318EB
:10C8400002900001195804460390504A0A40A97A00
:10C85000C902511808988205D2088A181A514C4901
:10C8600011402A7B00965643384CE57A2C010698F5
:10C870002418A719354E5419A5007D19059844436D
:10C880002819747B079D6C430519049FD2194148F0
:10C89000048854432A19089CD204520D51181D468D
:10C8A0000398195000F06AFA0146707A00190204E0
:10C8B0003E460CD080B2C000002900D1801E029FED
:10C8C000A5214900F3F706FC1F21014001E00021EA
:10C8D000029F38012818427983791B029A18C3797C
:10C8E0001B04D2182C4B1340437109045918090C2E
:10C8F000C171002C20D0154835460646007B009BB0
:10C900004343F17A0A01069F3A43D21841188B003B
:10C91000D218059B4B43D118727B079B5343C91810
:10C9200040191C4A1288424388180199884203D052
:10C9300001992246F3F71EFC09B0F0BDFF225C32DC
:10C94000034804A109A302F029FAC046E4D1010278
:10C95000AC3B01006D61635F74785F646573635F16
:10C96000636F6E73747275637400000054582044D2
:10C9700045534320696E646578206973206F76653E
:10C98000722072616E67650D0A000000FF0700E00B
:10C9900000F8FFFFE0D10102EFFFE00082B0FCF7FA
:10C9A00017FE052000252946FFF76AF806202946CC
:10C9B000FFF766F80A202946FFF762F809202946A2
:10C9C000FFF75EF80124204603F0C6FB284603F07B
:10C9D000C3FBFCF739FE2046FCF72CFE01F032FECB
:10C9E00001F02AFE6D4801686D480068890308D48B
:10C9F0000321090708402107884202D0FCF7B6FD51
:10CA000006E0FCF71BF9FCF7C9FD0020FDF7C0FCB0
:10CA1000FCF754FE0025284604F0DEFC032661A244
:10CA20003046314603F016FA30462946FBF724FC1F
:10CA3000F7F770FFFAF768FEFEF794FF5F4F381DB7
:10CA4000FCF7C0FBF7F75EFCF6F79AFBF7F7EFFE93
:10CA5000042630462946FFF713F8304621462A4679
:10CA6000FEF7A2FF052230462146FFF731F82046A7
:10CA70002146FEF7C1FF674E30462830504A0190EC
:10CA80002146FCF711FBFAF749F9A2024D494E4B3A
:10CA9000204603F05FFE01F0B3FBF6F75FFB4B4A65
:10CAA0002046214602F090F8494802F0BDF8494876
:10CAB000FCF746FDB87800280DD104E0FBF71EFA1C
:10CAC000B878002807D1F7F71DFF002803D1707A46
:10CAD000002815D13CE0FCF77DFC307A002802D01C
:10CAE0003572F6F7A9F9F7F721FFF6F733FFF7F7F5
:10CAF00063F9FAF717FEFCF74BFC707A002827D091
:10CB000075723079411C31713D2806D30020307197
:10CB1000012101982A4AFCF7C7FAFAF7ADFF2E481F
:10CB20000470F7F7EFFE002802D0BD70757107E0C2
:10CB300070791E28214600D32946B970401C7071B7
:10CB4000F7F776F97F20C105F069F3F704FCF0618F
:10CB50000B20FEF719FF3978002810D00029ADD13D
:10CB600001201E490870387000201D49087003F02C
:10CB7000CDFAFBF7C3F9B8780028ACD1A3E70129B7
:10CB80009CD1002038705049C88314490870012096
:10CB90001349087003F09AFA90E7C0461800004065
:10CBA000300001405557422073696D706C652065F7
:10CBB00078616D706C650D0A000000001C90010228
:10CBC0009D8F0000E0CD01028D09010071EB000096
:10CBD0007C3F00000DCC0000AE96010218900102CF
:10CBE00019900102014800687047C0460C000040DF
:10CBF00081B080B581B0039303AB009302F0A4FD34
:10CC000001B080BC02BC01B008470000014800210F
:10CC1000C161704780980102F0B581B000263046AE
:10CC20003146FDF71BFE0125AC022649264F304652
:10CC30003A462346FDF772FF3988244881423ED0A8
:10CC400064217E5262217E5260217E524422BE5275
:10CC5000FD87BD8778227A8702223A874322FA86A7
:10CC6000BE83FE811A4ABA817E810A223A81C82295
:10CC7000FA80184ABA803880FE8306203885F98405
:10CC8000FF20123078848730B88450203E523A8397
:10CC9000EFF3108072B630463146FDF7DFFD002815
:10CCA0000CD12A0300263046064D2946FDF730FDFB
:10CCB000054A304629462346FEF708FA62B601B017
:10CCC000F0BDC04600E0020432A90102AA550000EE
:10CCD000E1FF0000341200000020704710B500246E
:10CCE000002809D0002905D003464A000348194608
:10CCF000F3F740FA204610BDE04310BD3C9301021B
:10CD0000014600200A2901DAC0437047014A118018
:10CD10007047C046C49301020020704780B5018867
:10CD2000064A11808178064A1170C178054A11704F
:10CD30000079FCF773FB002080BDC0462E940102F1
:10CD40003094010294D20102044805490160152182
:10CD500009044160034981607047C0469C3000402F
:10CD60004100080034000700074800684069704728
:10CD7000FD20400004490968085C704702480068CB
:10CD80006221405C7047C0464494010210B50648D9
:10CD90000468064800686421F3F7B2F90221C94328
:10CDA0004143081910BDC04698D201029CD201022D
:10CDB0000A491A220A600A4948704878FF21090284
:10CDC000084A13688B43800380B2C018106006487D
:10CDD000202101600548016000207047702000405C
:10CDE0003494010204E400E080E200E000E100E0AD
:10CDF000F0B5A9B016460F460546C648002B0246B8
:10CE000000D01A463921CC003D21C900511811919A
:10CE10008242189206D001204202BE491898F3F7C8
:10CE2000A9F9189A6120111913910E21119C0A91E8
:10CE3000A170002F0D9501D00A2100E0092159238E
:10CE400017938300E1707842784113990870307825
:10CE500010901070F17AE17471785170B778977012
:10CE6000F178D1703579157174795471B179917106
:10CE7000F179D171317A1172717A5172B17A9172FC
:10CE80007E1EF0B200210328169106D870B28000F1
:10CE9000A1A210586A00805A16901798820018981C
:10CEA000C0181490F81E022804D3012E084604D896
:10CEB0009D4800E09D48031918781290189DA81805
:10CEC00017902846303015902C4656346D2080003F
:10CED0002950974A974B149E33627262B362F26292
:10CEE0003176F182139B597009229A70281841609B
:10CEF0008160C1600161109880008F490858F3F784
:10CF0000C7FD012F10900F9104D0022F05D17F2172
:10CF10007E2004E07C217B2001E05B215A20159DCE
:10CF2000A984207003200C90A080012666701F2029
:10CF30000B90A8821820A8740A46083A179BDA7644
:10CF4000169B129AD2184A439100189A9163B7021D
:10CF5000791E8B420E9109D978486080342068840C
:10CF60007748288277481399088339E07F2B10DDB2
:10CF7000802B18D031028B421BD071028B4227D1FB
:10CF80006E49618068846F4813990883CF20C00080
:10CF900025E0202B17D0402B1AD168486080042050
:10CFA000688469481BE0654860800620688467489B
:10CFB00015E06248608010206884624813990883F5
:10CFC000C520C0000BE0624860800220688404E055
:10CFD00004206884812040006080FF200230288285
:10CFE000104600F0D7FE1298102806D0402808D12D
:10CFF00008201499C876072000E00420179988704B
:10D0000002E017980C9981701898169A8078C11EC2
:10D0100002290CD3022811D001280CD12672BA4261
:10D0200000D900266672BA4213D8F44812E00D20E7
:10D030000002119908800120800201E00C98000292
:10D040002081BA4201D8EE4800E0FA2017998860A2
:10D050000EE0FA201799886013980078002811993B
:10D0600001D0E8484880E848139A1083E7480880D0
:10D07000A88CF3F76FFC0026E54B3246F3F7F2FA83
:10D0800002460B46E3493046F3F754FBE24B324687
:10D09000F3F7E8FAF3F7B0FC0746E080DF493046E3
:10D0A000109A0F9BF3F746FBDD4B3246F3F7DAFAA3
:10D0B000F3F7A2FC78434042800B608116990E98EA
:10D0C000814208D90C20149FB872D64817998883DA
:10D0D0001220189A0EE0480A189A149F01D00D20C9
:10D0E00003E0080A00D1DBE20A98B872CE4817992B
:10D0F00088831220F872D078052844D878440079C3
:10D10000400087440227402C3339C848B881C848BA
:10D110002FE0C046D4900102242201002422010005
:10D120003422010034220100141F01001B1F0100E2
:10D130003075000010270000D41F01000502000018
:10D14000FF060000040800000A0400003604000086
:10D1500003020000B748F881B748388013E0B748A9
:10D16000F881B7483882B74838600CE0B448B881D5
:10D17000B5481799C88306E0B4487882B448B880A7
:10D180000B9800069064AE483881A748F880B148F3
:10D1900002882A84B0480078E874B0480078119F6B
:10D1A0007875387D139000285ED0AD490A68102349
:10D1B000DA413A600A794B79CF8867801B029A1866
:10D1C0006A840A7A4B7A8F7AC87A0D7B65701B0263
:10D1D0009A183B04D21800061018179FF860487B75
:10D1E0008A7BCB7B3B77120210186081087C7877B2
:10D1F000487C149A9072887CD072C87C159B1874F5
:10D20000087D5874487D11909874C87D0A7E12027A
:10D2100012181A84887DD87418464B7EC375887E90
:10D22000CD7E2D022818B880087F4D7F2D0228184A
:10D23000F880887FB877C87FF8772020085C149D35
:10D2400028732120085C68732A20085C2A314D78F5
:10D250002D0228188D782D044019C9780906401828
:10D2600018998864119801E0EB7DA87C7D498B704A
:10D270000A8080001F38C882C883139800281FD0F6
:10D2800022227748825C034622335B781B029A187D
:10D290000A842422825C034624335B781B029A189A
:10D2A000CA842622825C034626335B781B029A18C6
:10D2B0008A832822825C2830407800028018888483
:10D2C0006948032569A2294602F0C4FD189F3878F1
:10D2D00014907B78B8780F90FA78B8791390F87931
:10D2E0001190387A1090787AB97A08900991009361
:10D2F0000F98019002921698039012980490139838
:10D3000005901198069010980790FAA2F8482946BF
:10D31000149B02F09FFD3D46643580212846F2F7BC
:10D3200042FFB878C11E02290ED3012800D18FE137
:10D33000022800D0ABE11691149078787F225043F8
:10D34000F7494018F74907E01691149078785B2266
:10D350005043F1494018F14941182846F2F70AFFB5
:10D360000D9D1898C6870E34324602E0641C0F2AC1
:10D370000ADA21780029F9D0491C8907C90F9140A0
:10D380000E43C687521CF1E71699022907D3149958
:10D39000491E012900D97DE14279D24901E0427953
:10D3A000CF4989180C78002D00D177E1C1790E9111
:10D3B000032900D94AE14279062A00D979E14921B5
:10D3C000890041181191E43010900E98401E12907F
:10D3D00019A800190F9000231392149403E01898D1
:10D3E000290600D15AE1052A5AD8C0467A44127952
:10D3F00052009744455C728598ABC0468813000084
:10D40000E20400000C080000060A0000040F0000FF
:10D410000000104130C1BD41000070400000F040EC
:10D420000000D041120C0000140B0000121200008A
:10D43000140E00000E160000130D0000121600005E
:10D440000E120000140B0E0A120800001016000045
:10D450000E0B00002E9401023094010294D20102BE
:10D46000A0D201029C94010201080000436173658F
:10D4700020706172616D65746572733A200D0A00E7
:10D480001693DFB2002F04D019A801223946F2F713
:10D4900083FE002C00D191E019A8C019BB498AE095
:10D4A000E8B2022867D00027022867D06BE00E9808
:10D4B000022872D1E8B2022800D103461693DFB2E7
:10D4C000002F04D019A801223946F2F765FE002C7E
:10D4D00074D019A8C019ACA16DE0E8B2022800D13F
:10D4E00004231693DFB2002F04D019A80122394675
:10D4F000F2F752FE002C61D019A8C0199FA15AE082
:10D50000E8B2022800D106231693DFB2002F04D020
:10D5100019A801223946F2F73FFE002C4ED019A877
:10D52000C01992A147E0E8B2022800D10C2316935B
:10D53000DFB2002F04D019A801223946F2F72CFEE1
:10D54000002C3BD019A8C019874934E0E8B2811EED
:10D550004A424A419700022804D119A801223946BB
:10D56000F2F71AFE002C16D019A8C0197CA1224689
:10D57000F2F700FE0FE00627022804D119A80122C5
:10D580003946F2F709FE002C05D019A8C0198049C8
:10D590002246F2F7EFFD169710E01693DFB2002F48
:10D5A00004D019A801223946F2F7F6FD002C05D067
:10D5B00019A8C01973492246F2F7DCFD3C193F2C2B
:10D5C00005D80F98C0194021091BF2F7ECFD1298FD
:10D5D0000228189801D2002002E0C078411E88413C
:10D5E00015990870611E2E46E8B202280CD1179AD0
:10D5F000517019A9119AB8C9B8C2B8C9B8C2B8C986
:10D60000B8C2B8C9B8C20DE0179A117019A9109A1A
:10D61000B8C9B8C2B8C9B8C2B8C9B8C2B8C9B8C21E
:10D62000C10709D180073546149C139A169B00D474
:10D63000D5E602208543D2E6FE20354605401898FF
:10D64000149C139A169B290628D0CCE637A231E009
:10D650001691149078780B994143334808181F3875
:10D660006F21C9430D9D7A180378D427D355437889
:10D67000D827D3558378DC27D355002900D170E60D
:10D68000C378E027D3551031001D189FEBE7012028
:10D69000404A10E00024002D00D087E629B0F0BDFC
:10D6A00080290ED30F20B872104817998883102054
:10D6B00020E525A20120014602F0CCFB189829B0F4
:10D6C000F0BD1020402904D3B8720849179B9983F4
:10D6D00010E5B87204481799888314200AE5C046FB
:10D6E0001B1F0100141F0100150F0000140B000088
:10D6F000010800002564202564202564202564207D
:10D7000025642025642025642025642025642025A7
:10D71000642025640D0A0000684501001DF7FFFF25
:10D72000803C010089FBFFFF704401007472785F48
:10D730006D6F646520706172616D657465722065DE
:10D7400072726F720D0A00004E736664207061720F
:10D75000616D65746572206572726F720D0A0000EA
:10D76000FFFFFFFF01FF0000D4220100FFFFFFFFCA
:10D77000FF0101FFFF01FF01FFFF01FFFFFFFF01AD
:10D78000FFFF01FFC0280100FFFF01FFF42201009D
:10D79000442201001E3C0100002800D10148064936
:10D7A00008607047D4900102F0B586B0002805D11A
:10D7B0000148006802E0C046449401023121C900DA
:10D7C000049141188A791F231A40CD79ED06AD0DD9
:10D7D000AA180D7AED066D0C52194D7AED062D0B37
:10D7E00052198D7AED06ED095219CD7AED06AD0884
:10D7F00052194D7CED075219BD4C22600A7B1A402C
:10D800004E7BF606B60DB2188E7BF606760C921994
:10D81000CE7BF606360B92190E79F606F6099219AA
:10D820004E79F606B608921962604A6AB14D2A40EE
:10D83000A2608A6A2A40E2602D22D20087183A7ECE
:10D840001A4003937E7EF606B60DB218BE7EF6062B
:10D85000760C9219FE7EF606360B92193E7FF6067E
:10D86000F60992197E7FF606B60892190E7CF60725
:10D8700092192261BA7F1A400597FE7FF606B60D0F
:10D88000B218049BC35CDB065B0CD2184B78DB063A
:10D890001B0BD2188B78DB06DB09D218CB78DB06A2
:10D8A0009B08D2186261CA692A40A2610A6A2A40AA
:10D8B000E2618A7C01252A40CB7CDB079B0F9A180A
:10D8C0000B7DDB075B0FD2184B7D9B07DB0ED2185D
:10D8D0008B7DDB079B0ED218CB7D1B079B0D9A1807
:10D8E0000B7E1B079B0CD2184B7E5B06DB0A134397
:10D8F0008A7E520612091A43CB7E5B075B081343EC
:10D900002362CA6A62620A6BA2624A6BE2628A6B33
:10D9100022633922D200835C1E462E4066635E423B
:10D920005E41B304AE04744F3C68B443E3183B60FB
:10D9300083185A782A409C782407E40EA2188C8F0A
:10D940006401A2186D4C1440C98FC905490A091910
:10D95000DA78D207120A89181A7912071209891877
:10D960005A79D207D2088918FB4EB1639968F163DE
:10D97000997904952940DA79D207920F51181A7BC8
:10D980005207D20E89185A7BD206920D51189A7BF3
:10D990005207D20C8918DA7BD206920B89181A7CAE
:10D9A000D206520A89185A7C520792090A43997C76
:10D9B000C906490851183164D97C039A11401A7D6F
:10D9C000D206920D51185A7DD206520C89189A7DB2
:10D9D000D206120B8918DA7DD206D2098918716431
:10D9E000197E0F2421405A7E120151189A7E12038B
:10D9F0008918DA7E1207120A51181A7F12071209C3
:10DA000089185A7F12078918B164997F01942140BF
:10DA1000DA7F1207120E51183D22D200835C5B0799
:10DA20005B0D5918841862781207520C8918A27875
:10DA3000D206120B8918E278D206D2098918F1644D
:10DA4000217907220A406179C9008918A279520612
:10DA5000920B5118E2799207120B8918227AD20799
:10DA60008A18BF490A60627AA37A1B029A18E37A7D
:10DA70001B04D2184A60E289BA4B13400394228AED
:10DA8000D2049209D2188A6003463033598CB64AC0
:10DA9000114002939A8CD205D20A51185622825C08
:10DAA00012068918B14D2960014656314A788C78A2
:10DAB0002402A2188C8864056409A218CC78240773
:10DAC00012196A60CA880C7AA407A40BA2184C7AAF
:10DAD0006407E40A1219AA604989E96049218900AA
:10DAE0004118FF226632821800921035002207E0AA
:10DAF00000300040FFFFFF0004040040FF3F000033
:10DB000084186427E65D03273E406523E35C9B079A
:10DB10001B0F9B196626A65DB607B60EF31867267F
:10DB2000A65DB601F318DBB26826A65DB607B60D92
:10DB3000F3186926A65DB607360DF3186A26A65DAA
:10DB4000B607B60CF3186B26A65DB607360CF318AD
:10DB50006C26A65DB607B60BF3186D26A65DB60754
:10DB6000360BF3186E26A65DB607B60AF3186F26B5
:10DB7000A65DB607360AF3187026A65DB607B60985
:10DB8000F3187126A65DB6073609F3187226A65D4E
:10DB9000B607B608F3187326A45DA407E31808C5F2
:10DBA0001032802AACD1019AD243704EB4180B784F
:10DBB0003B404D78AD072D0FEB188D78AD07AD0EBE
:10DBC000EB18CD78AD01EB18DBB20D79AD07AD0DDB
:10DBD000EB184D79AD072D0DEB188D79AD07AD0C18
:10DBE000EB18CD79AD072D0CEB180D7AAD07AD0B09
:10DBF000EB184D7AAD072D0BEB188D7AAD07AD0AFA
:10DC0000EB18CD7AAD072D0AEB180D7BAD07AD09EA
:10DC1000EB184D7BAD072D09EB188D7BAD07AD08DB
:10DC2000EB18CD7BAD07EB18A3641031121DBDD1ED
:10DC3000009B19785A785207520D51189A78D207DA
:10DC4000120D8918B164059B1968F164D97D5A6871
:10DC50001202511831659968454A0A40998A490566
:10DC600089187165D9683D4C2140B1651969214019
:10DC7000F165029E3178049D294082785207120F87
:10DC80005118C2799207920E8918427A9207920D22
:10DC90005118827A9207120D8918C27AD207920C13
:10DCA00089189A7DD207520C891872789207D20B84
:10DCB0008918B2781207D20A8918F2781207D209A5
:10DCC0008A182C490A60327C737C1B071B0D9A183A
:10DCD000B37C9B069B0BD218F37C1B079B0AD218C4
:10DCE000337DDB065B09D218737DDB071B09D21875
:10DCF0004A60B27D2A40C38F5B009A188A60826CAA
:10DD0000CA60C26C22400A61F27D7F231340328CCC
:10DD10005204520AD2184A6102698A614269CA6190
:10DD200082690A62C2694A62026A8A62426ACA6295
:10DD3000826A0A63C26A4A63039A927CD201121D04
:10DD40000A64027A3A40CA65808F074A1040086622
:10DD5000002006B0F0BDC04600300040FFFFFF00CD
:10DD60009C300040FF1F0000FF0300000040004007
:10DD7000FFFF1F000020004004480068806B8008FF
:10DD8000034909684900401809307047449401026A
:10DD90001004004010B52D21C9004118027A032A51
:10DDA00004D10079002807D0082006E08378DA1E25
:10DDB000022A05D2032412E0142088601C203DE0D2
:10DDC000012B02D1C8228A6012E00479042C01D30D
:10DDD000462404E0032C01D1322400E014248C609A
:10DDE0005B1E022B04D3022A10D24279154B01E0AC
:10DDF0004279154B9B181B78402B04D0102B06D171
:10DE00001423442405E02A233E2402E042793423EB
:10DE100048244B800C80022A06D0062A08D0052A06
:10DE200008D118224C2301E0142250230B8000E07B
:10DE30001C224A80C078042803D114204880642022
:10DE4000088010BD1B1F0100141F0100134800684B
:10DE50007047C04610B5104A107091700F490028E5
:10DE600013D050680861042048619078FF221202A4
:10DE70000B4B1C689443800380B20019186001208A
:10DE80004007084A1060084A1060002008600749EF
:10DE900001220A6010BDC0463494010218040040FB
:10DEA0001CE400E080E200E000E100E070000040DF
:10DEB000F0B591B0002801D1C04800688778F91EFC
:10DEC000022913D3012F21D0022F3CD11021CA43A4
:10DED00044782146193991423DD800970125B94A25
:10DEE00028462946234601F0B5FF53E10821CA43DD
:10DEF000447821462139914218D800970125B14A2A
:10DF000028462946234601F0A5FF43E10821CA43DC
:10DF1000447821460939914234D800970125A94A0D
:10DF200028462946234601F095FF33E1032F3CD0D4
:10DF3000042F43D1C3780125042B00D02DE10646E0
:10DF40002A02042343E00125A6A2284629463B468F
:10DF500001F080FF1EE1C3780125052B0AD8064693
:10DF60002A02284698401B21084230D10021052B67
:10DF700008462ED002200090914A2846294601F0FA
:10DF800069FF07E10646C3780021022B1ED3032B4D
:10DF90001CD0042B08460A461BD001250095884A50
:10DFA0002846294601F056FFF4E0C3780125032BEB
:10DFB00000D0FAE006462A02032308E0012583A2E6
:10DFC000284629463B4601F045FFE3E00A46012189
:10DFD00048020F91592189007518FD2149007118D7
:10DFE0000291314662313F05D219641E1F27274036
:10DFF0005C013C191443044332795207D20C22438A
:10E000002B789B065B0BD218B379DB071B0B1343F2
:10E010006D4D2B60F279032310931A40737A9B079E
:10E020009B0E9A18B37A5B07DB0D9A18F37ADB071D
:10E030009B0DD218337BDB075B0DD218737B1B075C
:10E040005B0CD218AA603269EA6072692A61B2690F
:10E050006A61F269AA61326AEA61726A2A62B26A24
:10E060006A620F980870F06AA8623F20C4432C359A
:10E070003046E4300F903046E5300E903046E630C2
:10E080000D903046E7300C903046E8300B9030462B
:10E09000E9300A903046EA3009903046EB3008907B
:10E0A0003046EC3007903046ED3006903046EE308A
:10E0B00005903046EF3004903046F03003903746FC
:10E0C000F1373046F230F3360F990A194021525C8D
:10E0D000109B1A400E9B1B195B5C9B071B0F9A1829
:10E0E0000D9B1B195B5C9B079B0E9A180C9B1B19C5
:10E0F0005B5C9B019A18D2B20B9B1B195B5C9B0764
:10E100009B0D9A180A9B1B195B5C9B071B0D9A18A9
:10E11000099B1B195B5C9B079B0C9A18089B1B199E
:10E120005B5C9B071B0C9A18079B1B195B5C9B078E
:10E130009B0B9A18069B1B195B5C9B071B0B9A1881
:10E14000059B1B195B5C9B079B0A9A18049B1B1978
:10E150005B5C9B071B0A9A18039B1B195B5C9B0764
:10E160009B099A183B195B5C9B071B099A180319BA
:10E170005B5C9B079B089A183319595C89078918BF
:10E1800002C51034A0D102980078042101430E4842
:10E19000C1630025284611B0F0BD04200090084A54
:10E1A0002846294601F056FEF4E703200090044A71
:10E1B0002846294601F04EFEECE7C0464494010291
:10E1C000F33B0100393C010000100040556E6465CE
:10E1D00066696E6564206D65616E2050524620252B
:10E1E000640D0A00496E76616C6964206D65616E2C
:10E1F000205052462025640D0A00000070477047E9
:10E2000080B50E490E480246083A1268920000D4C2
:10E21000603142680A4342600A490A6808239A4307
:10E220000A60091F012252040A600321890402685E
:10E230008A430260FBF732FA80BDC04620000080AE
:10E240002800004004020040B0B5032000072D491B
:10E250000A688243012568071018086000242046D8
:10E26000FFF7CDFF2046FFF7C9FFEFF310802840EE
:10E2700002D1EFF3108172B68021C943224A53685C
:10E280000B40536093680B409360D3680B40D3609E
:10E2900013690B40136153690B405361002800D18F
:10E2A00062B6B0BD70B50C4603210907154A136864
:10E2B0000B4313600122EFF31081114002D1EFF301
:10E2C000108272B68025EA430F4B5E6816405E608E
:10E2D0009E682E439E60DD681540DD601D69154017
:10E2E0001D615D6915405D61002900D162B600289D
:10E2F00002D00120FFF783FF002C02D00120FFF79E
:10E300007DFF70BD00040040D89501020D4A002930
:10E3100007D001290BD1012181401068884310608A
:10E3200007E00121814010680843106001E00121ED
:10E330008140101F02680A430121C907114301608F
:10E340007047C04644000040032804D840000649F6
:10E35000085A00B27047002000B27047032802D864
:10E360004000014A11527047CED201029E49087006
:10E370007047C04670B58AB00C460546FF20FC3099
:10E38000A8490E68315C59208000335CB27830783F
:10E3900008AE069609AE05960C4E04962126760622
:10E3A00003960B4E0296012601960E2600965B1CE4
:10E3B000DBB2F7F739FC0998F2F7F0FA2870089801
:10E3C000F2F7ECFA20700AB070BDC04600002041A0
:10E3D00000000443F0B58BB00446457C82480078C9
:10E3E0008249002822D000200880814A1080814B79
:10E3F00001269E761E830A907F4800787F4E3678ED
:10E400006DB205957E4D04957E4D03950AAD02953E
:10E410007D4D01950096F7F745F90A9D112020568C
:10E420007A497B4A00F022FC064626E000260E8050
:10E430006F4A16806F4B01209876188309966E48B4
:10E4400000786E4F3F786DB205956D4D04956D4D1A
:10E45000039509AD02956C4D01950097F7F722F9E8
:10E46000099D112021567F20C00500900190029641
:10E47000664A674B3046F8F769FA4320010628469A
:10E48000F1F7C2FFF2F78AFA089062480078002894
:10E4900024D05120800060494A7D42438D185F4856
:10E4A0000068A8642F46403750480078B874504838
:10E4B0000078F874554800783875554800787875B4
:10E4C00057480078F87550480069F2F767FAB87550
:10E4D00052484069E8644C4800686864FF20FE3098
:10E4E00050490968085C3922D2008918022812D3E1
:10E4F00003D04E48007801280DD14B4806604348B0
:10E5000000883A4A108042480088394A1080092021
:10E510000790089605E04448089A02603548C08B89
:10E5200007900B780022002B01D0114600E0D14368
:10E530000125002B01D0042300E0EB43A67AAD1B9C
:10E54000EE175B1971416568AE0F277AAD00ED19C2
:10E550005641677A3F1FF817ED1970414000EE0FE2
:10E5600080196D00EB1848418001990E41189801FF
:10E5700027239B02C31A91411D4805881B48008828
:10E58000854201D00798421B10202056C001194D2A
:10E590002D8C032D07D1E468E5176D0A6419E41585
:10E5A0000519EC170FE0E468E5176D0A6519EC171B
:10E5B000ED15C6174519744197B2002F00D03446A7
:10E5C000002F00D00546581BA141130409D012B2F8
:10E5D000D2015242D31780185941089BDA17C01A4A
:10E5E00091410BB0F0BDC046C69301023CAD0102A3
:10E5F0003AAD01029C940102B5900102B49001026F
:10E6000028A3010224A1010240AD01028AAD01024A
:10E6100088AD0102F4A601022CA40102642000408E
:10E6200038AD01024494010234AD010298AD0102FB
:10E63000C10D4002803070470120C0071B490860AF
:10E640007047C04610B519480068C10710D181074E
:10E6500011D4410712D4010713D4C10614D4810682
:10E6600015D4410616D48021084016D031A215E0F9
:10E6700001240FA213E0022411A210E0032414A22B
:10E680000DE0042416A20AE0052419A207E00624DE
:10E690001CA204E0072421A201E0254A040902206B
:10E6A000032101F0D7FB204610BDC0465C000040AE
:10E6B000526573657420627920504F520D0A000034
:10E6C000526573657420627920424F520D0A000032
:10E6D00052657365742062792050494E0D0A00001E
:10E6E0005265736574206279205744540D0A000006
:10E6F0005265736574206279204C4F434B55500D21
:10E700000A00000052657365742062792053572017
:10E710005265626F6F740D0A0000000052657365E8
:10E7200074206279205359535245510D0A0000005C
:10E730009E2E010052657365742062792044564410
:10E74000440D0A0001218140044A1F2802D01068AC
:10E750008843106010680843106070471C00004038
:10E76000F0B583B0029104469949F1F7B3FC054630
:10E77000984901942046F1F7ADFC9749461897490E
:10E78000714300956F189649441864212046F1F7AB
:10E79000A1FC3818A108471A92492046F1F7B0FCAD
:10E7A000381891494518914F05D464213046F1F746
:10E7B00091FC0C4614E0A6B264213046F1F78AFCC5
:10E7C000B7204000A20701D1002907D1884B73432D
:10E7D0000422D341874A934200D3401E0C46451978
:10E7E0000098474302980680192001013046F1F74E
:10E7F00071FC2A461F3A284600DB1046019BFF1891
:10E80000B30705D1002C03D01F2D05DA0120C5E088
:10E810001F2D0BDA0120C1E005461D3D034600DB3C
:10E820002B461C2808DC02201546B7E000290CD036
:10E830001C21451A0CD50CE019461F39184600DB7F
:10E8400008461F2B1DDA0320A8E01D21451A00D41D
:10E850002846002D08D401461F39024600DB0A462F
:10E860001F2804DA032099E00220154696E0154699
:10E870001E3D104600DB28461E2A0CDA04200D46F9
:10E880008CE005461E3D024600DB2A461E280BDAB8
:10E8900004200D4682E001461F39024600DB0A468D
:10E8A0001F280ADA052079E011461F39104600DBDF
:10E8B00008461F2A0BDA052070E015461E3D10465B
:10E8C00000DB28461E2A0CDA06200D4666E00546C7
:10E8D0001E3D024600DB2A461E280BDA06200D46A6
:10E8E0005CE001461F39024600DB0A461F280ADAAF
:10E8F000072053E011461F39104600DB08461F2A47
:10E900000BDA07204AE015461F3D134600DB2B4675
:10E910001F2A0CDA08200D4640E005461F3D02463E
:10E9200000DB2A461F280BDA08200D4636E0194680
:10E930001E39184600DB08461E2B0ADA09202DE096
:10E9400011461E39104600DB08461E2A0BDA092044
:10E9500024E01F28054601DB05461F3D1F280CDA71
:10E960000A200D461AE01F28054601DB05461F3D1B
:10E970001F2806DA0A200D4610E01E2D05DB0C20AC
:10E9800004E01E2D06DB0C2005E00B201E2D05DB10
:10E990001E3D03E00B201E2D00DB1E3D029EB070CD
:10E9A000681CF070E12001013846F1F793FB3071EB
:10E9B000C0B211494143CC193C212046F1F78AFBF2
:10E9C00070713B21C94341430819B07103B0F0BDD8
:10E9D000805101008033E101B207000093FEFFFF88
:10E9E000B107000070FEFFFFA7FA0A0080AEFEFF2D
:10E9F000295C8FC20BD7A300F0F1FFFFF0B581B007
:10EA00000446FFF721FCA08A00280ED0FFF71EFA6B
:10EA10002049086120482CCC2CC02CCC2CC02CCCFC
:10EA20002CC00020888101B0F0BDE08A194FB88168
:10EA3000A169BA891948F1F79DFB174D204629466F
:10EA40004CC84CC14CC84CC14CC84CC1FFF7FEF976
:10EA500038616E68FFF790F9301AB8622846FFF700
:10EA6000B9FC06460D460E48007BFFF76DFC012100
:10EA7000F970617C7971396C491C396481B2C90BB8
:10EA8000401800B2C1174010301A38658D417D65BD
:10EA900001B0F0BD309901020C9A0102D8D20102F6
:10EAA000B690010270B50446FFF7CEFBA08A1B4E5C
:10EAB0007082718A002908D0B08202207071002013
:10EAC0003082FFF7C3F9F06170BDE08A3082A1693E
:10EAD000328A1348F1F74EFB2046FFF77BFC0546D0
:10EAE0000C461048007BFFF72FFC81B2C90B401881
:10EAF00000B2C1174010281A30668C417466FFF7C7
:10EB0000A5F9B061F06C401CF064FEF73FF9F063CA
:10EB1000FAF78AFC30640120707170BDB096010272
:10EB200070D30102C4900102F0B581B0EFF3108000
:10EB300072B600200146FBF791FE0446002803D080
:10EB400062B6204601B0F0BD01273A030025074E0A
:10EB500028463146FBF7DCFDBB021A4A28463146FF
:10EB6000FCF7B4FA62B6204601B0F0BD00E0020442
:10EB700010B5F5F75CFE114CE078002801D0F9F7EC
:10EB8000F1F9F9F765FAF7F7A1FF0D49012048738C
:10EB90008A7B034693434B72521C8A73094A928FB5
:10EBA000002A08D00A7B8B78134304D0CA7A501C01
:10EBB000C87201209043607010BDC0461C900102D5
:10EBC0008098010232A9010270B514460D4606462E
:10EBD0001120FAF7E1FE2248042101600C4804608C
:10EBE0001E4805608660002E0DD0FF2000060949F2
:10EBF0000A6882430120C0071018086006480821EF
:10EC00000160064801601A200221FFF77FFB70BDFA
:10EC100070D4010200E400E080E200E000E100E0E6
:10EC20000C4908607047C04610B5044609480068A2
:10EC300060430949F1F764FA001908494860084837
:10EC40000022026002460C3A4B68136009680160BA
:10EC500010BDC0466CD4010240420F000C9001026E
:10EC60002C10014000480047C100000080B582B070
:10EC700013460A4600900348011D0348F7F712FEA9
:10EC800002B080BDACD401025CA0010210B50C49F9
:10EC90008A1C90420DD2401E0D4A50600D480368F8
:10ECA0000B4003218C071B1903600020906011604A
:10ECB00010BD04480449E622044B00F06FF8C0463A
:10ECC000FFFFFF00752E01008F2E01005B2E01005B
:10ECD00010E000E020ED00E0B0B50120EFF310817E
:10ECE000014002D1EFF3108272B6124A1368124C3F
:10ECF000226864688506114800682840850E5D1901
:10ED00002923DB006B43002C1D4606D1002809D1C6
:10ED10001E20684300290AD0B0BD121BD218551C12
:10ED20000028F5D01D461E2068430029F4D162B6A4
:10ED3000B0BDC046DCDF010214E000E004ED00E0FD
:10ED400080B50020FBF734F8404280BDB0B586B0F6
:10ED5000104869460A4638C838C238C838C2002444
:10ED60002046FBF72BF803992046FBF7C1F80198E2
:10ED7000012803D00824002804D102E0042400283C
:10ED800000D104460220FAF70FFEE0400249086075
:10ED900006B0B0BD201F0100F0DF010290B01C469C
:10EDA00005AB07C3EFF31080C00702D1EFF310806B
:10EDB00072B6EFF310800B9068460E907046089084
:10EDC00010AB0F93CF4F3E1D01200490C50230467B
:10EDD0002946224600F0B8FC00213154EFF30380AD
:10EDE0000990EFF308800C90EFF309800D90EFF39A
:10EDF00014800A9000F02CFC3868012833D80028D1
:10EE0000C14F00D0C14F2A20C1497A69920703D56A
:10EE10000A783A60401E491C0028F6D1B948041D02
:10EE20002046F1F7D5F9002807D079698907FAD586
:10EE300021783960401E641CF5E70220B5497A69E3
:10EE4000920703D50A783A60401E491C0028F6D183
:10EE50002A20AF497A69920703D50A783A60401EA2
:10EE6000491C0028F6D1FFF737FF0346AA4A30466F
:10EE70002946FDF7BDFE04463018291B089F3B1F9D
:10EE8000049A9343A5A2FDF7B3FE9E4909680129A0
:10EE900066D8001900299C4C00D09C4C00280AD050
:10EEA0009849091D6269920703D50A782260401EBD
:10EEB000491C0028F6D10A209F496269920703D5B0
:10EEC0000A782260401E491C0028F6D10598F1F707
:10EED0007FF9002809D061698907FAD5059A117868
:10EEE0002160401E521C0592F3E7022089496269A5
:10EEF000920703D50A782260401E491C0028F6D1EB
:10EF00000A208EA16269920703D50A782260401E0A
:10EF1000491C0028F6D10698F1F75AF9002809D0C3
:10EF200061698907FAD5069A11782160401E521C42
:10EF30000692F3E7022077496269920703D50A78BF
:10EF40002260401E491C0028F6D10A207EA1626979
:10EF5000920703D50A782260401E491C0028F6D18A
:10EF60007CA230462946079BFDF742FE65490968A9
:10EF700001290E9B1BD80029634900D06349002852
:10EF80000AD0604A121D4C69A40703D514780C609E
:10EF9000401E521C0028F6D102205E4A4C69A4078C
:10EFA00003D514780C60401E521C0028F6D16AA2CA
:10EFB00030462946FDF71CFE04463018291B694AD5
:10EFC0003B46FDF715FE4F490968012911D8001984
:10EFD00000294D4900D04D4900280AD0494A121D48
:10EFE0004B699B0703D513780B60401E521C002809
:10EFF000F6D15D4A30462946099F3B46FDF7F8FDAC
:10F000000446F800C00FB900C90F7A00D20F009271
:10F01000019102903019291BFB0F544AFDF7E8FDBE
:10F0200004193019291B3F233B40514AFDF7E0FDED
:10F0300034490968012911D820180029324900D023
:10F04000324900280AD02F4A121D4B699B0703D56D
:10F0500013780B60401E521C0028F6D1454A3046FA
:10F0600029460B9BFDF7C4FD04463018291B424A74
:10F070000A9BFDF7BDFD23490968012911D8001934
:10F080000029214900D0214900280AD01D4A121D1B
:10F090004B699B0703D513780B60401E521C002858
:10F0A000F6D1364A304629460C9BFDF7A1FD0446B1
:10F0B0003018291B324A0D9BFDF79AFD114909684A
:10F0C0000129114A0DD80019002908D00F4A06E07D
:10F0D0005169890703D531781160401E761C0028DC
:10F0E000F6D128490E98091AA94200D32946890861
:10F0F00000F03AFE24480068002800D0804700F065
:10F1000045F8C046C0E001020090014000A0014067
:10F11000CF2E01005D3C0100B82E01000D0A232313
:10F120002320415353455254204020307825303815
:10F1300058202323230D0A00922F010046554E43E9
:10F1400054494F4E3A2000004C494E452020202083
:10F150003A200000256400000D0A53503D25303848
:10F16000580D0A00572F01006D2F0100792F010063
:10F17000612F0100162F0100252F0100342F0100FF
:10F180003F2F010000F80202BCE00102F7480068CE
:10F19000012811D8002801D00B4800E0FC480C21C0
:10F1A0000A4A01E0002907D043699B07FAD5137882
:10F1B0000360491E521CF5E71E20FFF7C3FA00BF8B
:10F1C00000BF00BF00BFFAE700A00140C22E01004F
:10F1D0008AB00646E448B06600F03AFAFFF77CFDD4
:10F1E0000346E248041D01200590C502E04A20467E
:10F1F0002946FDF7FDFC074608942018DB4C0995CD
:10F20000E91BF36C3F2206921340DAA2FDF7F0FCF3
:10F210002168012910D8C0190029DD4900D0DD4935
:10F22000002809D0221D4B699B0703D513780B607A
:10F23000401E521C0028F6D1F36BD7A2089C204632
:10F24000099D2946FDF7D4FC0746291A2018336C7E
:10F25000069A134007D1D8A2FDF7CAFCC34C216817
:10F26000012907D917E0CEA2FDF7C2FCBF4C2168E7
:10F27000012910D8C0190029C54900D0C549002866
:10F2800009D0221D4B699B0703D513780B60401EE4
:10F29000521C0028F6D10027CBA5B80030580090AA
:10F2A000089809992A463B46FDF7A2FC21680129E6
:10F2B0000FD80029B64900D0B649002809D0221D30
:10F2C0004B699B0703D513780B60401E521C002826
:10F2D000F6D17F1C0D2FE0D1736BBFA2089C204696
:10F2E000099D2946FDF784FC074620189F4CE91B21
:10F2F000B36BBC4AFDF77CFC2168012910D8C0190A
:10F300000029A34900D0A349002809D0221D4B6938
:10F310009B0703D513780B60401E521C0028F6D1C2
:10F32000336CB14A089C2046099D2946FDF760FCD4
:10F330000746326CD000C00F9100C90F5300DB0F9D
:10F34000009301910290E019E91BD30FA74AFDF742
:10F350004FFC3246C619A019A91B1546136C069A14
:10F360001340A34AFDF744FC80490968012911D8DC
:10F3700080190029864900D0864900280AD07B4A96
:10F38000121D4B699B0703D513780B60401E521C5E
:10F390000028F6D12E466B6C964A089C2046099DA3
:10F3A0002946FDF725FC07462018E91B0796B36C94
:10F3B000914AFDF71DFC6D4A1168012910D8C0194A
:10F3C0000029734900D07349002809D0121D4B69E8
:10F3D0009B0703D513780B60401E521C0028F6D102
:10F3E0000798426E042360215C2004931A400B4668
:10F3F00000D003460693002A00D00846079E3358E3
:10F400007E4A089C2046099D2946FDF7F1FB0746E8
:10F4100006983358E019E91B794AFDF7E9FBC6194C
:10F42000A019A91B079A536E76A2FDF7E1FB4F497D
:10F430000968022911D280190029554900D055497F
:10F4400000280AD0494A121D4B699B0703D513783F
:10F450000B60401E521C0028F6D10798C36C06466C
:10F460006DA2089C2046099D2946FDF7C1FB074671
:10F470002018E91B336D6B4AFDF7BAFBC619A019BA
:10F48000A91B079F7B6D68A2FDF7B2FB8619A01927
:10F49000A91BBB6D67A2FDF7ABFB344909680129C5
:10F4A000059C11D880190029394900D03949002814
:10F4B0000AD02E4A121D4B699B0703D513780B60A7
:10F4C000401E521C0028F6D10798476B5D4A9742B0
:10F4D00037D2032087430026059CB00039580246E6
:10F4E000049B1A43BA5808230343FB580C250543D1
:10F4F0007D5900910192029303953B180898099950
:10F50000514AFDF775FB1949096801290FD80029EF
:10F510001F4900D01F49002809D0089A4B699B0752
:10F5200003D513780B60401E521C0028F6D11B2E09
:10F53000444A06D80798406B361DB10040189042E7
:10F54000CBD30798406B111A099A914201D88908C8
:10F5500000E0610200F008FC3C480068002800D090
:10F560008047FFF713FEC04622224B4DC0E0010248
:10F57000B82E01000D0A0D0A2323232045584345C8
:10F580005054494F4E202564202323230D0A0000A8
:10F590000090014000A0014050433D253038580004
:10F5A0002C20457863657074696F6E4E756D626569
:10F5B000723D25640D0A00002C2054687265616458
:10F5C0004D6F64650D0A000052252D32643D2530D3
:10F5D00038580D0A0000000053503D253038580DB2
:10F5E0000A000000572F01006D2F0100792F010044
:10F5F000612F0100162F0100252F0100342F01007B
:10F600003F2F01004558435F52455455524E3D250A
:10F610003038580D0A000000494353523D25303818
:10F62000580D0A004A2F01005343523D25303858E7
:10F630000D0A00004343523D253038580D0A0D0A8B
:10F640000000000000F80202FA2E0100BCE00102F6
:10F65000F0B583B0344D2C68012C06D8601E84416F
:10F66000204601F073FB0028FAD10120EFF310814E
:10F670000140019102D1EFF3108072B62B48285A55
:10F680002B49695A814245D02A68002A01D02A4E66
:10F6900000E0284E1F23DB020293284C022A27D2C7
:10F6A00005E01046214AA85282B2914232D087B278
:10F6B000B9420A4600D8621C131A21482B5218047A
:10F6C0000DD0E819001D9FB201E0002F07D073692B
:10F6D0009B07FAD5037833607F1E401CF5E7A242F2
:10F6E000DFD902981018DDE7304683B299420CD07A
:10F6F000024680B281420E4600D8661CA642F3D96B
:10F700000298301883B29942F2D108496852B01A6F
:10F710000B4968520B48002129540198002800D158
:10F7200062B603B0F0BDC046C0E001020A080000A6
:10F73000080800000090014000A00140FF07000001
:10F740000C0800000F080000F0B58DB007931746B5
:10F7500000240C9409AA13C215E006986849F0F732
:10F7600053FEF1F71BF9C117401848406549F0F7FF
:10F77000B1FC009509A806223346F9F7C9FABDE0A5
:10F78000002C00D5BEE138787F1C25280DD000283C
:10F7900000D1B7E10B9A511C0A9B9942F0D8099B02
:10F7A0009854641C0C940B91EAE70894002539786E
:10F7B00023390D2914D801207944097949008F444F
:10F7C000090F0F0F0F0F0F0F0B0F060F0F0D054334
:10F7D0007F1CECE70820FAE70420F8E70220F6E7B0
:10F7E0003878014630390024092902D9264639469D
:10F7F0000BE000260A2171430E18303E791C787800
:10F800000246303A0A2A0F46F4D32E2817D14A1C52
:10F81000487801463039092905D911464F1C253849
:10F82000532811D96AE000240A2161430C18303CA6
:10F83000511C50780246303A0A2A0A46F4D34F1C2B
:10F840002538532800D959E04000C04678448088C4
:10F8500040008744A000530053005300530053005E
:10F860005300530053005300530053005300530000
:10F8700053005300530053005300530053005300F0
:10F8800053005300530053005300530053005300E0
:10F8900053005300530060005300530053005300C3
:10F8A00053005300530053005300530053005300C0
:10F8B000530053005300530053009800530053006B
:10F8C00053005300530053005300530053005300A0
:10F8D000AD00B600530060005300590053005300C0
:10F8E00053005900530053005300DE0053005300EF
:10F8F000BD005300D3005300530098000C9C3FE719
:10F900000024744940420F00791C38780F4625388E
:10F910005328F3D898E70799C91D07208143086841
:10F9200007914968F1F7C8F800210690F0F796FFB3
:10F9300000280BD10B99481C0A9A904206D8099AC4
:10F940002D2353540899491C0C910B9007980830AB
:10F9500007900698F1F722F80095C21781185140D8
:10F9600009A822463346F9F7D3F90B98411C0A9AA5
:10F97000914200D9F1E6099A2E2313540B910C9869
:10F98000401C0C90E9E6079802C807900096019584
:10F9900009A8102239E00B98411C0A9A9142ADD86F
:10F9A000099A252313540B910C98401C0C90A5E741
:10F9B0000B9A511C079C201D0A9B994239D907902C
:10F9C0009CE7079802C80790009509A82246D3E64D
:10F9D000079901C9079109990A9A089E02E0401CFB
:10F9E000002E8BD40378002B88D00B9D6C1C944286
:10F9F000F5D84B55761C0C960B94F0E7079802C887
:10FA000007900096019509A80A222346F9F71EFAE5
:10FA100074E7079B10CB102C079308D300202146D6
:10FA2000401C0A09FF291146FAD806280AD80820DE
:10FA300009E02368099CA354089A521C0C920B916C
:10FA400007905BE7401C069009230C980B9D0999D1
:10FA500005910A9E04940DE0202104463046059E3F
:10FA6000715506462046049C401C154601460891E7
:10FA700000290AD45B1E0699994206D26A1CB2423A
:10FA8000EAD9089908910029F4D50C900B950898AB
:10FA9000002800D532E70126082501E06D1E360159
:10FAA000022DFBD220463146F0F714FB0F28F6D882
:10FAB0000C980590099803900A9806900B9D204693
:10FAC0003146F0F707FB691C069A914204D9089960
:10FAD000089100290CD511E00C4A125C039B5A5581
:10FAE000089A521C0D46059211460891002905D42A
:10FAF0007043241A3009102E0646E0D205980C9067
:10FB00000B95FBE620460DB0F0BDC0461422010067
:10FB100070B588B00022032803D9D243104608B03C
:10FB200070BD7F4CC34D2A510F4B104EEE508123B8
:10FB30001E010123AB5528602C1962600128EDD805
:10FB400007930022069205920492032303930292E4
:10FB500001920091411E8841694600F027FD02464E
:10FB6000104608B070BDC04604080000FFC0FFC0CA
:10FB7000F0B583B00C460023D943012C56DB074671
:10FB800002910126EFF31085354002D1EFF310808A
:10FB900072B65849584A505C002800D0A3E0565429
:10FBA0005E48115A5E48105A0196F202161A8142B6
:10FBB00040D832465218A24240DB00930295A6423A
:10FBC000354600DB25464C490818001D39462A46B3
:10FBD000F0F7D0FAA642484E04DA7919621B301DBC
:10FBE000F0F7C8FA4E48305A001981B24D4A914296
:10FBF00001D94D494018029D009B49497052304639
:10FC00004A4E805D002865D1EFF3108501980540CC
:10FC100002D1EFF3108072B6374A4048115A40487B
:10FC2000105A884232D1424813524FE00C462046C7
:10FC300003B0F0BD42425218A242BEDA3B4A2E4EF9
:10FC4000B25C002A0CD03A4AB25A51188AB2354CEA
:10FC5000A242284C029F01D9334A8918304A02E057
:10FC6000244C2F4A029F3355B152421A89B288421E
:10FC700002D22C488018421C93B22F4801212FA297
:10FC800000F0E8F83C46002DD1D128E0019F9755BF
:10FC9000884201D82348401C421A90B2800A01D001
:10FCA000019882022248144F3A52386801280DD830
:10FCB000431E9841104B5918091D92B21D4B00F07C
:10FCC0008BFE009B002801D00B488355002D029D20
:10FCD00000D162B6074808490B54002DA7D162B67F
:10FCE000204603B0F0BD21200201044804A108A36E
:10FCF000FFF754F80E080000C0E001020E300100CA
:10FD000074726163655F6F757470757400000000D4
:10FD10005452414345204255535900000A080000FF
:10FD200008080000FF07000000F8FFFF0F080000B0
:10FD30000C08000081FF000002FF00000D0A547251
:10FD400061636520627566666572206973206675F9
:10FD50006C6C2C2064697363617264732025752058
:10FD600062797465730D0A00F0B587B00546002608
:10FD700006960596049603960296800701D007B072
:10FD8000F0BD019102A8142126A2FCF731FF2949F8
:10FD90000968012911D80029274900D027490028DE
:10FDA0000BD002AA01E0002807D04B699B07FAD5C7
:10FDB00013780B60401E521CF5E701990029DED034
:10FDC000204C3746B8002B58D80724D0581EA042E4
:10FDD00004D31B4818181C4A90421CD802A81421AE
:10FDE0001AA2FCF705FF13490968012911D8002957
:10FDF000114900D0114900280BD002AA01E00028C7
:10FE000007D04B699B07FAD513780B60401E521C34
:10FE1000F5E7761C01997F1C8F42B0D2322ED1D3E8
:10FE2000ADE7C0460D0A4261636B74726163653A67
:10FE3000200D0A00C0E001020090014000A0014036
:10FE4000FFFFFFFCFFFF0200FEFF010025303858D6
:10FE50000D0A000081B0F0B5C4B00E4607464993C4
:10FE6000812000012F49085C002845D00292012022
:10FE7000050204A82946F0F796F9FCB20021C84310
:10FE80000C2C3AD8721E032A37D82748005DB0429E
:10FE9000084632D3F80535D50021B8050DD404A89D
:10FEA00001904018691AA20022A39B582E4AFCF721
:10FEB0009FFE0198F0F78CF9014678050ED404AF47
:10FEC0007818691AB20029A3D218121F1368264A9B
:10FED000FCF78EFE3846F0F77BF90146029A04AE35
:10FEE00070180C46691A49AB0393FFF72DFC0119F2
:10FEF0003046FFF73DFE00E0002044B0F0BC02BCFD
:10FF000001B00847FEF7E8FE034604A8019007A2E7
:10FF10002946FCF76DFE0198F0F75AF90146B8053D
:10FF2000BDD5CAE7C0E00102404801002531307567
:10FF3000207C2000B22F01000830010002300100B7
:10FF4000E12F0100AC2F0100CD2F0100FB2F01009C
:10FF5000F42F0100EF2F0100A52F0100B82F0100A1
:10FF6000C82F01009D2F0100C1380100E72F0100BB
:10FF7000D32F0100DA2F0100BE2F01000000000086
:10FF8000F0B581B00B460120EFF31084044002D19C
:10FF9000EFF3108172B6990F07D0022001212DA234
:10FFA000FFF758FF002C3DD141E02249224D0027A8
:10FFB0006F54224AAB5A224AAE5AF3189EB2F60A3E
:10FFC00001D0204E9B19AB52EFF31086064002D1B0
:10FFD000EFF3108372B6AA5A1C4BEB5A934202D12C
:10FFE00016482F521AE06854934201D8164B5B1CF6
:10FFF0009B1A99B2890A00D0830210482B522868B4
:020000040001F9
:1000000001280BD8411E8841A918091D9AB2104B2E
:1000100000F0E2FC002801D006482F54002E03D047
:10002000002C04D001B0F0BD62B6002CFAD162B64B
:1000300001B0F0BD0F080000C0E001020C08000094
:100040000A08000000F8FFFFFF0700000808000092
:1000500081FF000055415254204572726F72202575
:10006000780D0A0010B50446FEF7EEF8A08A0028C5
:1000700000D010BDFDF7EAFE034908620861486C34
:10008000401C486410BDC0463099010210B50446BA
:10009000FEF7DAF8A08A002800D010BD0A4CA06C48
:1000A000401CA064FDF7D2FE6062606C002805D0A1
:1000B000FDF7CCFE60650020606410BDA06920657E
:1000C0000120606410BDC046B096010210B50A2040
:1000D00000242146FBF7D4FC09202146FBF7D0FC85
:1000E0000124204600F038F80E200421FBF7C8FC5C
:1000F0000549204600F05AFAA2021549154B204640
:1001000000F028FB10BDC046DC940102B0B50E2003
:1001100000242146FBF7B4FC0D202146FBF7B0FC80
:100120000124204600F018F80A2004252946FBF790
:10013000A7FC09202946FBF7A3FC2046F9F77AFA29
:10014000A2020349034B204600F004FBB0BDC046A9
:10015000E0CD01028D09010070B5012801D901200F
:1001600070BD48224243734B9C58A5691F218D43A3
:10017000A5610625A5600F2525629C18A27C002A92
:1001800005D1627C002A02D1227C002A14D0636847
:10019000002B11D4251D0B40012216469E400C4B0E
:1001A0001E60BFF34F8FBFF36F8F2B68002B03D4FC
:1001B0000B409A4007490A60002803D0012804D167
:1001C000092000E00820F9F7DFFB0020A06170BDE6
:1001D00080E100E080E200E0F0B585B00D460278F5
:1001E000E348C368934219D0446D944216D08368A3
:1001F000934203D0016D914200D07FE09B1A591EBB
:100200008B41049348215943032D46D14418E16999
:1002100000294ED01C34002020606DE09B1A5A1E2D
:1002200093410493032D1AD1039548225A4384180D
:10023000A26B0121EFF310850D4002D1EFF310877F
:1002400072B6A7691026B743A761A669002E01D12F
:1002500018342160002D00D162B6039D0CE04821C6
:100260005943421891691832302902D01168102977
:100270004CD18021116000224821594340180021AF
:10028000816301628162243000210160002A33D041
:1002900004A82946904705B0F0BD4218916918326C
:1002A000302902D01168202939D180211160002223
:1002B00016E00395E26B0126EFF31085354002D17D
:1002C000EFF3108172B6A1692027B943A161A1693A
:1002D000002901D118342660002D00D162B6039D9B
:1002E0004821594340180021C163C1624163303045
:1002F00000210160002ACBD105B0F0BD00920E4A6A
:100300002E329C480D490E4BFEF748FD10680093B5
:10031000019098480949084A0A4BFEF73FFD1068CA
:1003200000930190044A243292480449054BFEF799
:1003300035FDC046FC940102B10200008A30010084
:100340005F30010043300100F0B585B004904821D2
:100350000A464243864B9C58E6690F2535409A1859
:10036000167C002E31D04F2040026169014200D13D
:1003700085E0A06904218843A06102202062012059
:1003800081076918D161D36BEFF31084044002D167
:10039000EFF3108572B695692026B543956195698E
:1003A000002D00D173E010463C30002C00D162B625
:1003B00000240460D4625463303200201060002BAB
:1003C00063D004A8984705B0F0BD0C2D5DD8C04699
:1003D0007D442D796D00AF4467586B580658A16372
:1003E0005858585806009569202D04D015461835E0
:1003F0002D68302D49D1156B566B3432AE4217D271
:100400006669360714D5646815686E1C1660484323
:100410001818C06A445504980C4644431A19156BC1
:10042000566B3432AE4203D21C5966693607EAD4A1
:100430001268AA4229D14143585882690524A2432F
:1004400082615A18D36B0121EFF31080084002D16A
:10045000EFF3108472B694692025AC4394619469DB
:10046000002C02D114461834216014463C34002874
:1004700000D162B600212160D16251639CE70C2D4E
:1004800000D176E7012D00D173E705B0F0BD154628
:100490001835286010463C30002C00D187E787E7EC
:1004A0000420206205B0F0BD0120206205B0F0BD3F
:1004B00008252562164618369569102D02D0356834
:1004C000302D4BD10396566A15462835976AB742A8
:1004D00028D1A06902218843A061936B0121EFF329
:1004E0001080084002D1EFF3108472B6039E346886
:1004F0001027BC4334603468002C00D131601446AE
:100500003834002800D162B60021216029601162D0
:10051000243200201060002BB7D052E70220206266
:1005200005B0F0BD2A68B242AFD262699207ACD57D
:100530002A68561C2E6048431818006A805C2060A8
:1005400004980A4642439D18AC6A6E6AB4429CD233
:1005500028359C5862699207EAD496E73168009082
:100560000191044804A1094A09A3FEF717FCC046FB
:10057000FC94010229300100756172745F69727127
:100580005F68616E646C6572000000003D030000EE
:100590005561727420256420737461746520676FDF
:1005A00065732077726F6E6720256400F0B585B0A3
:1005B0000E460546022804D3002E02D1012005B0C4
:1005C000F0BD002D03D0012D08D1092400E008243E
:1005D0002046F9F7E1F92046FEF7B4F848216943CF
:1005E000E74A505883691F240294A343836106237A
:1005F00083600F230193036257180023BB62BB6320
:10060000FB633B627B62FB623B63317F3974727FC9
:100610007A74B27FBA7404937B637368B268F468C7
:10062000920022435B1E032B0ED8C0467B441B79ED
:100630005B009F4401050307082304E0282302E030
:10064000182300E038231A43C260C907090F7269F2
:100650009201D2B28918B2699207920E8918491C88
:10066000816079613169012901D122210161012D66
:100670005CD831680E2959D23846123003900324D1
:10068000002D01D0204600E004204C432D490E19D6
:10069000B178F9F711FA3968CA68802510462843FD
:1006A000C8602848005D73781B021818C862AA4306
:1006B000CA60F9F749FA03980078002809D138464A
:1006C00011300078002804D1384610300078002816
:1006D00027D07868002815D4032102468A431B4995
:1006E00053588407E40EFF26A640B343A5401D439C
:1006F00055500299014001208840A24908601449E0
:1007000008600EE08107C90EFF228A40019C044068
:10071000083C032084430C48235893438D401D43D9
:1007200025500120B861049805B0F0BD0248034986
:10073000DA22034BFEF732FB293001009C30010026
:1007400079300100A81F01001CED00E000E400E08A
:1007500000E100E0F0B58FB00E900125002900D136
:100760004BE0039304910592002A00D145E001215A
:10077000EFF3108201910A4002D1EFF3108172B6BB
:100780004827029747437E49CE19B5690023302D8B
:1007900023D831461831C0467D442D796D00AF44D1
:1007A00020242626262626262626262626262626F1
:1007B0005E262626262626262626262626262626A1
:1007C00018262626262626262626262626262626D7
:1007D00018000223002A0CD00CE0402D01D0802DFF
:1007E00005D10123002A04D004E020240C60002A53
:1007F00000D162B61D46002B02D028460FB0F0BDD6
:10080000002575630399F1630499F16205993163D9
:100810005B4CE35959691322D202114205D00621DB
:1008200099600F21196271699960317C00290CD09F
:10083000F56109950895079506950D950B9502218B
:100840000A91012810D017200FE0717C9A690029C5
:100850002CD0952002439A6128460FB0F0BD302479
:100860000C60002AC5D0C5E71920049F0C90706861
:10087000002805D41F2108400199814041480160AA
:1008800014209861B06806A9F9F7CEF90E9802997C
:1008900041436018806861583B4A0092091D3A46FE
:1008A000059BF9F731FA28460FB0F0BD3436110632
:1008B00002D580218A439A6131680025059A9142C8
:1008C0002DD205955D694F214A0215421BD1E905DC
:1008D00002D4029CF24F0AE0596833685C1C346011
:1008E000029C6043EE4F3818C06AC1540E982146EE
:1008F00041437E18736B346BA34238D234367B5835
:100900005D691542E3D002211962019EB1072943B6
:100910003546E34CEFF31082324006D008E029461A
:10092000019EEFF31082324002D1EFF3108372B6D2
:10093000029B4343E01883692024A34383618369B6
:10094000002B05D0002A08D0C26B002A0AD154E738
:10095000034618331E60002AF6D162B6C26B002A25
:1009600000D14AE70EA8904728460FB0F0BD2946AF
:10097000059D019E3C46EFF310823240D5D0D7E76B
:10098000FC94010280E200E0D901010080B5012061
:1009900082020249024BFFF7DDFE80BDE0CD01027D
:1009A0008D090100B0B582B079208400E54D285D45
:1009B00001A90870652080002818F3F70DF82F2092
:1009C000C000285829190122024BFFF7C3FE02B0CC
:1009D000B0BDC046A5090100F0B591B01090012648
:1009E000002900D19BE003930591002A00D196E0F5
:1009F00007900121EFF310800291084002D1EFF33C
:100A0000108172B604924823069307994B43D64946
:100A1000C9188D690026302D6ED80C461834AD00EB
:100A2000374602A675593E46AF46C046010B010047
:100A3000090B01000D0B01000D0B01000D0B010056
:100A40000D0B01000D0B01000D0B01000D0B010042
:100A50000D0B01000D0B01000D0B01000D0B010032
:100A60000D0B01000D0B01000D0B0100F10A01003F
:100A70000D0B01000D0B01000D0B01000D0B010012
:100A80000D0B01000D0B01000D0B01000D0B010002
:100A90000D0B01000D0B01000D0B01000D0B0100F2
:100AA0000D0B01000D0B01000D0B01009F0B010050
:100AB0000D0B01000D0B01000D0B01000D0B0100D2
:100AC0000D0B01000D0B01000D0B01000D0B0100C2
:100AD0000D0B01000D0B01000D0B01000D0B0100B2
:100AE0000D0B01000D0B01000D0B0100F10A0100BF
:100AF000022600280CD00CE0402D01D0802D05D11D
:100B00000126002804D004E010252560002800D12B
:100B100062B6002E069D944F049C079802D0304682
:100B200011B0F0BD00268E62039A8A63059A0A62AC
:100B30004C620A7C002A0BD00C960B960A960996FA
:100B400008960E9602220D9201282DD018202CE036
:100B50008A7C2831002A3BD00A68A24216D22B4652
:100B60004343FA585469A40710D50868441C0C6024
:100B7000F918096A085C10601098294641437A18F0
:100B800011462831936A526A9342E8D34543785913
:100B9000816982220A438261304611B0F0BD30255E
:100BA00025600028B4D0B4E71A200F90C86808A9BF
:100BB000F9F73AF8109845437A597819C0683949D5
:100BC000009105992346F9F79FF8304611B0F0BD22
:100BD000FB589A69140602D58024A2439A610A68D8
:100BE0000026049882422ED25D694F22520215429D
:100BF00007980AD002211962029EB10729431FE01B
:100C000028315D6915423E46F4D137465C69A40738
:100C100002D40699544E0AE00C68661C0E600699D0
:100C20004843514E3018006A005D186010984143E7
:100C3000735871188C6A4E6AB442E1D329463E4615
:100C4000069D494F01E0314607985A6A002AFCD1B7
:100C5000EFF31082029B1A4002D1EFF3108372B6B9
:100C60004543781983691024A34383618369002B6A
:100C700005D0002A09D0826B002A0BD14FE703462A
:100C80001833029C1C60002AF5D162B6826B002AE0
:100C900000D144E710A89047304611B0F0BDC046DF
:100CA000FC940102D9010100B0B5264900684A68E8
:100CB000824202D10D1D002016E080228A58824215
:100CC00003D10D46803501200EE0FC228A58824275
:100CD00003D10D46FC35022006E02F22D2008B58AE
:100CE00083422ED18D1803207C2242438C18A068A9
:100CF000012814D0002824D140342046F3F75BFAB1
:100D000001462046F3F72DFA2046F3F754FA00285F
:100D100017D006C828680C4BFFF75EFEB0BD403404
:100D20002046F3F748FA01462046F3F71AFA204620
:100D3000F3F741FA002804D006C82868024BFFF7F1
:100D40004BFEB0BD58BE0102A90C01004821414331
:100D5000054842189269D20601D4002070474058D5
:100D60004169012008407047FC94010280B5114898
:100D70000078C00110490978890101430F480078C3
:100D8000400108430E490978090101430D480078E4
:100D9000C00008430C490978890001430B480078DA
:100DA000400008430A4909780143C8B2F3F7B4FC8C
:100DB00080BDC046E09E0102AE9601021D90010278
:100DC00064EA010299AD0102E19E010224A301023D
:100DD00025A30102F0B587B00146012702250528A9
:100DE0003A4600D02A4600200929014600D0114683
:100DF000C900374A54180E210591615EFDF7AEFA1D
:100E00001026A15F3846FDF7A9FA1227E15F2846B0
:100E1000FDF7A4FA06951425615F03200490FDF701
:100E20009DFA0598235EA05FE15F625F00AD07C594
:100E300028A2069F3846049D2946FFF70BF8204656
:100E4000263004263146FBF749FF2620235E282062
:100E5000205E2A21615E2C22A25E00900191029206
:100E600024A238462946FEF7F5FF27463E37384686
:100E70003146FBF751FF3E20235E06983C5EB95F8A
:100E80000622BA5E00940191029221A207462E46E4
:100E90002946FEF7DFFF56240D4D285FFBF730FF94
:100EA0002B5F2C4621A2384631463546FEF7D2FF4D
:100EB000264658363046FBF70FFF5820235EF05F7A
:100EC00000901FA238462946FEF7C4FF07B0F0BDC8
:100ED000C4A00102546F4620616E742064656C6189
:100EE00079732025642025642025642025640D0A5B
:100EF0000000000050446F412064656C61797320EC
:100F000025642025642025642025640D0A00000046
:100F100050446F41206761696E7320256420256409
:100F20002025642025640D0A0000000050446F4114
:100F300020616E742073706163652025640D0A0062
:100F400050446F4120616E676C65206F6666736503
:100F500074732025642025640D0A0000F0B587B065
:100F600015467A4B1A680F24A2432F783A431A6029
:100F7000774C23462C3B774A1A600490034622465E
:100F8000283A12681207FAD5734E092F029306D930
:100F9000754A326072600C2F09D175480FE0042F3A
:100FA00007D9704A3260704A7260092F06D37148BF
:100FB00005E06A4830607060694800E06B486E4A3E
:100FC0001060EB7AFF2B039102D10020B0620AE09F
:100FD00003210B406948C05C40220243B2620220F8
:100FE000674AFEF737FF029F0021384605952A46DB
:100FF0000B46FBF7FDFE06460225032161A22846AB
:1010000001913346FEF726FF06963046FCF7C4FBF7
:1010100001210498009108402CD13D4033D1604912
:1010200000283AD1002D1ED06548A062E0622063FE
:1010300060636448606264480860152085046E1C23
:101040008E608D60642420460F46F8F77DFD3E607B
:101050003D602046F8F778FD281D386003215BA22B
:101060004E48FEF7F7FE0598007BFAF7CFFF06988B
:1010700007B0F0BD2E4605460698FCF719FF284636
:1010800035463D40CBD02E4605460698FCF78CFBF6
:101090002846354642490028C4D0424808614248A3
:1010A0004861424888611520C86141480168402272
:1010B0000A43026007210803274B5A6982430098BC
:1010C0004003101858610522039842432A480368D8
:1010D0009818334E766B47780F40995C0907490E94
:1010E000C919CA03334B33409A18C9015118324AFF
:1010F00089182B4A51632A49896B38229143827897
:101100005207920E891804220A4325498A63124B1A
:1011100019690279019E3240C0784007C00E8018DC
:101120001F2291430818186155204003411C21607B
:1011300020606420F8F708FD204A18483146039BD8
:10114000FEF788FE1649002D8DD06DE7040400409F
:101150002C60004000040080000600400F040F04D3
:10116000312A01000304030400040004622B01007F
:1011700000290100932C010048940102C42D0100B4
:10118000C830010050485920706172616D7320733E
:1011900065747320253038780D0A000002080000BD
:1011A0009060004012A83E009DD79B5AD579BD495A
:1011B000340200403F0080FF40400000AA300100A0
:1011C0002008820002D50F00020255007577625F89
:1011D00072785F696E69740D0A00000080B522485C
:1011E0000021017022480078C00120490978890156
:1011F000014320480078400108431F490978C9008D
:1012000001431E480078800008431D4909784900C1
:1012100001431C4800780843C0B2F3F77DFA80BD53
:1012200080B51148012101701048007880011049F3
:101230000978C90101430F480078400108430E496D
:101240000978C90001430D480078800008430C4923
:101250000978490001430B480078084310210143F5
:10126000C8B2F3F759FA80BD64EA0102AE960102F2
:10127000E09E01021D90010299AD0102E19E010272
:1012800024A3010225A30102F0B581B01820FDF7C7
:1012900059FA1920FDF756FA002420462146F8F79E
:1012A00027F820462146FAF735FE012603257F233D
:1012B000304629462A46FAF745FF3046FBF7EAF85A
:1012C00002273846FBF774FD30463146FCF7C2FD75
:1012D00003A238462946FEF7BDFD204601B0F0BD09
:1012E0007577625F6F70656E0D0A0000F0B581B0B2
:1012F000164600910446002001273946FCF7D2FF2C
:10130000EFF310853D4002D1EFF3108072B6272035
:10131000400170430A21EEF7DDFE0246002C02D0A8
:101320000020009901E002200021FBF7B9F80446F3
:10133000FBF780F9002D00D162B6204601B0F0BD68
:1013400070B504460E4D29680F2001400629FAD0D9
:1013500029680140072912D10120EFF310860640C9
:1013600002D1EFF3108072B6FCF770FDFA30A8607E
:10137000002C01D0FAF7E0FE002E00D162B670BD5D
:1013800000040040F0B581B01D460E460446022A16
:1013900009D1012738463946FCF784FF0096002220
:1013A000384629460FE0174601200021FCF77AFF56
:1013B000012F04D1009600202946024603E0009642
:1013C000022000210A462346FBF74CF90446FBF7AE
:1013D00031F9204601B0F0BD70B5002801D00120E0
:1013E00070BD0325A9020F4802680F4B535000241B
:1013F0009460012253030D4E3360BFF34F8FBFF350
:101400006F8F0B4E336003685A5084720481102032
:10141000F8F7BAFA022007A22946FEF71BFD20467C
:1014200070BDC0468C95010251E5CC1A80E100E008
:1014300080E200E057445420636C6F73650D0A002E
:101440000FB47CB50C0009AD01D0611E00E0002195
:1014500001910090074B6A462946089800F012F95E
:10146000002C02D0009A002111707CBC08BC04B092
:1014700018470000BD1D01007CB51D4616460C0036
:1014800001D0611E00E0002101910090054B6A46E9
:101490002946304600F0F6F8002C02D0009A0021D0
:1014A00011707CBDBD1D01002021020C01D0102156
:1014B0001046020A01D010460839020901D0104630
:1014C000091F820801D01046891E420801D0881EDB
:1014D0007047081A704700000048704708900102E2
:1014E00002E008C8121F08C1002AFAD170477047ED
:1014F000002001E001C1121F002AFBD1704700004B
:10150000F0B51FB486B00998089A030D0021024374
:1015100014D05148514A1818504305141198012805
:1015200010981AD0281A401C00264D4F4D4900969D
:1015300001910490002812DA444211E0119801242C
:1015400049A3012801D11098C1430698119A8460DB
:101550000360C26041600BB0F0BD4042E4E7044666
:10156000210500203F4A001C51410391029012E0E6
:10157000E00707D032463B4601990098EFF772F832
:101580000191009032463B4610461946EFF76AF843
:1015900006460F466410002CEAD10498039B0028ED
:1015A000029A0999089806DAEFF75CF8019B009A0D
:1015B000EFF758F805E0EFF7BDF8019B009AEFF759
:1015C000B9F804460E460022284BEFF77FFC03D8FB
:1015D0000020C043014607E00022254B204631464B
:1015E000EEF78EFFEFF752FC102409E0002C0ADB27
:1015F0000A220023EFF77CFA079B30321A55641E4B
:1016000002460A43F2D11122641C079B121B1C19CB
:10161000119B012B03D0012308430ED10AE008439C
:1016200004D0112010900020119077E71098151A1F
:101630006D1E0BE01098824202DD00236D1C03E05A
:10164000824201DA00236D1E002BEED0069811991C
:101650008260C16030C07EE701FCFFFF104D0000DA
:10166000000014400000F03F300000000000F04394
:101670000000E03F30380A2801D2012070470020E6
:1016800070470000FFB597B00646002518E22528F0
:1016900077D100242746FD49049400E00443761CDA
:1016A00032780120203A90400842F7D130782A2839
:1016B0000ED00222307801463039092916D8049913
:1016C0000A235943303940181443761C0490F1E73B
:1016D000189802C804911890002904DA01204003E8
:1016E00004434842049002200443761C30782E289C
:1016F00014D1042004437078761C2A2809D1189844
:10170000761C80C8189009E00A214F43303FC71962
:10171000761C3078014630390929F5D930786C28A3
:1017200010D006DC4C281AD068280ED06A2817D1B1
:1017300004E0742813D07A2812D110E0012040056B
:1017400004430CE00121090501E0032109050C43D4
:101750007178814203D1012000052418761C761C83
:101760003078119066280BD013DC58287DD009DC26
:1017700000287BD04528F6D04628F4D047281AD137
:10178000A5E118E0632835D0642870D0652812D10F
:101790009DE170286CD008DC6728F1D069287BD0E7
:1017A0006E280DD06F2806D1BAE073282ED0752888
:1017B00071D0782859D01A9A199990476D1C7EE1FA
:1017C0006002400F022809D003280DD00428189881
:1017D00001680DD00D60001D189070E11898EA178F
:1017E00001680D604A60F6E7189801680D80F2E71D
:1017F0000D70F0E718986A4601781172001D189074
:101800000020507202A80090012005E0189802C83C
:10181000189000200091C04361070DD5002101E020
:101820000199491C0191B94212DA8142F8DB009A10
:10183000515C0029F4D10BE0002101E00199491C21
:1018400001918142FADB019A0099895C0029F5D166
:10185000019904981A9B471A21463846199A00F0B4
:1018600097FA0199401945180BE04FE02CE113E07D
:101870004EE0009800990078491C00911A9A199935
:1018800090470198401E0190401CF2D121463846F5
:101890001A9B199A10E137E00A200021009001916B
:1018A0006002410F022907D0189A01CA1892C21784
:1018B0009446032908D00AE01898C01DC108C90041
:1018C00005C91891944607E000B2C217944604294E
:1018D00002D140B2C1178C4600226146944506DA17
:1018E0000A460021404291418C462D2102E021050B
:1018F00004D52B216A461173012103E0E10701D0D1
:101900002021F7E7029155E00A200AE0102008E0C4
:10191000102000900021042004430191082703E0D7
:1019200008200021019100906002410F022907D098
:10193000189A01CA189200229446032908D008E098
:101940001898C01DC108C90005C91891944603E044
:1019500080B2042900D1C0B200210291210729D50B
:101960001199702906D0009A1021019B4A401A4310
:1019700005D00EE040216A461173012108E061465E
:10198000014306D030216A46117311995173022127
:101990000291009A0821019B4A401A430AD16146EC
:1019A000014301D1610705D530216A461173012138
:1019B0007F1E02911199582904D035A10E910DA9CD
:1019C0000D910DE037A1F9E76146019B009AEFF711
:1019D0008FF80E9B8C469B5C0D9A521E0D921370D5
:1019E00061460143F0D10D9805A9081A20300190F5
:1019F000600703D501200004844300E0012701981B
:101A0000874201DD381A00E000200199009041185A
:101A1000029809180498401A0490E00306D421465D
:101A20001A9B199A049800F0B3F94519002706E0AB
:101A300003A81A9AC05D199990476D1C7F1C0298E3
:101A40008742F5DBE0030CD521461A9B199A0498CE
:101A500000F09EF9451904E01A9A30201999904730
:101A60006D1C0099481E00900029F5DC08E00D98D7
:101A70000D990078491C0D911A9A199990476D1C7F
:101A80000199481E01900029F1DC63E10928010059
:101A900030313233343536373839616263646566E4
:101AA00000000000303132333435363738394142A6
:101AB000434445460000000000F05AF94519761CE1
:101AC0003078002800D0E2E528461BB0F0BD600762
:101AD00000D406271898C01DC108C90048680A68C4
:101AE0000831C30FDB071891190001D09CA108E051
:101AF000210501D59BA104E0E10701D09AA100E0F6
:101B00009AA1430011985B08109165280CD006DC5F
:101B1000452809D046281DD0472841D141E06628F4
:101B200018D067283CD13CE00021112F01DB1120A7
:101B300000E0781C0191009008A911A8FFF7E0FCD3
:101B4000139905910021119A15927F1C1298019703
:101B5000009150E00120C00703900120019008A9E6
:101B6000009711A8FFF7CCFC139A14990592002254
:101B7000119B009212981593059A0192002901D0A9
:101B8000104602E0791C40180190381A01D50198DE
:101B900004E04042401E0090781C0190C01B02905F
:101BA00043E0012F00DA01270021112F01DD112070
:101BB00000E038460191009008A911A8FFF7A0FCA9
:101BC00013990591119A002112981592009101978D
:101BD00021070CD40599B94201DB019900E001917C
:101BE000012904DD159A491E515C302906D0B842FE
:101BF00001DA011D05DA0121029115E00199491E62
